S00A000039304D2E53313954
S21401000000FC002041BB0200250802002508020072
S214010010250802002508020025080200000000004D
S2140100200000000000000000000000005504010070
S2140100302508020000000000EF0401002508020068
S21401004025080200250802002508020025080200EE
S21401005025080200250802002508020025080200DE
S21401006025080200250802002508020025080200CE
S21401007025080200250802002508020025080200BE
S214010400FFFFFFFFFFFFFFFFFFFFFFFFFEFFFFFFF7
S21401042001DF704701DFFFF7FEBFD048006872B6F4
S214010430018B39B9416AC269D369994200F00280D9
S21401044062B603DF62B6704703DF7047FFF7FEBF91
S21401045002DF704772B61EF0040F0CBFEFF308817F
S214010460EFF30981896911F8021C032940F007801E
S21401047000B500F02CF85DF804EB00F026B8012971
S21401048040F00480B948006800F059B8022940F0ED
S2140104901C80B6480068C1698A6842F001028A6019
S2140104A000B502B4016C11F0010F00F0058000B533
S2140104B023F0BCFA5DF804EB02BC4A680B681360D3
S2140104C05A6000F004F85DF804EB62B6704707B5B1
S2140104D0A748416811F0805F40F00880EFF3118271
S2140104E0A2F1100280F82220A249416007BD72B62F
S2140104F09E480068EFF3098C9F498A78EFF31183D1
S2140105002CE9FC4FC369C3F814C0996A11F0020FB5
S21401051000F01580D3F834C0984A52F8041B4CF802
S214010520041B52F8041B4CF8041B52F8041B4CF82D
S214010530041BF1EE101A4CF8081B8CEC200A72B65C
S214010540416A0A688A4240F00580896809007FF49A
S214010550F8AFFEE74162C261938C4383916A11F062
S214010560020F00F01A80836C9A4200F016808264B3
S214010570D2F834C0814C5CF8043B44F8043B5CF888
S214010580043B44F8043B5CF8043B44F8043B5CF849
S214010590083BE1EE103ABCEC200AD2F814C0BCE8E5
S2140105A0FC4F83F311888CF3098802B4016C11F0B7
S2140105B0010F00F0058000B523F0C4FA5DF804EBE6
S2140105C002BC02B400B521F043FB5DF804EB02BCAB
S2140105D067486B49416062B6704772B600B5634BB7
S2140105E01B68198B01F101011983664801B4EFF309
S2140105F01182EFF30581586B07B4EFF30880586357
S2140106000846196C11F0010F00F004800FB423F0B6
S214010610E3FA0FBC1A6B0AB900F042B8904200F236
S2140106203F80DA6A811AC0F23B809A6B4FEAD101A9
S2140106304FEA8101515809B900F032B80A6832B15F
S214010640824200F00680096909427FF4F7AF00F0A4
S21401065027B8C8684A6808B462B6904772B608BC3C
S214010660196C11F0010F00F00680EFF305800FB44E
S21401067023F0F4FA0FBC07BC586301BC198B01398F
S2140106801983DA69906A10F4805F40F00C8029B90A
S214010690596A0968914218BFFFF719FF62B600BD93
S2140106A09A6AFFF7D8BF40F40030906262B600BD88
S2140106B072B6F1B42D4B1B68D3F834C00CF1100C94
S2140106C05CF804EB304820F00100CCF818009CE8F8
S2140106D0FF005DF804CBACF1040C27F400772CE99D
S2140106E0FF00F0BC8CF3088862B670471F480068AC
S2140106F0C369996AD3F834C0204A52F8041B4CF8EF
S214010700041B52F8041B4CF8041B52F8041B4CF84B
S214010710041BF1EE101A4CF8081B8CEC200A7047EB
S2140107204FF08002D0E84F1F00290CBFC0E8432FCE
S21401073000F003B8002B7FF4F5AF08467047EFF3DF
S21401074009807047EFF30880704780F30888704788
S214010750EFF30380704762B6704772B67047704613
S214010760704778467047EFF3148070470C06FF1FFA
S21401077000ED00E00000001020ED00E034EF00E0A6
S21401078000000008000000005C06010010B5054CE2
S214010790237833B9044810B10448AFF3008001212F
S2140107A0217010BD3006FF1F0000000030980300C6
S2140107B008B5064B1BB106480649AFF3008006484C
S2140107C0016811B1054A02B1904708BD000000005A
S2140107D0309803003406FF1F3006FF1F000000009C
S2140107E080B586B000AF786039604FF00003FB73C8
S2140107F04FF000033B6140F63D33C1F6FF734FF007
S21401080000021A7007F10F03786839681A460FF06C
S21401081053FE0346FB75FB7D83F00103DBB2002B21
S21401082011D07B68012B0CDD4AF61060C0F2030084
S2140108301BF07AFB4FF0FF333B614FF00103FB7572
S21401084001E001F053FEFB7D002B15D0FB7B002B56
S21401085009D03B681B684AF63860C0F203001946A7
S2140108601BF062FB08E03B681B684AF64060C0F27A
S214010870030019461BF058FB3B69184607F1180799
S214010880BD4680BDF0B58DB002AF786039604FF0DF
S21401089000037B754FF000033B6240F63D33C1F623
S2140108A0FF734FF000021A7007F115037868396874
S2140108B01A460FF001FE034687F8273097F82730CF
S2140108C083F00103DBB2002B00F05A817B68012B19
S2140108D00DDD4AF61060C0F203001BF025FB4FF059
S2140108E0FF333B624FF0010387F8273048E14FF0B2
S2140108F00003FB77A9E0FB7F03F14101FA7F40F695
S214010900C823C1F6FF7333F812301A46F87F40F653
S2140109107423C1F6FF7333F810304AF64C60C0F208
S21401092003001BF001FB4FF00003BB837EE0BB8B93
S21401093003F101034AF66C60C0F2030019461BF08E
S214010940F3FAF87FB98B41F25012C1F6FF720B46EB
S2140109504FEA43035B184FEA83034FF4965101FBBA
S21401096000F15B18D3181B68FB60FA684FF00303AD
S214010970C0F200139A420BD9FB6803F17F43A3F13F
S2140109800403FB604AF68060C0F203001BF0CCFA59
S214010990FE68F87FB98B41F25012C1F6FF720B4622
S2140109A04FEA43035B184FEA83034FF4965101FB6A
S2140109B000F15B18D3181B791D46F87FB98B41F2FD
S2140109C05012C1F6FF720B464FEA43035B184FEA1B
S2140109D083034FF4965101FB00F15B18D31803F122
S2140109E001031B791C46F87FB98B41F25012C1F600
S2140109F0FF720B464FEA43035B184FEA83034FF43B
S214010A00965101FB00F15B18D31803F102031B7921
S214010A1000934AF68860C0F2030031462A46234610
S214010A201BF082FABB8B03F10103BB83FA7F40F60E
S214010A307423C1F6FF7333F81230BA8B9A42FFF46F
S214010A4076AFFB7F03F10103FB7740F22353C1F638
S214010A50FF731B78FA7F9A42FFF44DAF40F6B863F6
S214010A60C1F6FF731B784AF6A060C0F20300194670
S214010A701BF05AFA40F68233C1F6FF731B881A46FA
S214010A8040F6B063C1F6FF731B884AF6C460C0F235
S214010A90030011461A461BF047FA4FF43833BB6180
S214010AA002F0F2FA4FF00003BB8356E041F2F8037E
S214010AB0C1F6FF731A6807F10C031046B9694FF0C7
S214010AC0040203F0A9FF41F2F803C1F6FF731A68A6
S214010AD0BB6903F104031046194603F025FD0346DE
S214010AE0FB7541F2F803C1F6FF731A68BB6903F19F
S214010AF005031046194603F017FD0346BB7541F280
S214010B00F803C1F6FF731968BB6903F1060207F122
S214010B101203084611464FF0020203F07DFFBB693F
S214010B2003F10803BB61B98BFD68FC7DB87D7B8A48
S214010B301A4613464FEA83039B184FEA4303009075
S214010B4001934AF6F460C0F203002A4623461BF0DE
S214010B50EBF9BB8B03F10103BB8340F68233C1F68D
S214010B60FF731B88BA8B9A42A0D302F0A9FA40F60B
S214010B70B063C1F6FF731B88002B01D001F0CCFED9
S214010B8097F82730002B15D07B7D002B09D03B68CA
S214010B901B684AF63860C0F2030019461BF0C4F918
S214010BA008E03B681B684AF64060C0F2030019463D
S214010BB01BF0BAF93B6A184607F12C07BD46F0BD93
S214010BC0F0B59BB006AF786039604FF0000387F848
S214010BD033304FF00003BB644FF0000387F8473013
S214010BE04FF0000387F846304FF0000387F8453092
S214010BF04FF0000387F844304FF49673BB6307F158
S214010C003303786839681A460FF056FC034687F8AE
S214010C104F3097F84F3083F00103DBB2002B00F022
S214010C2016817B68022B14D13B6803F104031A6812
S214010C3007F10C03104619460FF0FAFB0346002B8A
S214010C4007D0FA6813464FEA83039B184FEA43031B
S214010C50BB637B68012B03D07B68022B40F0EA80E4
S214010C604FF000033B64DFE04FF0000387F84E309F
S214010C704FF00003FB6315E007F12C02FB6BD31862
S214010C801A7840F6FC63C1F6FF73F96B5B181B78A4
S214010C909A4203D04FF0010387F84E30FB6B03F105
S214010CA00103FB63FB6B042BE6D94FF47043C4F2DC
S214010CB00F031B6903F02003002B0CBF0023012345
S214010CC087F837304FF47043C4F20F031B6903F4FF
S214010CD00033002B0CBF0023012387F836304FF278
S214010CE04003C4F20F031B6903F40003002B0CBF7F
S214010CF00023012387F835304FF47143C4F20F0304
S214010D001B6903F01003002B0CBF0023012387F897
S214010D10343097F8372097F847309A4211D197F830
S214010D20362097F846309A420BD197F8352097F837
S214010D3045309A4205D197F8342097F844309A42C4
S214010D4003D04FF0010387F84E3097F84E30002B52
S214010D5034D040F6FC63C1F6FF731B78194640F6A3
S214010D60FC63C1F6FF735B781A4640F6FC63C1F676
S214010D70FF739B781C4640F6FC63C1F6FF73DB7875
S214010D809C4640F6FC63C1F6FF731B799E4697F8B6
S214010D90376097F8365097F8350097F83430CDF825
S214010DA000C0CDF804E002960395049005934AF638
S214010DB03070C0F2030023461BF0B6F84FF0000374
S214010DC0FB630FE040F6FC63C1F6FF73FA6B9B18FA
S214010DD01A7807F12C01FB6BCB181A70FB6B03F129
S214010DE00103FB63FB6B042BECD997F8373087F8CC
S214010DF0473097F8363087F8463097F8353087F819
S214010E00453097F8343087F8443040F63D33C1F624
S214010E10FF734FF000021A704FF064001DF006FFDA
S214010E203B6C03F101033B643A6CBB6B9A42FFF4E3
S214010E301BAF0CE04AF61060C0F203001BF074F81A
S214010E404FF0FF33BB644FF0010387F84F3097F83C
S214010E504F30002B16D097F83330002B09D03B6863
S214010E601B684AF68C70C0F2030019461BF05CF84A
S214010E7008E03B681B684AF6A070C0F203001946FA
S214010E801BF052F8BB6C184607F15407BD46F0BD7F
S214010E9080B588B000AF786039604FF00003FB740E
S214010EA04FF00003BB6140F63D33C1F6FF734FF0D0
S214010EB000021A7007F11303786839681A460FF0B2
S214010EC0FBFA0346FB77FB7F83F00103DBB2002BC3
S214010ED000F05E837B68012B72D14AF6BC70C0F2CB
S214010EE003001BF021F84AF6E070C0F203001BF085
S214010EF01BF84BF20800C0F203001BF015F84BF28A
S214010F002800C0F203001BF00FF84BF24800C0F2B5
S214010F1003001BF009F84BF26800C0F203001BF057
S214010F2003F84BF29000C0F203001AF0FDFF4BF2FB
S214010F30B400C0F203001AF0F7FF4BF2D800C0F27B
S214010F4003001AF0F1FF4BF20010C0F203001AF092
S214010F50EBFF4BF22010C0F203001AF0E5FF4BF254
S214010F604010C0F203001AF0DFFF4BF26010C0F22F
S214010F7003001AF0D9FF4BF28410C0F203001AF0F6
S214010F80D3FF4BF2AC10C0F203001AF0CDFF4BF2C8
S214010F90DC10C0F203001AF0C7FF4BF20420C0F2C7
S214010FA003001AF0C1FF4BF22C20C0F203001AF026
S214010FB0BBFF4FF0FF33BB614FF00103FB77E7E266
S214010FC07B68032B40F0D8823B6803F104031A6860
S214010FD007F10C03104619460FF02AFA0346002BB8
S214010FE000F0BD823B6803F108031A6807F10803A5
S214010FF0104619460FF01CFA0346002B00F0AF828C
S214011000FB68002B23D0FB685A2B20D8FA68BB68F4
S214011010002B04D04BF25023C0F2030303E04BF243
S2140110205423C0F203034BF25820C0F203001146CA
S2140110301A461AF079FFFB68DBB203F1FF33DAB226
S214011040BB68DBB2104619460DF0B2FE85E2FB68BE
S214011050642B2BD9FB68762B28D8FB68A3F1640296
S214011060BB68002B04D04BF25023C0F2030303E00D
S2140110704BF25423C0F203034BF26820C0F2030084
S21401108011461A461AF050FFFB68DBB2A3F165035E
S214011090DAB2BB68002B0CBF00230123DBB210467B
S2140110A019464FF001020DF053FD56E2FB68C82BBE
S2140110B02BD9FB68DA2B28D8FB68A3F1C802BB68DA
S2140110C0002B04D04BF25023C0F2030303E04BF293
S2140110D05423C0F203034BF27820C0F203001146FA
S2140110E01A461AF021FFFB68DBB203F13703DAB2C6
S2140110F0BB68002B0CBF00230123DBB21046194648
S2140111004FF002020DF024FD27E2FB68642B00F08D
S2140111100A81642B12D85C2B6DD05C2B04D8002B73
S21401112029D05B2B4ED018E25E2B00F0B0805E2BF0
S214011130C0F087805F2B00F0D0800EE2C82B00F055
S2140111408281C82B09D8782B00F03B81792B00F0DF
S2140111505981772B00F01481FFE140F22D12934262
S21401116000F0AF81B3F5977F00F0CB81B3F5967FA2
S21401117000F09681F1E1BB68002B04D04BF25023BE
S214011180C0F2030303E04BF25423C0F203034BF215
S2140111908C20C0F2030019461AF0C6FE4FF0000379
S2140111A07B610BE07B69DAB2BB68DBB2104619469D
S2140111B00DF0FEFD7B6903F101037B617B69592B11
S2140111C0F0D9CAE1BB68002B04D04BF25023C0F221
S2140111D0030303E04BF25423C0F203034BF2A020B7
S2140111E0C0F2030019461AF09FFEBB68DBB2184630
S2140111F00DF0C0FDB1E1BB68002B04D04BF25023CB
S214011200C0F2030303E04BF25423C0F203034BF294
S214011210B020C0F2030019461AF086FEBB68002B08
S21401122007D04FF24003C4F20F034FF480025A6016
S21401123093E14FF24003C4F20F034FF480029A6029
S2140112408BE1BB68002B04D04BF25023C0F20303A2
S21401125003E04BF25423C0F203034BF2C020C0F26A
S214011260030019461AF060FEBB68002B07D04FF248
S2140112708003C4F20F034FF480525A606DE14FF2BF
S2140112808003C4F20F034FF480529A6065E1BB6895
S214011290002B04D04BF25023C0F2030303E04BF2C1
S2140112A05423C0F203034BF2D020C0F203001946C8
S2140112B01AF03AFEBB68002B07D04FF28003C4F247
S2140112C00F034FF480225A6047E14FF28003C4F2C5
S2140112D00F034FF480229A603FE1BB68002B04D0D5
S2140112E04BF25023C0F2030303E04BF25423C0F247
S2140112F003034BF2E820C0F2030019461AF014FE6D
S214011300BB68002B07D04FF28003C4F20F034FF4E3
S21401131000429A6021E14FF28003C4F20F034FF4BA
S21401132000425A6019E1BB68002B04D04BF25023EF
S214011330C0F2030303E04BF25423C0F203034BF263
S214011340FC20C0F2030019461AF0EEFD4FF0000330
S2140113507B6111E07B69DAB2BB68002B0CBF00230E
S2140113600123DBB2104619464FF001020DF0F0FBE7
S2140113707B6903F101037B617B69112BEAD9ECE000
S214011380BB68002B04D04BF25023C0F2030303E0EA
S2140113904BF25423C0F203034BF21030C0F20300A9
S2140113A019461AF0C1FDBB68002B0CBF00230123B0
S2140113B0DBB24FF0120019464FF000020DF0C8FBE9
S2140113C0CBE0BB68002B04D04BF25023C0F20303E2
S2140113D003E04BF25423C0F203034BF21C30C0F27D
S2140113E0030019461AF0A0FDBB68002B0CBF0023B2
S2140113F00123DBB24FF0130019464FF000020DF047
S214011400A7FBAAE0BB68002B04D04BF25023C0F226
S214011410030303E04BF25423C0F203034BF22C30D8
S214011420C0F2030019461AF07FFDBB68002B0CBF03
S21401143000230123DBB24FF0140019464FF00002DF
S2140114400DF086FB89E0BB68002B04D04BF25023DD
S214011450C0F2030303E04BF25423C0F203034BF242
S2140114603C30C0F2030019461AF05EFD4FF000034F
S2140114707B6111E07B69DAB2BB68002B0CBF0023ED
S2140114800123DBB2104619464FF002020DF060FB55
S2140114907B6903F101037B617B69112BEAD95CE06F
S2140114A0BB684BF25030C0F2030019461AF03CFDFF
S2140114B0BB68DBB243F02803DBB2184605F038F808
S2140114C04BE0BB68002B04D04BF25023C0F2030361
S2140114D003E04BF25423C0F203034BF26430C0F234
S2140114E0030019461AF020FDBB68002B04D04FF00C
S2140114F0AF0005F01DF830E04FF0AE0005F018F82B
S2140115002BE0BB68002B04D04BF25023C0F2030340
S21401151003E04BF25423C0F203034BF27430C0F2E3
S214011520030019461AF000FDBB68002B08D04FF0E7
S214011530A40004F0FDFF4FF0AF0004F0F9FF0BE04C
S2140115404FF0AC0004F0F4FF4FF0AE0004F0F0FFF3
S2140115504FF0A50004F0ECFF00BFBB6932E04BF290
S2140115608430C0F203001AF0DFFC4FF0FF33BB619A
S2140115704FF00103FB770BE04AF61060C0F2030060
S2140115801AF0D2FC4FF0FF33BB614FF00103FB773B
S214011590FB7F002B15D0FB7C002B09D03B681B681A
S2140115A04BF2A030C0F2030019461AF0BDFC08E069
S2140115B03B681B684BF2BC30C0F2030019461AF0B8
S2140115C0B3FCBB69184607F12007BD4680BD00BFC6
S2140115D080B588B000AF786039604FF00003FB75C6
S2140115E04FF00003BB6107F11703786839681A46A4
S2140115F00EF062FF0346FB7740F63D33C1F6FF73FC
S2140116004FF000021A70FB7F83F00103DBB2002B60
S21401161049D07B68032B3AD13B6803F104031A686F
S21401162007F11003104619460EF002FF0346002B81
S21401163020D03B6803F108031A6807F10C03104633
S21401164019460EF0F5FE0346002B13D0FA683B69E7
S2140116504BF2DC30C0F2030011461A461AF064FC65
S2140116603B69DAB2FB68DBB2104619460DF0CAFEDA
S214011670BB6932E04BF28430C0F203001AF054FC2E
S2140116804FF0FF33BB614FF00103FB770BE04AF6E7
S2140116901060C0F203001AF047FC4FF0FF33BB6145
S2140116A04FF00103FB77FB7F002B15D0FB7D002B52
S2140116B009D03B681B684BF2F830C0F203001946AC
S2140116C01AF032FC08E03B681B684BF21440C0F28B
S2140116D0030019461AF028FCBB69184607F12007D3
S2140116E0BD4680BD80B588B000AF786039604FF0E8
S2140116F00003FB754FF00003BB6140F63D33C1F6B6
S214011700FF734FF000021A7007F117037868396803
S2140117101A460EF0D1FE0346FB77FB7F83F00103EA
S214011720DBB2002B49D07B68032B3AD13B6803F12F
S21401173004031A6807F11003104619460EF078FEE6
S2140117400346002B20D03B6803F108031A6807F113
S2140117500C03104619460EF06BFE0346002B13D001
S2140117603A69FB684BF23840C0F2030011461A464C
S2140117701AF0DAFB3B69DAB2FB68DBB210461946AF
S2140117800DF0D8FABB6932E04BF28430C0F20300A8
S2140117901AF0CAFB4FF0FF33BB614FF00103FB7732
S2140117A00BE04AF61060C0F203001AF0BDFB4FF0E2
S2140117B0FF33BB614FF00103FB77FB7F002B15D096
S2140117C0FB7D002B09D03B681B684BF25840C0F2EA
S2140117D0030019461AF0A8FB08E03B681B684BF2A9
S2140117E07840C0F2030019461AF09EFBBB69184602
S2140117F007F12007BD4680BD80B586B000AF786092
S21401180039604FF00003FB734FF000033B6140F675
S2140118103D33C1F6FF734FF000021A7007F10F0354
S214011820786839681A460EF047FE0346FB75FB7D5D
S21401183083F00103DBB2002B5BD07B68012B0FD159
S21401184040F2A853C1F6FF731B684BF28070C0F2DA
S214011850030019461AF068FB4FF00103FB7548E0D8
S2140118607B68022B39D13B6803F104031A6807F140
S2140118700803104619460EF0DBFD0346002B1FD069
S21401188040F2A853C1F6FF731B684BF2AC70C0F26E
S214011890030019461AF048FBBA6840F2A853C1F68D
S2140118A0FF731A6040F2A853C1F6FF731B684BF230
S2140118B0C470C0F2030019461AF036FB3B6938E0E3
S2140118C04BF28430C0F203001AF02EFB4FF0FF33C8
S2140118D03B614FF00103FB750BE04AF61060C0F266
S2140118E003001AF021FB4FF0FF333B614FF0010379
S2140118F0FB75FB7D002B1BD0FB7B002B09D03B68C7
S2140119001B684BF2D470C0F2030019461AF00CFBA8
S2140119100EE03B681B684BF2E470C0F20300194608
S2140119201AF002FB4BF2F870C0F203001AF0FCFA50
S2140119303B69184607F11807BD4680BD80B586B0DD
S21401194000AF786039604FF00003FB734FF0FF3350
S2140119503B6140F63D33C1F6FF734FF000021A704B
S21401196007F10F03786839681A460EF0A5FD03469D
S214011970FB75FB7D83F00103DBB2002B4FD07B6848
S214011980012B17D140F2C143C1F6FF731B78002B20
S21401199004D04BF25023C0F2030303E04BF254236E
S2140119A0C0F203034BF61400C0F2030019461AF006
S2140119B0BBFA34E04FF00103FB757B68022B28D19C
S2140119C03B6803F104031A6807F108031046194639
S2140119D00EF02EFD0346002B14D0BB68002B07D05B
S2140119E040F2C143C1F6FF734FF001021A7006E0E0
S2140119F040F2C143C1F6FF734FF000021A704FF078
S214011A00000326E04BF28430C0F203001AF08CFA91
S214011A1005E04AF61060C0F203001AF085FAFB7D75
S214011A20002B15D0FB7B002B09D03B681B684BF6BF
S214011A303400C0F2030019461AF076FA08E03B6853
S214011A401B684BF64000C0F2030019461AF06CFA08
S214011A503B69184607F11807BD4680BD80B586B0BC
S214011A6000AF786039604FF00003FB734FF0FF332F
S214011A703B6140F63D33C1F6FF734FF000021A702A
S214011A8007F10F03786839681A460EF015FD03460C
S214011A90FB75FB7D83F00103DBB2002B4FD07B6827
S214011AA0012B17D140F2C043C1F6FF731B78002B00
S214011AB004D04BF25023C0F2030303E04BF254234D
S214011AC0C0F203034BF65400C0F2030019461AF0A5
S214011AD02BFA34E04FF00103FB757B68022B28D10B
S214011AE03B6803F104031A6807F108031046194618
S214011AF00EF09EFC0346002B14D0BB68002B07D0CB
S214011B0040F2C043C1F6FF734FF001021A7006E0BF
S214011B1040F2C043C1F6FF734FF000021A704FF057
S214011B20000326E04BF28430C0F203001AF0FCF901
S214011B3005E04AF61060C0F203001AF0F5F9FB7DE5
S214011B40002B15D0FB7B002B09D03B681B684BF69E
S214011B503400C0F2030019461AF0E6F908E03B68C3
S214011B601B684BF64000C0F2030019461AF0DCF978
S214011B703B69184607F11807BD4680BD80B586B09B
S214011B8000AF786039604FF00003FB734FF0FF330E
S214011B903B6140F63D33C1F6FF734FF000021A7009
S214011BA007F10F03786839681A460EF085FC03467C
S214011BB0FB75FB7D83F00103DBB2002B4FD07B6806
S214011BC0012B17D140F2A453C1F6FF731B78002BEB
S214011BD004D04BF25023C0F2030303E04BF254232C
S214011BE0C0F203034BF67400C0F2030019461AF064
S214011BF09BF934E04FF00103FB757B68022B28D17B
S214011C003B6803F104031A6807F1080310461946F6
S214011C100EF00EFC0346002B14D0BB68002B07D039
S214011C2040F2A453C1F6FF734FF001021A7006E0AA
S214011C3040F2A453C1F6FF734FF000021A704FF042
S214011C40000326E04BF28430C0F203001AF06CF970
S214011C5005E04AF61060C0F203001AF065F9FB7D54
S214011C60002B15D0FB7B002B09D03B681B684BF67D
S214011C703400C0F2030019461AF056F908E03B6832
S214011C801B684BF64000C0F2030019461AF04CF9E7
S214011C903B69184607F11807BD4680BD80B586B07A
S214011CA000AF786039604FF00003FB734FF0FF33ED
S214011CB03B6140F63D33C1F6FF734FF000021A70E8
S214011CC007F10F03786839681A460EF0F5FB0346EC
S214011CD0FB75FB7D83F00103DBB2002B4FD07B68E5
S214011CE0012B17D140F25353C1F6FF731B78002B1B
S214011CF004D04BF25023C0F2030303E04BF254230B
S214011D00C0F203034BF69400C0F2030019461AF022
S214011D100BF934E04FF00103FB757B68022B28D1E9
S214011D203B6803F104031A6807F1080310461946D5
S214011D300EF07EFB0346002B14D0BB68002B07D0A9
S214011D4040F25353C1F6FF734FF001021A7006E0DA
S214011D5040F25353C1F6FF734FF000021A704FF072
S214011D60000326E04BF28430C0F203001AF0DCF8E0
S214011D7005E04AF61060C0F203001AF0D5F8FB7DC4
S214011D80002B15D0FB7B002B09D03B681B684BF65C
S214011D903400C0F2030019461AF0C6F808E03B68A2
S214011DA01B684BF64000C0F2030019461AF0BCF857
S214011DB03B69184607F11807BD4680BD80B586B059
S214011DC000AF786039604FF00003FB734FF00003FB
S214011DD03B6140F63D33C1F6FF734FF000021A70C7
S214011DE007F10F03786839681A460EF065FB03465B
S214011DF0FB75FB7D83F00103DBB2002B1DD07B68F6
S214011E00012B0CDD4AF61060C0F203001AF08CF8C4
S214011E104FF0FF333B614FF00103FB750DE021F0FE
S214011E202FFD21F071FA03464BF6B400C0F2030011
S214011E3019461AF079F800F0F5FCFB7D002B15D059
S214011E40FB7B002B09D03B681B684BF6CC00C0F22D
S214011E50030019461AF068F808E03B681B684BF661
S214011E60D000C0F2030019461AF05EF83B69184626
S214011E7007F11807BD4680BD80B586B000AF786013
S214011E8039604FF00003FB734FF000033B6140F6EF
S214011E903D33C1F6FF734FF000021A7007F10F03CE
S214011EA0786839681A460EF007FB0346FB75FB7D1A
S214011EB083F00103DBB2002B11D07B68012B0CDD14
S214011EC04AF61060C0F203001AF02EF84FF0FF3306
S214011ED03B614FF00103FB7501E00CF0C3FFFB7D96
S214011EE0002B15D0FB7B002B09D03B681B684AF6FC
S214011EF03860C0F2030019461AF016F808E03B688D
S214011F001B684AF64060C0F2030019461AF00CF846
S214011F103B69184607F11807BD4680BD80B59EB0DF
S214011F2000AF786039604FF0000387F86F304FF0EC
S214011F3000033B6740F63D33C1F6FF734FF00002E6
S214011F401A7007F16F03786839681A460EF0B4FA0A
S214011F50034687F8773097F8773083F00103DBB2D2
S214011F60002B4CD07B68012B0DDD4AF61060C0F2C9
S214011F70030019F0D9FF4FF0FF333B674FF0010321
S214011F8087F877303BE04BF6DC00C0F2030019F02F
S214011F90CBFF4BF61C10C0F2030019F0C5FF07F18A
S214011FA008034BF63010C0F20300194619F020FF63
S214011FB007F1080318464BF63411C0F2030125F069
S214011FC0F1F80346002B14D14BF64010C0F2030083
S214011FD019F0AAFF41F2F803C1F6FF731B68184611
S214011FE002F09CF84BF66410C0F2030019F09CFF57
S214011FF005E04BF67C10C0F2030019F095FF97F848
S2140120007730002B16D097F86F30002B09D03B683D
S2140120101B684AF63860C0F20300194619F084FFBF
S21401202008E03B681B684AF64060C0F203001946A8
S21401203019F07AFF3B6F184607F17807BD4680BD59
S21401204080B5A0B000AF786039604FF0000387F824
S21401205077304FF0FF33BB6740F63D33C1F6FF7371
S2140120604FF000021A7007F17703786839681A464C
S2140120700EF022FA034687F87F3097F87F3083F018
S2140120800103DBB2002B00F094807B68012B19D191
S21401209040F22353C1F6FF731B781A4613464FEAE4
S2140120A0C3039B184FEA43034BF69010C0F203009C
S2140120B0194619F039FF4BF6AC10C0F2030019F0BF
S2140120C033FF76E04FF0010387F87F307B68022B01
S2140120D069D13B6803F104031A6807F170031046DF
S2140120E019460EF0A5F90346002B55D03B6F012B80
S2140120F043D93B6F052B40D84BF61C10C0F20300AA
S21401210019F012FF07F10C034BF63010C0F2030072
S214012110194619F06DFE07F10C0318464BF63411FB
S214012120C0F2030125F03EF80346002B1ED13B6F9B
S214012130DAB240F22353C1F6FF731A7040F223530A
S214012140C1F6FF731B781A4613464FEAC3039B1862
S2140121504FEA43034BF6E410C0F20300194619F0A8
S214012160E3FE01F0FDFD0CF07DFE12E04BF67C1067
S214012170C0F2030019F0D8FE0BE04BF60820C0F2BF
S214012180030019F0D1FE4BF62420C0F2030019F02B
S214012190CBFE4FF0000328E04BF28430C0F2030080
S2140121A019F0C2FE05E04AF61060C0F2030019F00D
S2140121B0BBFE97F87F30002B16D097F87730002BB0
S2140121C009D03B681B684BF63400C0F20300194681
S2140121D019F0AAFE08E03B681B684BF64000C0F207
S2140121E00300194619F0A0FEBB6F184607F18007D9
S2140121F0BD4680BD80B586B000AF786039604FF0CF
S2140122000003BB744FF0FF337B6140F63D33C1F6EC
S214012210FF734FF000021A7007F1120378683968ED
S2140122201A460EF049F90346FB74FB7C83F0010362
S214012230DBB2002B39D07B68022B30D13B6803F12F
S21401224004031A6807F10C03104619460EF0F0F85D
S2140122500346002B29D0FB683F2B11D8FB684BF6B1
S2140122604420C0F20300194619F05EFE4FF08100CB
S21401227004F05EF9FB68DBB2184604F059F90BE08E
S2140122804BF60820C0F2030019F04EFE4BF6602014
S214012290C0F2030019F048FE4FF000031FE04AF6B3
S2140122A01060C0F2030019F03FFEFB7C002B15D036
S2140122B0BB7C002B09D03B681B684BF68020C0F224
S2140122C00300194619F030FE08E03B681B684BF620
S2140122D08C20C0F20300194619F026FE7B691846C9
S2140122E007F11807BD4680BD80B586B000AF78609F
S2140122F039604FF00003BB744FF0FF337B6140F64B
S2140123003D33C1F6FF734FF000021A7007F1120356
S214012310786839681A460EF0CFF80346FB74FB7CE2
S21401232083F00103DBB2002B38D07B68022B2FD160
S2140123303B6803F104031A6807F10C0310461946BB
S2140123400EF076F80346002B28D0FB68072B10D832
S214012350FB684BF6A020C0F20300194619F0E4FD15
S214012360FB68DBB243F02003DBB2184604F0E0F86A
S2140123700BE04BF60820C0F2030019F0D5FD4BF632
S214012380C420C0F2030019F0CFFD4FF000031FE098
S2140123904AF61060C0F2030019F0C6FDFB7C002B64
S2140123A015D0BB7C002B09D03B681B684BF6E020A0
S2140123B0C0F20300194619F0B7FD08E03B681B6838
S2140123C04BF6EC20C0F20300194619F0ADFD7B690F
S2140123D0184607F11807BD4680BD00BF80B586B018
S2140123E000AF786039604FF00003FB734FF0FF33A6
S2140123F03B6140F63D33C1F6FF734FF000021A70A1
S21401240007F10F03786839681A460EF055F8034647
S214012410FB75FB7D83F00103DBB2002B47D07B68A5
S214012420012B14D140F2A053C1F6FF731A6844F68B
S214012430D353C1F26203A3FB02134FEA93134BF685
S2140124400030C0F20300194619F06EFD2FE04FF080
S2140124500103FB757B68022B23D13B6803F1040360
S2140124601A6807F10803104619460DF0E1FF034606
S214012470002B1CD0BB684BF62C30C0F2030019466B
S21401248019F052FDBB684FF47A7202FB03F240F278
S214012490A053C1F6FF731A6001F0B8FC4FF00003B9
S2140124A01FE04AF61060C0F2030019F03DFDFB7D07
S2140124B0002B15D0FB7B002B09D03B681B684BF625
S2140124C05430C0F20300194619F02EFD08E03B68AF
S2140124D01B684BF66C30C0F20300194619F024FD58
S2140124E03B69184607F11807BD4680BD90B585B013
S2140124F002AF4BF68C30C0F2030019F015FD4BF617
S2140125009C30C0F2030019F00FFD40F22353C1F6D0
S214012510FF731B781A4613464FEAC3039B184FEA0C
S21401252043034BF6AC30C0F20300194619F0FCFC2D
S2140125304BF6C030C0F203004BF6E431C0F20301A3
S2140125404BF6F032C0F2030219F0EEFC4DF61063C2
S214012550C0F203031B684BF60440C0F203001946A1
S21401256019F0E2FC4BF61440C0F203004FF00301F1
S21401257019F0DAFC41F2FE03C1F6FF731B884BF635
S2140125802840C0F203004FF417711A4619F0CCFC2C
S21401259041F2FC03C1F6FF731B884BF64C40C0F2B8
S2140125A00300194619F0C0FC40F6CC63C1F6FF7370
S2140125B01B78002B04D04BF66843C0F2030303E0FC
S2140125C04BF66C43C0F203034BF67440C0F20300B3
S2140125D0194619F0A9FC40F63833C1F6FF731B788B
S2140125E0022B04D14BF66843C0F2030303E04BF61B
S2140125F06C43C0F203034BF68840C0F20300194651
S21401260019F092FC40F22753C1F6FF731B784BF684
S2140126109440C0F20300194619F086FC40F222539A
S214012620C1F6FF731B78012B04D14BF6AC43C0F205
S214012630030303E04BF6B443C0F203034BF6BC407E
S214012640C0F20300194619F06FFC40F66A33C1F672
S214012650FF731B781A4640F25853C1F6FF7353F8BE
S21401266022304BF6C840C0F20300194619F05CFC54
S21401267040F66833C1F6FF731B781A4640F6693395
S214012680C1F6FF731B784BF6DC40C0F2030011461F
S2140126901A4619F049FC40F2A053C1F6FF731A68B6
S2140126A044F6D353C1F26203A3FB02134FEA93131A
S2140126B04BF6FC40C0F20300194619F035FC40F613
S2140126C0CA63C1F6FF731B78002B04D04BF6205368
S2140126D0C0F2030303E04BF62453C0F203034BF6A8
S2140126E02850C0F20300194619F01EFC40F6443388
S2140126F0C1F6FF731B784BF64050C0F20300194633
S21401270019F012FC40F6D663C1F6FF731B784BF640
S2140127105850C0F20300194619F006FC40F6433340
S214012720C1F6FF731B784BF67050C0F203001946D2
S21401273019F0FAFB4BF68450C0F2030019F0F4FBD3
S2140127404FF00003FB7138E0FB7903F14101FA79A0
S21401275040F6C823C1F6FF7333F812301C46FA79E7
S21401276040F68823C1F6FF739B5C002B04D04BF622
S2140127702053C0F2030303E04BF62453C0F20303D5
S214012780F87940F68022C1F6FF72125C002A04D066
S2140127904BF62052C0F2030203E04BF62452C0F27D
S2140127A0030200924BF69850C0F20300224619F03D
S2140127B0BBFBFB7903F10103FB7140F22353C1F626
S2140127C0FF731B78FA799A42BED340F62D73C1F691
S2140127D0FF731B78002B04D04BF62053C0F2030383
S2140127E003E04BF62453C0F203034BF6D050C0F27D
S2140127F00300194619F098FB00F00EF807F10C07D4
S214012800BD4690BD80B483B000AF0346FB7107F1AF
S2140128100C07BD4680BC704780B400AFBD4680BC87
S214012820704700BF80B58AB000AF4FF000037B62EF
S2140128304FF480133B6240F20003C0F20103FB61D8
S21401284040F20003C0F2040303F1FF33BB614FF013
S2140128500003C1F6FF737B614FF400333B6147F21F
S2140128607073C1F6FF73FB604FF6F073C2F200039C
S21401287003F1FF33BB6020F047FD03467B607A6AB5
S2140128803B6AD31803F1FF334BF6E450C0F2030062
S214012890796A1A463B6A19F047FBBA69FB69D31A8B
S2140128A003F101034BF61060C0F20300F969BA693F
S2140128B019F03AFB7A693B69D31803F1FF334BF6FB
S2140128C04060C0F2030079691A463B6919F02CFB97
S2140128D0FB6803F1FF32F9687B69CB1A4BF66C6033
S2140128E0C0F20300796919F01FFB4BF6A060C0F235
S2140128F00300F968BA687B6819F016FBBA687B684A
S214012900D31A4BF6DC60C0F20300194619F00CFB33
S21401291007F12807BD4680BD80B5ADF51C7D00AF2B
S21401292007F1D0031A464FF4C97310464FF0000161
S2140129301A4624F031FC07F104031A464FF0C90386
S21401294010464FF000011A4624F026FC00F09CFBCE
S21401295041F2F803C1F6FF731A6807F266231046C0
S2140129604FF48051C0F23F014FF0020202F054F8DA
S21401297041F2F803C1F6FF731A6807F5197310469A
S2140129804FF47C114FF0020202F046F8B7F86432B9
S214012990002B11D041F2F803C1F6FF731B681846ED
S2140129A04FF47041C0F23E014FF4966247F2C013F5
S2140129B0C1F6FF7302F030F800F082FB4FF000031F
S2140129C0A7F86E32AEE0B7F86E3240F25B2202FB39
S2140129D003F303F58053C7F8683200F055FB41F264
S2140129E0F803C1F6FF731A6807F104031046D7F817
S2140129F068124FF0C90202F00FF841F2F803C1F66F
S214012A00FF731968D7F8683203F1C90207F1D003DA
S214012A10084611464FF4C97201F0FEFF00F050FB64
S214012A20B7F86E22B7F86E1247F2C013C1F6FF73FD
S214012A3053F821304BF6FC60C0F2030011461A46EB
S214012A4019F072FA4BF62070C0F2030019F06CFA16
S214012A504FF0010387F86D321BE097F86D3207F1EE
S214012A600402D35C002B0ED097F86D2297F86D32D6
S214012A7007F10401CB5C4BF63470C0F2030011463B
S214012A801A4619F051FA97F86D3203F1010387F8E7
S214012A906D3297F86D32C82BDFD94BF64870C0F20D
S214012AA0030019F041FA4BF64C70C0F2030019F01E
S214012AB03BFA4FF0010387F86D3223E097F86D2259
S214012AC007F1D00333F81230002B15D097F86D12AA
S214012AD097F86D2207F1D00333F812301A461346E1
S214012AE04FEA83039B184FEA43034BF66070C0F22C
S214012AF003001A4619F018FA97F86D3203F101032C
S214012B0087F86D3297F86D32C82BD7D94BF64870D7
S214012B10C0F2030019F008FAB7F86E3203F10103A8
S214012B20A7F86E32B7F86432B7F86E229A42FFF40D
S214012B304AAF07F51C77BD4680BD00BF80B582B0A1
S214012B4000AF786021F042FB0CF068FD0CF02CFD24
S214012B504CF24400C0F2030019F0E6F940F22353A8
S214012B60C1F6FF731B781A4613464FEAC3039B1838
S214012B704FEA43034CF26400C0F20300194619F011
S214012B80D3F94CF27800C0F203004CF29C01C0F27B
S214012B9003014CF2A802C0F2030219F0C5F94DF682
S214012BA01063C0F203031B684CF2BC00C0F20300C2
S214012BB0194619F0B9F94CF2CC00C0F2030019F02D
S214012BC0B3F94CF2FC00C0F2030019F0ADF9FFF7BF
S214012BD023FE4CF22010C0F2030019F0A5F94FF2C3
S214012BE04003C4F20F034FF400225A604FF4FA7008
S214012BF01CF01CF80BF096FB00F010F84BF6747006
S214012C00C0F203004FF000010DF0E2F94CF23C1067
S214012C10C0F2030019F088F9F0E700BF80B500AFF5
S214012C2000F044F821F0D2FA4FF025004FF00301EE
S214012C304FF000020EF0BEFB41F2B800C1F6FF7085
S214012C404FF0000120F094FC0346002B07D04CF215
S214012C505C20C0F2030019F067F9FDF7F9FB0EF0EE
S214012C60E3F80346012B06D04CF27C20C0F20300A9
S214012C7019F05AF905E04CF29820C0F2030019F059
S214012C8053F980BD80B582B000AF786078680FF0E8
S214012C90BDFA41F2B800C1F6FF704FF0010120F015
S214012CA079FC07F10807BD4680BD00BF80B500AFBF
S214012CB040F24C60C1F6FF704FF02001C8F20001EF
S214012CC04FF000024FF002030FF0A6F8034683F020
S214012CD00103DBB2002B07D04CF2B820C0F2030090
S214012CE019F022F9FDF7B4FB40F24C60C1F6FF7013
S214012CF04FF001010FF0C6F940F24C60C1F6FF70CB
S214012D004FF001014FF001020FF0D0F840F24C6095
S214012D10C1F6FF704FF002010FF020FA034683F070
S214012D200103DBB2002B07D04CF2D420C0F2030023
S214012D3019F0FAF8FDF78CFB40F24C60C1F6FF7013
S214012D400FF076FA0346184642F68541C0F20101B5
S214012D5040F24C62C1F6FF7221F050F940F24C602D
S214012D60C1F6FF700FF064FA034618464FF00301F0
S214012D704FF0010218F0DCFD40F24C60C1F6FF7026
S214012D804FF001010FF018FA80BD00BF80B500AF0B
S214012D9040F63833C1F6FF734FF000021A704FF059
S214012DA0000006F003F84FF0000006F07BF805F08F
S214012DB04FFF0BF081FE04F03FFA4FF020004FF07A
S214012DC000014FF000024FF0000302F0B1FE4FF495
S214012DD07043C4F20F034FF010025A604FF06400C4
S214012DE01BF024FF4FF013004FF001014FF00002DB
S214012DF00BF0AEFE4CF2FC20C0F2030019F094F882
S214012E0040F62D73C1F6FF734FF001021A7040F2BF
S214012E10A453C1F6FF734FF000021A7040F24C4003
S214012E201BF004FF0BF02AFE4CF23430C0F2030014
S214012E3019F07AF84FF064001BF0F8FE4FF003002B
S214012E400EF0FCF94FF000000EF0F8F94CF24830A5
S214012E50C0F2030019F068F84FF47043C4F20F0390
S214012E604FF010029A6040F62D73C1F6FF734FF0D3
S214012E7000021A7040F2A453C1F6FF734FF001022C
S214012E801A704FF47043C4F20F034FF010029A60A9
S214012E904FF0010006F006F80BF0F0FD03F002FD1E
S214012EA000F006F84FF064001BF0C0FE80BD00BFC6
S214012EB080B582B000AF4FF00003FB7140F2505373
S214012EC0C1F6FF734FF6FE721A80FB79142B17D1E9
S214012ED04CF25830C0F2030019F026F84FF02200E9
S214012EE04FF000014FF000024FF0000302F020FE09
S214012EF04FF4FA701BF09AFE4FF00003FB7126E0C8
S214012F00FB79002B0CBF00230123DBB2FA7902F117
S214012F100102FA71002B0CD04CF29C30C0F2030077
S214012F2019F002F8FB79012B03D14FF0070004F0EA
S214012F3005FA4FF023004FF000014FF000024FF06A
S214012F40000302F0F5FD4FF496701BF06FFE40F2A1
S214012F505053C1F6FF731B881BB213F1020FB4D096
S214012F6003F0A0FC07F10807BD4680BD80B582B01E
S214012F7000AF78604CF2E030C0F2030018F0D4FFE6
S214012F804FF064001BF052FE00F096FF00F0A4F82C
S214012F9040F26363C1F6FF734FF001021A7040F20C
S214012FA0C043C1F6FF731B78002B67D040F25D6308
S214012FB0C1F6FF731B78002B12D040F25D63C1F699
S214012FC0FF734FF000021A7000F05EF840F64333CC
S214012FD0C1F6FF731B78184600F04CFB00F070F842
S214012FE040F26163C1F6FF731B78002B10D040F2EC
S214012FF06163C1F6FF734FF000021A7040F6B863C2
S214013000C1F6FF731B78184600F03CFC0AF082F903
S21401301040F25E63C1F6FF731B78002B0CD040F2C2
S2140130205E63C1F6FF734FF000021A7000F02CF8D1
S21401303000F07CFB00F044F840F25F63C1F6FF73DA
S2140130401B78002B06D040F25F63C1F6FF734FF08A
S21401305000021A7040F26063C1F6FF731B78002B02
S2140130600CD040F26063C1F6FF734FF000021A7095
S21401307000F00AF800F0B0FB00F022F84FF0640010
S2140130801BF0D4FD8BE700BF80B500AF09E04FF021
S21401309001001BF0CBFD4CF2FC30C0F2030018F02F
S2140130A043FF40F25C63C1F6FF731B78002BEED141
S2140130B040F25C63C1F6FF734FF001021A7080BDE7
S2140130C080B400AF40F25C63C1F6FF734FF00002BC
S2140130D01A70BD4680BC704780B588B000AF41F21B
S2140130E0F803C1F6FF731B68002B02D14FF00003F3
S2140130F080E24CF21040C0F2030018F015FF41F2D6
S214013100F803C1F6FF731B6818464FF4A041C0F2DE
S2140131103F0101F009FA0346BB77BB7F012B02D9B9
S214013120BB7F052B02D900F01BFE05E040F22353BE
S214013130C1F6FF73BA7F1A7041F2F803C1F6FF7346
S2140131401B6818464FF47041C0F23F0101F0ECF9DC
S21401315003467B774CF23040C0F2030018F0E4FEE1
S2140131607B7FFF2B06D14CF24040C0F2030018F0E3
S214013170DBFE07E07B7F4CF25040C0F203001946AD
S21401318018F0D2FE7B7F032B4DD04CF25440C0F298
S214013190030018F0C9FE41F2F803C1F6FF731B687D
S2140131A0184600F0BBFF4FF0000000F063FA4FF046
S2140131B0010000F05FFA4FF0020000F05BFA4FF0FA
S2140131C0030000F057FA4FF0040000F053FA00F045
S2140131D0ADFA00F0C5FD00F051FD00F017FE41F21A
S2140131E0F803C1F6FF731B6818464FF47041C0F22E
S2140131F03F0100F0CDFF0346002B0ED041F2F8034D
S214013200C1F6FF731B6818464FF47041C0F23F01C8
S2140132104FF0030201F0E2F805E04CF2A040C0F2E4
S214013220030018F081FE41F2F803C1F6FF731A6835
S21401323007F1100310464FF4C041C0F23F014FF0B2
S214013240020201F0E9FB41F2F803C1F6FF731A68C6
S21401325007F1100303F1020310464FF4E041C0F2F8
S2140132603F014FF0020201F0D7FB41F2F803C1F62D
S214013270FF731A6807F1100303F1040310464FF4B5
S2140132807E114FF0020201F0C7FB41F2F803C1F6CE
S214013290FF731A6807F1100303F1060310464FF493
S2140132A01041C0F23F014FF0020201F0B5FB41F2BE
S2140132B0F803C1F6FF731A6807F1100303F1080358
S2140132C010464FF42041C0F23F014FF0020201F0D8
S2140132D0A3FB4FF00003FB772CE0FB7F4FEA430391
S2140132E007F12001CB1833F8102C4FF6FF739A42E2
S2140132F00DD1FA7F40F6C823C1F6FF734FF00001E7
S21401330023F81210FB7F184600F0B4F90EE0FA7F9E
S214013310FB7F4FEA430307F12001CB1833F8101C5B
S21401332040F6C823C1F6FF7323F81210FB7F03F1A2
S2140133300103FB7740F22353C1F6FF731B78FA7F34
S2140133409A42CAD340F22353C1F6FF731B78FB7728
S2140133500CE0FA7F40F6C823C1F6FF734FF0C801B0
S21401336023F81210FB7F03F10103FB77FB7F042B8D
S214013370EFD941F2F803C1F6FF731B6818464FF404
S2140133805041C0F23F0101F0CFF803463B773B7F47
S214013390FF2B09D140F22253C1F6FF734FF0010211
S2140133A01A7000F0C3F905E040F22253C1F6FF732C
S2140133B03A7F1A7041F2F803C1F6FF731B6818468C
S2140133C04FF46041C0F23F0101F0AEF80346FB76D0
S2140133D0FB7E042B09D940F66A33C1F6FF734FF022
S2140133E000021A7000F0F8F905E040F66A33C1F6FB
S2140133F0FF73FA7E1A7041F2F803C1F6FF731B6879
S21401340018464FF40051C0F23F0101F08DF8034613
S2140134101A4640F6B863C1F6FF731A7040F6B863F1
S214013420C1F6FF731B78632B16D940F66F33C1F6CE
S214013430FF734FF000021A7040F6B863C1F6FF73CF
S2140134404FF000021A7040F6B863C1F6FF731B789E
S214013450184600F017FA15E040F6B863C1F6FF7398
S2140134601B78002B07D140F66F33C1F6FF734FF080
S21401347000021A7006E040F66F33C1F6FF734FF094
S21401348001021A7041F2F803C1F6FF731A6807F1D8
S2140134900E0310464FF46041C0F23E014FF00202A7
S2140134A001F0BAFA41F2F803C1F6FF731A6807F1A0
S2140134B00C0310464EF20201C0F23E014FF002022A
S2140134C001F0AAFA07F10E0318464FF0020101F0C7
S2140134D06BFB0346002B09D107F10C0318464FF08E
S2140134E0020101F061FB0346002B0CD04FF00003F4
S2140134F0FB814FF00003BB81FA89BB891046194650
S21401350000F056FA10E0FA8940F6B8339A420BD921
S2140135104FF00003FB814FF00003BB81FA89BB89A2
S2140135201046194600F044FA41F2F803C1F6FF735B
S2140135301A6807F10A0310464FF48051C0F23F01A2
S2140135404FF0020201F068FA41F2F803C1F6FF7388
S2140135501A6807F10403104641F20601C0F23F0162
S2140135604FF0040201F058FA07F10A0318464FF02B
S214013570020101F019FB0346002B12D04FF00003A5
S2140135807B8141F2F803C1F6FF731A6807F10A035B
S21401359010464FF48051C0F23F014FF0020201F095
S2140135A08BF907F1040318464FF0040101F0FCFA09
S2140135B00346002B12D04FF000037B6041F2F80364
S2140135C0C1F6FF731A6807F10403104641F20601BB
S2140135D0C0F23F014FF0040201F06EF94FF4405083
S2140135E0C0F23F0040F2A051C1F6FF7100F008F8AA
S2140135F04FF00103184607F12007BD4680BD00BF06
S21401360080B584B000AF7860396041F2F803C1F646
S214013610FF731A6807F10C03104679684FF004022D
S21401362001F0FAF9FB68B3F1FF3F06D13B681B686E
S2140136307868194600F008F802E0FA683B681A60F4
S21401364007F11007BD4680BD80B582B000AF786037
S214013650396041F2F803C1F6FF731A683B4610461B
S21401366079684FF0040200F0B3FF07F10807BD4682
S21401367080BD00BF80B584B000AF0346FB7141F248
S214013680F803C1F6FF731B68002B02D14FF000034D
S21401369047E0FB7903F2F6334FEA0333FB6041F26E
S2140136A0F803C1F6FF731A6807F10A031046F968B2
S2140136B04FF0020201F0B0F9FA7940F6C823C1F6DC
S2140136C0FF7333F812207B899A4228D041F2F8031F
S2140136D0C1F6FF731B681846F96800F059FD0346EA
S2140136E0002B13D041F2F803C1F6FF731A68FB7979
S2140136F04FEA430140F6C823C1F6FF73CB181046C4
S214013700F9684FF0020200F063FF08E04CF2C44093
S214013710C0F2030018F008FC4FF0000301E04FF080
S2140137200103184607F11007BD4680BD80B582B07B
S21401373000AF41F2F803C1F6FF731B68002B02D1FC
S2140137404FF0000342E041F2F803C1F6FF731B6835
S21401375018464FF45041C0F23F0100F0E5FE034623
S214013760FB7140F22253C1F6FF731B78FA799A4235
S2140137702AD041F2F803C1F6FF731B6818464FF4CE
S2140137805041C0F23F0100F003FD0346002B12D06A
S21401379041F2F803C1F6FF731A6840F22253C1F6EC
S2140137A0FF731B7810464FF45041C0F23F011A4692
S2140137B000F014FE08E04CF2E440C0F2030018F0FA
S2140137C0B3FB4FF0000301E04FF00103184607F189
S2140137D00807BD4680BD00BF80B582B000AF41F28C
S2140137E0F803C1F6FF731B68002B02D14FF00003EC
S2140137F042E041F2F803C1F6FF731B6818464FF426
S2140138006041C0F23F0100F08FFE0346FB7140F6B7
S2140138106A33C1F6FF731B78FA799A422AD041F2CD
S214013820F803C1F6FF731B6818464FF46041C0F2F7
S2140138303F0100F0ADFC0346002B12D041F2F80325
S214013840C1F6FF731A6840F66A33C1F6FF731B7838
S21401385010464FF46041C0F23F011A4600F0BEFD2B
S21401386008E04CF22450C0F2030018F05DFB4FF064
S214013870000301E04FF00103184607F10807BD46B3
S21401388080BD00BF80B584B000AF0346FB7141F236
S214013890F803C1F6FF731B68002B02D14FF000033B
S2140138A040E0FFF7F1FB41F2F803C1F6FF731B6836
S2140138B018464FF40051C0F23F0100F035FE0346B2
S2140138C0FB73FA79FB7B9A4228D041F2F803C1F6E2
S2140138D0FF731B6818464FF40051C0F23F0100F019
S2140138E057FC0346002B0ED041F2F803C1F6FF73D6
S2140138F01A68FB7910464FF40051C0F23F011A4690
S21401390000F06CFD0AE04CF24850C0F2030018F0DB
S2140139100BFBFFF7D5FB4FF0000303E0FFF7D0FBEF
S2140139204FF00103184607F11007BD4680BD00BFE2
S21401393080B584B000AF0346FB8041F2F803C1F6C0
S214013940FF731B68002B02D14FF000032AE0FFF73C
S2140139509BFB41F2F803C1F6FF731B6818464FF450
S2140139607C1100F015FC0346002B0FD041F2F80342
S214013970C1F6FF731A6807F1060310464FF47C116F
S2140139804FF0020200F098FFF86008E04CF26C502D
S214013990C0F2030018F0C8FA4FF00003FB60FFF70F
S2140139A08FFBFB68184607F11007BD4680BD00BFB8
S2140139B080B584B000AF02460B46FA80BB8041F268
S2140139C0F803C1F6FF731B68002B02D14FF000030A
S2140139D03FE0FFF759FB41F2F803C1F6FF731B689E
S2140139E018464FF46041C0F23E0100F0D1FB034699
S2140139F0002B22D041F2F803C1F6FF731A6807F1D3
S214013A00060310464FF46041C0F23E014FF0020239
S214013A1000F052FFF86041F2F803C1F6FF731A682E
S214013A2007F1040310464EF20201C0F23E014FF0C8
S214013A30020200F041FFF86008E04CF29450C0F238
S214013A40030018F071FA4FF00003FB60FFF738FB34
S214013A50FB68184607F11007BD4680BD80B584B0E7
S214013A6000AF786041F2F803C1F6FF731B68002BC4
S214013A7002D14FF000032DE0FFF706FB41F2F803F9
S214013A80C1F6FF731B6818464FF47041C0F23E0141
S214013A9000F07EFB0346002B10D041F2F803C1F67E
S214013AA0FF731B6818464FF47041C0F23E014FF495
S214013AB096627B6800F08CFDF86008E04CF2C85016
S214013AC0C0F2030018F030FA4FF00003FB60FFF776
S214013AD0F7FAFB68184607F11007BD4680BD00BF20
S214013AE080B582B000AF4FF00003FB7141F2F803DE
S214013AF0C1F6FF731B68002B02D14FF000032EE0C6
S214013B00FFF7C2FA4FF00003FB7121E0FB7903F1E6
S214013B1001034FEA03333B6041F2F803C1F6FF733A
S214013B201B681846396800F033FB0346002B0BD19F
S214013B304CF20060C0F20300396818F0F5F9FFF79F
S214013B40BFFA4FF000030AE0FB7903F10103FB71B2
S214013B50FB792C2BDAD9FFF7B3FA4FF0010318469D
S214013B6007F10807BD4680BD80B582B000AF4FF0B3
S214013B700003FB7141F2F803C1F6FF731B68002BCB
S214013B8002D14FF000032EE0FFF77EFA4FF000035C
S214013B90FB7121E0FB7903F12E034FEA03333B600F
S214013BA041F2F803C1F6FF731B681846396800F046
S214013BB0EFFA0346002B0BD14CF22460C0F203004F
S214013BC0396818F0B1F9FFF77BFA4FF000030AE005
S214013BD0FB7903F10103FB71FB79052BDAD9FFF7BA
S214013BE06FFA4FF00103184607F10807BD4680BD7E
S214013BF080B584B000AF0346FB80FB8840F25B22B1
S214013C0002FB03F303F58053FB6041F2F803C1F6B0
S214013C10FF731B68002B02D14FF0000327E0FFF76C
S214013C2033FA41F2F803C1F6FF731B681846F968C8
S214013C304FF0C902104B00F0CBFC03467B8141F2EA
S214013C40F803C1F6FF731A68FB6803F1C90310464F
S214013C5019464FF4C97246F65073C1F6FF7300F069
S214013C60B7FC03467B81FFF72BFA4FF0010318469A
S214013C7007F11007BD4680BDE270FF1F80B582B018
S214013C8000AF41F2F803C1F6FF731B68002B02D1A7
S214013C904FF000035FE041F2F803C1F6FF731B68C3
S214013CA018464FF47D1100F073FA0346002B47D0F7
S214013CB040F27053C1F6FF731B684FF47D1019462E
S214013CC0FFF7C2FC40F27453C1F6FF731B684FF452
S214013CD08240C0F23F001946FFF7B6FC4FF00003E2
S214013CE0FB7129E0FB7903F57D3303F101034FEA0C
S214013CF003131A46F97940F27853C1F6FF7353F865
S214013D00213010461946FFF79FFCFB7903F57D33FA
S214013D1003F111034FEA03131A46F97940F28C5363
S214013D20C1F6FF7353F8213010461946FFF78CFC95
S214013D30FB7903F10103FB71FB79042BD2D908E06F
S214013D404CF24860C0F2030018F0EEF84FF00003A2
S214013D5001E04FF00103184607F10807BD4680BD94
S214013D6080B582B000AF41F2F803C1F6FF731B685D
S214013D70002B02D14FF0000342E041F2F803C1F6F6
S214013D80FF731B6818464FF4A041C0F23F0100F0D4
S214013D90CBFB0346FB7140F22353C1F6FF731B783E
S214013DA0FA799A422AD041F2F803C1F6FF731B68EA
S214013DB018464FF4A041C0F23F0100F0E9F903466E
S214013DC0002B12D041F2F803C1F6FF731A6840F2D5
S214013DD02353C1F6FF731B7810464FF4A041C0F27F
S214013DE03F011A4600F0FAFA08E04CF27060C0F2A1
S214013DF0030018F099F84FF0000301E04FF00103BB
S214013E00184607F10807BD4680BD00BF80B582B0E1
S214013E1000AF41F2F803C1F6FF731B68002B02D115
S214013E204FF0000342E041F2F803C1F6FF731B684E
S214013E3018464FF44051C0F23F0100F075FB0346AF
S214013E40FB71FA7940F2A053C1F6FF731B689A42E0
S214013E502AD041F2F803C1F6FF731B6818464FF4E7
S214013E604051C0F23F0100F093F90346002B12D0F7
S214013E7041F2F803C1F6FF731B6818464FF4405130
S214013E80C0F23F014FF0040240F2A053C1F6FF73A7
S214013E9000F09EFB08E04CF29460C0F2030018F0BC
S214013EA043F84FF0000301E04FF00103184607F115
S214013EB00807BD4680BD00BF80B582B000AF4CF29A
S214013EC0BC60C0F203004FF0000118F0E7F80246AC
S214013ED041F2F803C1F6FF731A6041F2F803C1F626
S214013EE0FF731B68002B08D14CF2C460C0F20300BC
S214013EF018F01AF84FF000038DE04FF43453C0F277
S214013F0031137B6041F2F803C1F6FF731A6807F1BB
S214013F100403104640F602611A4618F027F80346D5
S214013F20002B0AD04CF2D460C0F2030017F0FCFF5D
S214013F3000F076F84FF000036DE04FF000037B6071
S214013F4041F2F803C1F6FF731A6807F1040310463D
S214013F5040F604611A4618F009F80346002B0AD009
S214013F604CF2E460C0F2030017F0DEFF00F058F8F0
S214013F704FF000034FE04FF001037B6041F2F8037E
S214013F80C1F6FF731A6807F10403104640F60A618A
S214013F901A4617F0EBFF0346002B0AD04CF2F460EA
S214013FA0C0F2030017F0C0FF00F03AF84FF000032C
S214013FB031E04FF000037B6041F2F803C1F6FF7376
S214013FC01A6807F10403104640F608611A4617F00E
S214013FD0CDFF0346002B0AD04CF20470C0F203005A
S214013FE017F0A2FF00F01CF84FF0000313E041F2B7
S214013FF0F803C1F6FF731B68184600F02BF841F270
S214014000F803C1F6FF731B6818464FF0000100F075
S21401401059F94FF00103184607F10807BD4680BD60
S21401402080B582B000AF41F2F803C1F6FF731B689A
S214014030184618F0E9F978607B68002B06D04CF238
S2140140401470C0F20300796817F06EFF07F10807D5
S214014050BD4680BD80B584B000AF786040F2646331
S214014060C1F6FF734FF090021A7040F26463C1F616
S214014070FF734FF000025A7040F26463C1F6FF739B
S2140140804FF000029A7040F26463C1F6FF734FF07E
S2140140900002DA70786840F26461C1F6FF714FF091
S2140140A0040217F07DFD0346FB60FB68042B08D075
S2140140B04CF23C70C0F2030017F036FF4FF00003DD
S2140140C026E007F10803786819464FF0020217F058
S2140140D0C5FE0346FB60786818F064F93B7A1A4619
S2140140E07B7A4CF24C70C0F2030011461A4617F068
S2140140F01BFF3B7ABF2B09D17B7A4A2B06D140F2B4
S2140141006263C1F6FF734FF001021A704FF00103AC
S214014110184607F11007BD4680BD00BF80B584B0C4
S21401412000AF786078684FF0010100F08BF878688E
S21401413000F01CF940F26463C1F6FF734FF0C7024A
S2140141401A70786840F26461C1F6FF714FF001029F
S21401415017F026FD0346FB60786818F023F909E09E
S2140141604FF47A701AF062FD4CF26870C0F20300E8
S21401417017F0DAFE786800F0F9F8034603F0010359
S214014180002BEDD1FB68184607F11007BD4680BD30
S21401419080B584B000AF7860396078684FF001016F
S2140141A000F050F8786800F0E1F840F26463C1F678
S2140141B0FF734FF020021A704FF00303FB6013E009
S2140141C0FB68C3F103034FEAC3033A6822FA03F319
S2140141D0DAB240F26463C1F6FF73F9685B181A70CD
S2140141E0FB6803F1FF33FB60FB68002BE8D17868BE
S2140141F040F26461C1F6FF714FF0040217F0D0FC83
S2140142000346FB60786818F0CDF84FF028001AF0E6
S2140142100DFD09E04CF26C70C0F2030017F084FE4D
S2140142204FF005001AF002FD786800F09FF803468B
S21401423003F00103002BEDD1FB68184607F11007C8
S214014240BD4680BD80B584B000AF78600B46FB707C
S214014250FB78002B07D040F26463C1F6FF734FF082
S21401426006021A7006E040F26463C1F6FF734FF06F
S21401427004021A70786840F26461C1F6FF714FF06B
S214014280010217F08DFC0346FB60786818F08AF887
S21401429009E04CF29470C0F2030017F045FE4FF0AF
S2140142A005001AF0C3FC786800F060F8034603F0D6
S2140142B00103002BEDD1FB68184607F11007BD4638
S2140142C080BD00BF80B586B000AF78600B46FB703E
S2140142D04FF000033B6140E078684FF00101FFF7C3
S2140142E0B1FFFB78002B03D04FF0FF03FB7302E016
S2140142F04FF00003FB7340F26463C1F6FF734FF0A7
S21401430001021A7040F26463C1F6FF73FA7B5A70B9
S214014310786840F26461C1F6FF714FF0020217F04F
S2140143203FFC03467B61786818F03CF809E04CF2E4
S214014330C070C0F2030017F0F7FD4FF005001AF049
S21401434075FC786800F012F8034603F00103002BB1
S214014350EDD13B6903F101033B613B69002BBBD007
S2140143607B69184607F11807BD4680BD80B584B045
S21401437000AF78604FF0FF03FB7240F26463C1F652
S214014380FF734FF005021A70786840F26461C1F657
S214014390FF714FF0010217F003FC0346FB60FB6858
S2140143A0012B07D04CF2E870C0F2030017F0BCFDF9
S2140143B0FB7A0DE007F10B03786819464FF001020E
S2140143C017F04CFD0346FB60786817F0EBFFFB7AAD
S2140143D0184607F11007BD4680BD00BF80B586B000
S2140143E000AFF860B9601346FB71F8684FF0010141
S2140143F0FFF728FFF868FFF7B9FF40F26463C1F6DC
S214014400FF734FF002021A704FF003037B6113E053
S2140144107B69C3F103034FEAC303BA6822FA03F3C5
S214014420DAB240F26463C1F6FF7379695B181A70F9
S2140144307B6903F1FF337B617B69002BE8D140F296
S2140144406463C1F6FF73FA791A71F86840F2646121
S214014450C1F6FF714FF0050217F0A2FB03467B6120
S214014460F86817F09FFF09E04CF2F870C0F20300FD
S21401447017F05AFD4FF005001AF0D8FBF868FFF761
S21401448075FF034603F00103002BEDD17B69184647
S21401449007F11807BD4680BD80B586B000AFF8604D
S2140144A0B9601346FB714FF00003FB752CE0FB79F6
S2140144B0F868B9681A46FFF791FFF868B96800F01E
S2140144C033F80346BB75BA7DFB799A4202D14FF0A9
S2140144D0010324E0BB7DFF2B08D04CF61C00C0F284
S2140144E0030017F021FD4FF0000318E0FB7D03F1F8
S2140144F001034CF64400C0F20300194617F014FD00
S214014500FB7D03F10103FB75FB7D022BCFD94CF636
S2140145107000C0F2030017F007FD4FF000031846C5
S21401452007F11807BD4680BD80B584B000AF78603E
S21401453039604FF00003FB7240F26463C1F6FF730B
S2140145404FF003021A704FF00303FB6013E0FB68A1
S214014550C3F103034FEAC3033A6822FA03F3DAB25C
S21401456040F26463C1F6FF73F9685B181A70FB6862
S21401457003F1FF33FB60FB68002BE8D1786840F25B
S2140145806461C1F6FF714FF0040217F009FB0346A0
S214014590FB60FB68042B07D04CF68C00C0F20300CE
S2140145A017F0C2FCFB7A0DE007F10B037868194699
S2140145B04FF0010217F052FC0346FB60786817F0D3
S2140145C0F1FEFB7A184607F11007BD4680BD00BF15
S2140145D080B58AB000AFF860B9607A603B604FF092
S2140145E00003BB614FF000037B617B683B6158E1D0
S2140145F0F8684FF00101FFF725FEF868FFF7B6FEF1
S2140146003B697B62BB68DBB2C3F580727B6A9A4208
S21401461004D2BB68DBB2C3F580737B623A697B6AFE
S214014620D31A3B6140F26263C1F6FF731B78002B1D
S21401463007D040F26463C1F6FF734FF0AD021A7003
S21401464006E040F26463C1F6FF734FF002021A708F
S2140146504FF003033B6213E03B6AC3F103034FEAE7
S214014660C303BA6822FA03F3DAB240F26463C1F60E
S214014670FF73396A5B181A703B6A03F1FF333B62BA
S2140146803B6A002BE8D1F86840F26461C1F6FF711D
S2140146904FF0040217F084FA0346BB614FF004039F
S2140146A07B6140F26263C1F6FF731B78002B00F05A
S2140146B0AE804FF000033B623DE03B6A002B17D013
S2140146C040F26463C1F6FF734FF0AD021A70F868EA
S2140146D040F26461C1F6FF714FF0010217F060FA13
S2140146E00346BA69D318BB617B6903F101037B6199
S2140146F03A683B6AD318F86819464FF0020217F079
S2140147004FFA0346BA69D318BB617B6903F102030A
S2140147107B61F86817F046FE4FF00003FB6103E08B
S214014720FB6903F10103FB61FB693B2BF8D93B6A8B
S21401473003F102033B627A6A3B6AD31A012BBCD8A7
S2140147403A6A7B6A9A4249D23B6A002B17D040F2FA
S2140147506463C1F6FF734FF0AD021A70F86840F259
S2140147606461C1F6FF714FF0010217F019FA0346B2
S214014770BA69D318BB617B6903F101037B613A68AF
S2140147803B6AD3181A7840F26463C1F6FF731A7055
S21401479040F26463C1F6FF734FF0FF025A70F86887
S2140147A040F26461C1F6FF714FF0020217F0F8F9AA
S2140147B00346BA69D318BB617B6903F102037B61C7
S2140147C0F86817F0EFFD4FF00003FB6103E0FB69AB
S2140147D003F10103FB61FB693B2BF8D940F26463EB
S2140147E0C1F6FF734FF004021A70F86840F2646174
S2140147F0C1F6FF714FF0010217F0D2F90346BA690C
S214014800D318BB617B6903F101037B610DE07B6A11
S214014810F86839681A4617F0C3F90346BA69D31817
S214014820BB617A697B6AD3187B61F86817F0BAFDB9
S214014830BA697B699A4209D04CF69C00C0F2030023
S21401484017F072FB7A683B69D31A2FE0BA687B6A65
S214014850D318BB603A687B6AD3183B6040F2626348
S214014860C1F6FF731B7883F00103DBB2002B0FD078
S2140148704FF005001AF0DAF90AE04CF6A800C0F28B
S214014880030017F051FB4FF005001AF0CFF900E0D6
S21401489000BFF868FFF76AFD034603F00103002B2B
S2140148A0EBD13B69002B7FF4A3AE7B68184607F17A
S2140148B02807BD4680BD00BF90B58BB002AFF8603B
S2140148C0B9607A603B604FF00003FB7792E0F868CE
S2140148D0B9687A683B68FFF77BFEF868B9687A685A
S2140148E040F26873C1F6FF7300F096F878617A6952
S2140148F07B689A4206D04CF6CC00C0F2030017F053
S21401490013FB73E0386840F26871C1F6FF717A688C
S21401491022F028FC0346002B02D14FF0010375E07C
S2140149204CF6F000C0F20300B9687A6817F0FCFA9A
S2140149304CF61C10C0F2030017F0F6FA4FF0000315
S214014940BB612FE03A68BB69D3181B781A4640F260
S2140149506873C1F6FF73B9695B181B781C46396822
S214014960BB69CB18197840F26873C1F6FF73B86952
S2140149701B181B78994204D14CF62C13C0F2030382
S21401498003E04CF63013C0F2030300934CF63410E8
S214014990C0F20300B969234617F0C6FABB6903F1F2
S2140149A00103BB61BA697B689A42CBD340F2687057
S2140149B0C1F6FF70796800F0F7F8034683F001034B
S2140149C0DBB2002B08D04CF65010C0F2030017F0F3
S2140149D0ABFA4FF0000319E0FB7F03F101034CF63D
S2140149E07810C0F20300194617F09EFAFB7F03F118
S2140149F00103FB77FB7F022B7FF669AF4CF6A41011
S214014A00C0F2030017F090FA4FF00003184607F1C2
S214014A102407BD4690BD00BF80B586B000AFF860E4
S214014A20B9607A603B6040F26463C1F6FF734FF091
S214014A3003021A704FF003037B6113E07B69C3F135
S214014A4003034FEAC303BA6822FA03F3DAB240F269
S214014A506463C1F6FF7379695B181A707B6903F1A9
S214014A60FF337B617B69002BE8D1F86840F2646113
S214014A70C1F6FF714FF0040217F092F803467B610E
S214014A807B69042B08D04CF6C010C0F2030017F067
S214014A904BFA4FF0000381E007F11003F86840F687
S214014AA00D611A4617F062FA0346002B08D04CF641
S214014AB0D010C0F2030017F037FA4FF000036DE094
S214014AC03B6943F400333B6107F11003F86840F695
S214014AD00E611A4617F04AFA0346002B08D04CF628
S214014AE0E010C0F2030017F01FFA4FF0000355E084
S214014AF0F86817F057FC7B68F86839681A4617F0AB
S214014B00ADF903467B6107F11003F86840F61761BB
S214014B101A4617F02BFA0346002B08D04CF6F01075
S214014B20C0F2030017F000FA4FF0000336E007F179
S214014B301003F86840F60D611A4617F017FA034697
S214014B40002B08D04CF60020C0F2030017F0ECF959
S214014B504FF0000322E03B6923F400333B6107F189
S214014B601003F86840F60E611A4617F0FFF903467F
S214014B70002B08D04CF61020C0F2030017F0D4F931
S214014B804FF000030AE07A697B689A4205D04CF63A
S214014B902020C0F2030017F0C7F97B69184607F119
S214014BA01807BD4680BD00BF80B485B000AF7860F1
S214014BB039604FF00003FB730EE07B681B78FF2B18
S214014BC002D04FF000030DE07B6803F101037B6028
S214014BD0FB7B03F10103FB73FA7B3B689A42ECD340
S214014BE04FF00103184607F11407BD4680BC704715
S214014BF080B59EB000AF78604FF000037B674CF63F
S214014C003020C0F203004FF0000117F047FA0246C9
S214014C1040F67403C1F6FF731A6040F67403C1F6DA
S214014C20FF731B68002B10D14CF63820C0F203002E
S214014C3017F07AF94CF65020C0F2030017F074F919
S214014C404FF000001CF0DEFF5AE04CF66820C0F280
S214014C50030017F069F94FF0C80019F0E7FF01F0FB
S214014C60C9F900E000BF40F2C143C1F6FF731B78EB
S214014C70002B18D040F67403C1F6FF731A6807F1CB
S214014C800803104619464FF0030200F03DF8386756
S214014C903B6F002B07DD3B6FDBB207F108021046C6
S214014CA0194600F08BF84FF002001AF0BFF840F6F4
S214014CB02D73C1F6FF731B78002B1DD07B6F03F19C
S214014CC001037B677A6F40F6C4139A42CADD40F649
S214014CD02D73C1F6FF731B784CF68420C0F20300D7
S214014CE0194617F021F94CF69820C0F2030017F088
S214014CF01BF90AF0B7F8B5E74FF000037B67B1E799
S214014D0007F17807BD4680BD80B588B000AFF86072
S214014D10B9607A604FF00003FB614FF00003BB619E
S214014D2028E0F86817F002FB0346FB74BB69BA6813
S214014D30D318FA7C1A70FB7C0A2B0CD1BB6903F1E1
S214014D40FF33BA68D3181B780D2B04D1BB6903F166
S214014D50FF337B6126E0BB6903F10103BB61BB69DD
S214014D60642B1ED0FB69002B05D0FB6903F1FF33D2
S214014D70FB6100E000BFF86817F034F90346002B2A
S214014D80CFD14FF001001AF051F8FB6903F101038E
S214014D90FB61FA697B689A42ECD36FF001037B6191
S214014DA000E000BFBB69BA68D3184FF000021A7062
S214014DB07B69184607F12007BD4680BDB0B594B0A3
S214014DC006AF78600B46FB704FF0000387F834306F
S214014DD04FF0000387F8333040F6CF63C1F6FF7318
S214014DE01B78002B40F05686FB7803F1FF33FB70EF
S214014DF0FB78002B00F050867B681B7887F83230F2
S214014E0097F8323087F837304FF0010387F836309D
S214014E100FE097F836307A68D3181A7897F8373053
S214014E20D31887F8373097F8363003F1010387F83F
S214014E30363097F83620FB789A42EAD397F837301F
S214014E400D2B05D897F8373003F1140387F8373060
S214014E50FB787A68D3181B7897F837209A427AD06D
S214014E6078684CF6B421C0F203014FF0050222F037
S214014E70B5F90346002B07D14CF6BC20C0F203005F
S214014E8017F052F800F00FBEFB7803F10103FB7038
S214014E904CF6E020C0F2030017F046F897F83210FF
S214014EA0FA78FB787868C3181B7897F83700009073
S214014EB04CF6F020C0F2030017F036F84FF000036E
S214014EC087F8363011E097F836307A68D3181B78B1
S214014ED04CF62C30C0F20300194617F025F897F867
S214014EE0363003F1010387F8363097F83620FB7821
S214014EF09A42E8D34CF63430C0F2030017F014F8A7
S214014F004FF0000387F8363018E097F836307A68A5
S214014F10D3181B781F2B0BD997F836307A68D3181D
S214014F201B784CF63C30C0F20300194616F0FCFF25
S214014F3097F8363003F1010387F8363097F83620B4
S214014F40FB789A42E1D34CF64030C0F2030016F0EB
S214014F50EBFF00F0A8BD97F83230202B10D1FB787C
S214014F60022B40F09B857B6803F101031B784CF60E
S214014F704430C0F20300194616F0D6FF00F093BD88
S214014F8097F83230562B19D1FB78012B06D097F8BB
S214014F903230184601F01CF800F085BD40F6393372
S214014FA0C1F6FF734FF00C021A7040F25053C1F66F
S214014FB0FF734FF6FF721A8000F075BD97F8323016
S214014FC0582B22D1FB78032B06D097F8323018469F
S214014FD000F0FEFF00F067BD7B6803F101031B785C
S214014FE04FEA03139AB27B6803F102031B784FEA78
S214014FF09303DBB213439AB240F25053C1F6FF73E8
S2140150001A8008F077FF00F04EBD97F83230622B19
S2140150101BD1FB78012B06D097F83230184600F0EA
S214015020D7FF00F040BD41F2FE03C1F6FF731B88B7
S2140150304CF65C30C0F20300194616F075FF4FF0CF
S214015040050002F07BF900F02EBD40F62E73C1F686
S214015050FF731B78002B40F0238597F83230322BF4
S21401506040D1FB78072B06D097F83230184600F06F
S214015070AFFF00F018BD7B6803F105031B784FEA0C
S21401508003139AB27B6803F106031B784FEA930376
S214015090DBB213439BB29AB241F2FC03C1F6FF7333
S2140150A01A8041F2FC03C1F6FF731B88B3F5177F24
S2140150B000F0F98441F2FC03C1F6FF731B884CF63D
S2140150C08430C0F20300194616F02EFF4FF006009A
S2140150D002F034F94FF000004FF0010109F0EEFE46
S2140150E000F0E1BC97F83230332B57D1FB78052B13
S2140150F006D097F83230184600F06AFF00F0D3BCAD
S2140151007B6803F101031B784FEA03139AB27B68AD
S21401511003F102031B784FEA9303DBB213439BB2FE
S2140151209AB241F2FE03C1F6FF731A8041F2FE0302
S214015130C1F6FF731B88B3F5177F15D041F2FE0346
S214015140C1F6FF731B884CF6C030C0F20300194647
S21401515016F0EAFE4FF0050002F0F0F84FF00000FE
S2140151604FF0010109F0AAFE7B6803F103031B78E7
S2140151704FEA03139AB27B6803F104031B784FEAE4
S2140151809303DBB213439BB29BB223F400633B86CB
S2140151903B8E184606F05AF900F085BC97F8323077
S2140151A0342B15D1FB78022B06D097F832301846EF
S2140151B000F00EFF00F077BC7B6803F101031B785B
S2140151C0A3F11403DBB2184608F046FE00F06BBCF0
S2140151D097F83230352B12D1FB78012B06D097F891
S2140151E03230184600F0F4FE00F05DBC40F66D3338
S2140151F0C1F6FF734FF000021A7000F054BC97F826
S2140152003230452B35D17B6803F101031B784FEA19
S21401521003139AB27B6803F102031B784FEA9303E8
S214015220DBB213439BB29AB241F2FE03C1F6FF739F
S2140152301A8041F2FE03C1F6FF731B88B3F5177F90
S2140152400FD041F2FE03C1F6FF731B884CF65C30AB
S214015250C0F20300194616F067FE4FF0050002F093
S2140152606DF87B6803F10503184605F0DDFD00F0D7
S2140152701ABC97F83230462B11D1FB78172B06D083
S21401528097F83230184600F0A3FE00F00CBC7B689D
S21401529003F10303184606F05FF800F004BC97F824
S2140152A03230472B34D17B6803F101031B784FEA78
S2140152B003139AB27B6803F102031B784FEA930348
S2140152C0DBB213439BB29AB241F2FE03C1F6FF73FF
S2140152D01A8041F2FE03C1F6FF731B88B3F5177FF0
S2140152E00FD041F2FE03C1F6FF731B884CF65C300B
S2140152F0C0F20300194616F017FE4FF0050002F043
S2140153001DF87B6803F10503184606F099F9CAE310
S21401531097F83230512B60D1FB78052B05D097F8E2
S2140153203230184600F054FEBDE37B6803F10103FA
S2140153301B784FEA9303DBB203F00303DAB240F6BD
S2140153404533C1F6FF731A707B6803F101031B78BE
S2140153504FEA1313DBB203F00103002B0CBF00234B
S2140153600123DBB287F82F307B6803F102031B7839
S214015370A3F11403DBB2184608F0AAFF7B6803F119
S21401538003031B784FEA03139AB27B6803F1040305
S2140153901B784FEA9303DBB213439BB29AB240F6F3
S2140153A0BA63C1F6FF731A8040F64533C1F6FF7340
S2140153B0197897F82F30002B0CBF00230123DAB29F
S2140153C040F6BA63C1F6FF731B88084611461A46B3
S2140153D003F0D0FD01F02AFB65E397F83230522B3B
S2140153E040F01881FB78102B05D097F8323018461C
S2140153F000F0EEFD57E37B6803F101031B784FEAEB
S2140154009303DBB203F00303DAB240F64533C1F689
S214015410FF731A707B6803F101031B7803F0030323
S21401542087F834307B6803F101031B784FEA931346
S214015430DBB203F00103002B0CBF0023012387F826
S21401544033307B6803F102031B78A3F1140387F85A
S2140154502F307B6803F103031B78A3F11403DBB23F
S214015460184608F035FF7B6803F104031B784FEA02
S21401547003139AB27B6803F105031B784FEA930383
S214015480DBB213439BB29AB240F6BA63C1F6FF731E
S2140154901A807B6803F106031B784FEA03139AB25E
S2140154A07B6803F107031B784FEA9303DBB21343D0
S2140154B09BB2BB857B6803F108031B78A3F1140339
S2140154C087F82B307B6803F109031B78A3F11403DB
S2140154D087F82A307B6803F10A031B78A3F11403CB
S2140154E087F829307B6803F10B031B78A3F11403BB
S2140154F087F828307B6803F10C031B78A3F11403AB
S21401550087F827307B6803F10D031B78A3F114039A
S21401551087F826307B6803F10E031B78A3F114038A
S21401552087F825307B6803F10F031B78A3F114037A
S21401553087F8243097F82B204EF68063C0F23603A6
S21401554003FB02F297F82A3044F6206101FB03F3CD
S214015550D21897F829304FF0640101FB03F3D118F4
S21401556097F825304FEA1313DBB21A4613464FEA73
S21401557083039B184FEA4303CB181A4640F6982339
S214015580C1F6FF731A6097F828204EF68063C0F2C2
S214015590360303FB02F297F8273044F6206101FB3D
S2140155A003F3D21897F826304FF0640101FB03F39A
S2140155B0D11897F8253003F00F0213464FEA8303FC
S2140155C09B184FEA4303CB181A4640F69C23C1F6B4
S2140155D0FF731A6040F67003C1F6FF734FF00102C5
S2140155E01A7040F64533C1F6FF73187840F6BA6371
S2140155F0C1F6FF731A88BB8DDCB297F82F1097F8A7
S214015600343097F833500095019403F07BFD01F098
S2140156100DFA48E297F83230532B0ED1FB78022B65
S21401562040F040827B6803F101031B78A3F1140369
S214015630DBB2184608F04CFE35E297F83230632BA1
S2140156401ED1FB78032B05D097F83230184600F0B0
S214015650BFFC28E27B6803F101031B784FEA0313C2
S2140156609AB27B6803F102031B784FEA9303DBB21D
S21401567013439BB27B847B8C184603F0D1FF12E266
S21401568097F83230552B40F08A80FB78072B05D0EF
S21401569097F83230184600F09BFC04E27B6803F171
S2140156A001031B784FEA03139AB27B6803F10203E6
S2140156B01B784FEA9303DBB213439BB29AB240F6D0
S2140156C0BA63C1F6FF731A807B6803F103031B7884
S2140156D04FEA03139AB27B6803F104031B784FEA7F
S2140156E09303DBB213439BB23B847B6803F1050350
S2140156F01B78A3F11403FB777B6803F106031B7881
S214015700A3F11403BB774FF0000387F835303CE074
S21401571097F8352040F6C823C1F6FF7333F81220F8
S21401572040F6BA63C1F6FF731B889A4227D140F64A
S2140157304333C1F6FF7397F835201A7001F0F8F974
S214015740398C97F835301A464FEAC202D3184FEA19
S2140157504303DAB2FB7FD318DAB297F8353018462E
S2140157604FEAC000C3184FEA4303D8B2BB7FC31841
S214015770DBB209B2084611461A4607F0ABFE97F8A7
S214015780353003F1010387F8353040F22353C1F673
S214015790FF731B7897F835209A42B9D383E197F8BF
S2140157A03230572B6BD1FB780B2B05D097F8323064
S2140157B0184600F00DFC76E17B6803F101031B78C7
S2140157C04FEA03139AB27B6803F102031B784FEA90
S2140157D09303DBB213439BB2BB837B6803F10303E2
S2140157E01B784FEA9303FB767B6803F104031B786F
S2140157F04FEA9303BB767B6803F105031B784FEAF8
S21401580093037B767B6803F106031B784FEA031349
S2140158109AB27B6803F107031B784FEA9303DBB266
S21401582013439BB2FB827B6803F108031B784FEAA4
S21401583093037B757B6803F109031B784FEA930397
S2140158403B757B6803F10A031B784FEA9303FB74ED
S214015850BB8BFC8A18B2F97EBA7E7B7E24B200949A
S2140158607C7D01943C7D0294FC7C03944FF0000403
S21401587004944FF00004059407F09CFF13E197F899
S2140158803230592B10D1FB78012B05D097F83230E6
S214015890184600F09DFB06E140F64433C1F6FF735F
S2140158A04FF002021A70FEE097F83230612B2FD1CA
S2140158B0FB78032B05D097F83230184600F088FBAA
S2140158C0F1E07B6803F101031B784FEA03139AB2F8
S2140158D07B6803F102031B784FEA9303DBB21343A1
S2140158E09AB240F25053C1F6FF731A8040F25053F9
S2140158F0C1F6FF731B881BB2B3F5FA6F40F0D38075
S21401590040F25053C1F6FF734FF6FF721A80CAE099
S21401591097F83230652B3DD17B6803F101031B7884
S2140159204FEA03139AB27B6803F102031B784FEA2E
S2140159309303DBB213433B8240F25053C1F6FF732D
S2140159401B88B7F910201BB29A4209D097F832305B
S2140159504CF6F030C0F20300194616F0E5FAA2E064
S21401596040F67633C1F6FF731B7883F00103DBB292
S214015970002B00F0988040F66F33C1F6FF731B785A
S214015980002B00F090807B6803F10303184607F0B4
S2140159906FFA88E097F83230812B6BD1FB78042BB5
S2140159A005D097F83230184600F012FB7BE07B6892
S2140159B003F101031B784FEA03139AB27B6803F1E4
S2140159C002031B784FEA9303DBB213439BB29AB2EE
S2140159D040F6BA63C1F6FF731A807B6803F10303CE
S2140159E01B78A3F11403FB734FF0000387F83530DF
S2140159F036E097F8352040F6C823C1F6FF7333F832
S214015A00122040F6BA63C1F6FF731B889A4221D171
S214015A1040F64333C1F6FF7397F835201A7040F607
S214015A204333C1F6FF731B78184601F081F803F083
S214015A305BF997F835301A464FEAC202D3184FEA97
S214015A404303DAB2FB7BD318DBB218464FF00001F2
S214015A5007F004FE97F8353003F1010387F8353077
S214015A6040F22353C1F6FF731B7897F835209A420C
S214015A70BFD318E097F83230852B14D1FB78012B71
S214015A8005D097F83230184600F0A2FA0BE008F07D
S214015A90C5F908E000BF06E000BF04E000BF02E071
S214015AA000BF00E000BF07F13807BD46B0BD00BF2C
S214015AB080B586B000AFF860B9601346FB714FF051
S214015AC00003BB754FF00003FB750AE0FB7DBA6867
S214015AD0D3181A78BB7DD318BB75FB7D03F1010380
S214015AE0FB75FA7DFB799A42F0D3BB7D0D2B03D86B
S214015AF0BB7D03F11403BB75FB79BA68D318BA7D75
S214015B001A70FB7903F10103BA68D3184FF00D023E
S214015B101A70FB7903F10203F868B9681A4616F0A1
S214015B203FF84FF00003184607F11807BD4680BD41
S214015B3080B588B000AF3B600346FB710B46BB7176
S214015B401346BB80FB793B72FB79A3F12003712BD3
S214015B5000F2128201A252F823F000BF255D010077
S214015B602D5D0100355D01003D5D0100795F01009D
S214015B70795F0100795F0100795F0100795F0100BB
S214015B80795F0100795F0100795F0100795F0100AB
S214015B90795F0100795F0100795F0100455D0100D1
S214015BA07D5E0100855E0100C75E0100795F010030
S214015BB0795F0100795F0100795F0100795F01007B
S214015BC0795F0100795F0100795F0100795F01006B
S214015BD0795F0100795F0100795F0100795F01005B
S214015BE0795F0100795F0100795F0100795F01004B
S214015BF0795F0100795F0100795F0100795F01003B
S214015C00795F0100795F0100795F0100795F01002A
S214015C10795F0100795F0100795F01001D5F010076
S214015C20795F0100795F0100795F0100795F01000A
S214015C30795F0100795F0100795F0100795F0100FA
S214015C40795F0100795F0100795F0100795F0100EA
S214015C50795F0100795F0100795F0100795F0100DA
S214015C60795F0100795F0100795F0100795F0100CA
S214015C70795F0100795F0100795F0100795F0100BA
S214015C80795F0100795F0100795F0100795F0100AA
S214015C90795F0100795F0100795F0100795F01009A
S214015CA0795F0100795F0100795F0100795F01008A
S214015CB0795F0100795F0100795F0100795F01007A
S214015CC0795F0100795F0100795F0100795F01006A
S214015CD0795F0100795F0100795F0100795F01005A
S214015CE0795F0100795F0100795F0100795F01004A
S214015CF0CF5E0100E15E0100795F0100795F01007E
S214015D00F35E0100795F0100795F0100795F0100B0
S214015D10795F0100795F0100795F01000D5F010085
S214015D20155F01004FF00103FB7718E14FF0010307
S214015D30FB7714E14FF00103FB7710E14FF001030D
S214015D40FB770CE140F64333C1F6FF731B781A4626
S214015D5040F6C823C1F6FF7333F812304FEA131327
S214015D609BB2DBB223F00303DBB27B7240F6433314
S214015D70C1F6FF731B781A4640F6C823C1F6FF73B7
S214015D8033F81230DBB24FEA8303DBB2BB7240F664
S214015D90C823C1F6FF731B884FEA13139BB2DBB20D
S214015DA023F00303DBB2FB7240F6C823C1F6FF7390
S214015DB01B88DBB24FEA8303DBB23B7340F6C82392
S214015DC0C1F6FF735B884FEA13139BB2DBB223F075
S214015DD00303DBB27B7340F6C823C1F6FF735B880F
S214015DE0DBB24FEA8303DBB2BB7340F6C823C1F6CE
S214015DF0FF739B884FEA13139BB2DBB223F00303B6
S214015E00DBB2FB7340F6C823C1F6FF739B88DBB297
S214015E104FEA8303DBB23B7440F6C823C1F6FF7337
S214015E20DB884FEA13139BB2DBB223F00303DBB22A
S214015E307B7440F6C823C1F6FF73DB88DBB24FEAFA
S214015E408303DBB2BB7440F6C823C1F6FF731B891C
S214015E504FEA13139BB2DBB223F00303DBB2FB74EE
S214015E6040F6C823C1F6FF731B89DBB24FEA8303F2
S214015E70DBB23B754FF00D03FB7770E04FF001038B
S214015E80FB776CE0BB884FEA13139BB2DBB223F0BF
S214015E900303DBB27B72BB88DBB24FEA8303DBB260
S214015EA0BB723B684FEA1313DBB223F00303DBB28A
S214015EB0FB723B68DBB24FEA8303DBB23B734FF006
S214015EC00503FB774BE04FF00103FB7747E0BB7917
S214015ED003F11403DBB27B724FF00203FB773EE063
S214015EE0BB7903F11403DBB27B724FF00203FB773D
S214015EF035E040F22353C1F6FF731B7803F1140318
S214015F00DBB27B724FF00203FB7728E04FF0010310
S214015F10FB7724E04FF00103FB7720E040F250537B
S214015F20C1F6FF731B881BB24FEA23139BB2DBB289
S214015F3023F00303DBB27B7240F25053C1F6FF73CA
S214015F401B88DBB24FEA8303DBB2BB72BB7903F17A
S214015F501403DBB2FB724FF00403FB7700BF40F67D
S214015F607403C1F6FF73196807F10802FB7F084640
S214015F7011461A46FFF79CFD07F12007BD4680BD76
S214015F8080B582B000AF786040F67403C1F6FF7347
S214015F901B68184679684FF01B02FFF789FD07F169
S214015FA00807BD4680BD00BF80B582B000AF7860EF
S214015FB040F67403C1F6FF731B68184679684FF004
S214015FC00A02FFF775FD07F10807BD4680BD00BF51
S214015FD080B582B000AF0346FB71FB794CF64440B6
S214015FE0C0F20300194615F09FFF07F10807BD46EA
S214015FF080BD00BF80B582B000AF4CF66C40C0F2E9
S21401600003004FF0000116F049F8024640F6780307
S214016010C1F6FF731A6040F67803C1F6FF731B687A
S214016020002B06D14CF67440C0F2030015F07CFF3D
S214016030F9E04CF68C40C0F2030015F075FF4CF603
S214016040A843C0F203033B603B684CF6A840C0F28D
S2140160500300194615F068FF40F67803C1F6FF7392
S2140160601A683B46104640F604511A4615F07EFF64
S2140160700346002B06D14CF6CC40C0F2030015F0C7
S21401608053FF05E04CF6D040C0F2030015F04CFF7C
S2140160904CF6D840C0F2030015F046FF40F67803F0
S2140160A0C1F6FF731A683B46104640F603511A467E
S2140160B015F05CFF0346002B08D13B684CF6F44014
S2140160C0C0F20300194615F02FFF05E04CF6D0404C
S2140160D0C0F2030015F028FF4FF003033B603B6856
S2140160E003F1FF334CF6F840C0F20300194615F0F1
S2140160F01BFF40F67803C1F6FF731A683B4610464D
S21401610040F60E511A4615F031FF0346002B06D114
S2140161104CF6CC40C0F2030015F006FF05E04CF645
S214016120D040C0F2030015F0FFFE4CF62C50C0F232
S214016130030015F0F9FE40F67803C1F6FF731A68FE
S2140161403B46104640F60F511A4615F00FFF034620
S214016150002B0AD13B6803F1FF334CF6F440C0F242
S2140161600300194615F0E0FE05E04CF6D040C0F2FB
S214016170030015F0D9FE4FF2C003C4F20F034FF02F
S21401618080025A604FF28003C4F20F034FF480225C
S2140161905A604FF28003C4F20F034FF400425A6074
S2140161A04FF28003C4F20F034FF480429A604FF01F
S2140161B00003FB801CE0FA8840F67C03C1F6FF73FF
S2140161C04FF000019954FA8840F68433C1F6FF7304
S2140161D04FF0000143F82210FA8840F64813C1F642
S2140161E0FF734FF000019954FB8803F10103FB8014
S2140161F0FB88C82BDFD940F67C00C1F6FF704FF054
S214016200C90100F015F84FF0020018F00FFE40F635
S2140162107C00C1F6FF704FF0C90100F009F84FF09D
S214016220020018F003FE07F10807BD4680BD00BF57
S21401623080B586B000AF786039604FF000033B74DC
S2140162404FF46143FB6040F67803C1F6FF731A68AA
S21401625007F10C03104640F604511A4615F086FE67
S2140162600346002B05D04CF65C50C0F2030015F037
S2140162705BFE4FF00003FB6040F67803C1F6FF7348
S2140162801A6807F10C03104640F603511A4615F03A
S2140162906DFE0346002B0DD140F67803C1F6FF7361
S2140162A01A6807F11003104619464FF0010215F05F
S2140162B077FC05E04CF67850C0F2030015F034FE8A
S2140162C040F67803C1F6FF731B68184616F06AF8A5
S2140162D040F67803C1F6FF731B68184640F618515E
S2140162E04FF0000215F042FE03467B614CF6A843D0
S2140162F0C0F20303FB6040F67803C1F6FF731A6829
S21401630007F10C03104640F604511A4615F02EFE0E
S2140163100346002B05D04CF69850C0F2030015F04A
S21401632003FE4FF00003FB6040F67803C1F6FF73EF
S2140163301A6807F10C03104640F603511A4615F089
S21401634015FE0346002B0BD140F67803C1F6FF730A
S2140163501A683B68104679681A4615F021FC05E074
S2140163604CF6B850C0F2030015F0DEFD07F1180731
S214016370BD4680BD80B500AF09F0D6F84FF2800368
S214016380C4F20F034FF6FF72C0F204025A614FF2D5
S2140163904003C4F20F034FF400625A604FF2400309
S2140163A0C4F20F034FF400129A604FF24003C4F296
S2140163B00F034FF480225A604FF28003C4F20F039A
S2140163C04FF28002C4F20F02126922F0FF021A6035
S2140163D009F0C8F84CF66470C0F2030015F0A4FD8D
S2140163E04FF0F80000F0A4F84FF0000000F0A0F81D
S2140163F04FF0A20000F09CF84FF0A10000F098F8D2
S2140164004FF0200000F094F84FF0C00000F090F834
S2140164104FF0220000F08CF84FF02F0000F088F8C3
S2140164204FF00A0018F002FC4FF0250000F080F84B
S2140164304FF0810000F07CF84FF0190000F078F87A
S2140164404FF0400000F074F84FF0A60000F070F82E
S2140164504FF0A40000F06CF84FF0AF0000F068F8C1
S2140164604FF00A0018F0E2FB00F04CFA80BD00BFC6
S21401647080B483B000AF02460B46FA71BB7141F29D
S2140164801513C1F6FF73FA791A7041F21413C1F6A7
S214016490FF73BA791A7007F10C07BD4680BC7047C6
S2140164A080B582B000AF7860396009E07B681B7800
S2140164B01846396800F0FCF87B6803F101037B603D
S2140164C07B681B78002BF1D107F10807BD4680BD1C
S2140164D080B582B000AF0346FB71FB7903F104037C
S2140164E0FB71FB794FEA1313DBB2DBB243F0100307
S2140164F0DBB2DBB2184600F01BF8FB7903F00F03A2
S214016500DBB2184600F014F807F10807BD4680BD57
S21401651080B582B000AF0346FB71FB7963F04F0391
S214016520DBB2184600F004F807F10807BD4680BD47
S21401653080B582B000AF0346FB7108F0F5FF4FF25D
S2140165408003C4F20F034FF6FF72C0F204025A61D1
S2140165504FF0020009F012F84FF28003C4F20F0365
S2140165604FF28002C4F20F02126922F0FF01FA799B
S2140165700A431A604FF24003C4F20F034FF480122D
S2140165809A604FF24003C4F20F034FF400629A6020
S2140165904FF24003C4F20F034FF480229A604FF289
S2140165A04003C4F20F034FF400125A604FF001008B
S2140165B008F0E4FF4FF24003C4F20F034FF4001259
S2140165C09A604FF24003C4F20F034FF480225A60E0
S2140165D04FF28003C4F20F034FF47F42C0F204026D
S2140165E05A6108F0BFFF07F10807BD4680BD00BF2E
S2140165F080B582B000AF0346FB7108F095FF4FF2FD
S2140166008003C4F20F034FF6FF72C0F204025A6110
S2140166104FF0020008F0B2FF4FF28003C4F20F03FE
S2140166204FF28002C4F20F02126922F0FF01FA79DA
S2140166300A431A604FF24003C4F20F034FF480126C
S2140166405A604FF24003C4F20F034FF400629A609F
S2140166504FF24003C4F20F034FF480229A604FF2C8
S2140166604003C4F20F034FF400125A604FF00100CA
S21401667008F084FF4FF24003C4F20F034FF40012F8
S2140166809A604FF24003C4F20F034FF480225A601F
S2140166904FF28003C4F20F034FF47F42C0F20402AC
S2140166A05A6108F05FFF07F10807BD4680BD00BFCD
S2140166B080B584B000AF03463960FB714FF000032C
S2140166C0FB734FF00103BB7341F21413C1F6FF7362
S2140166D01B781A463B681B78C3F180039A4240F345
S2140166E08D8041F21413C1F6FF734FF000021A7049
S2140166F041F21513C1F6FF731B7803F10103DAB2F9
S21401670041F21513C1F6FF731A7041F21513C1F663
S214016710FF731B78082B71D141F21513C1F6FF7375
S2140167204FF000021A7069E03B685B78082B2DD9A0
S2140167304FF00203BB7341F21413C1F6FF731B78CB
S2140167401846FFF7C5FE41F21513C1F6FF731B7815
S21401675003F1FF33DBB21846FFF7DAFE3B685A68EF
S214016760FB79A3F12003B97B01FB03F339680978B0
S21401677001FB03F1FB7BB87B00FB03F303F1010391
S214016780CB18D3181B781846FFF732FF41F21413C3
S214016790C1F6FF731B781846FFF79AFE41F21513F0
S2140167A0C1F6FF731B781846FFF7B2FE3B685A68BE
S2140167B0FB79A3F12003B97B01FB03F33968097860
S2140167C001FB03F1FB7BB87B00FB03F3CB18D3186B
S2140167D01B781846FFF70CFFFB7B03F10103FB73E5
S2140167E041F21413C1F6FF731B7803F10103DAB209
S2140167F041F21413C1F6FF731A7000E000BF3B6844
S2140168001B78FA7B9A428FD341F21413C1F6FF73B9
S2140168101B78DBB25BB2002B2EDB3B685B78082B68
S21401682016D941F21513C1F6FF731B7803F1FF3336
S214016830DBB21846FFF76CFE4FF00000FFF7D8FEFC
S21401684041F21413C1F6FF731B781846FFF740FE9A
S21401685041F21513C1F6FF731B781846FFF758FE71
S21401686041F21413C1F6FF731B781846FFF730FE8A
S2140168704FF00000FFF7BCFEFB7B03F10103FB7347
S21401688041F21413C1F6FF731B7803F10103DAB268
S21401689041F21413C1F6FF731A7007F11007BD46D3
S2140168A080BD00BF80B500AF00F026F84FF00000B5
S2140168B04FF0010100F056F84FF001004FF00101D2
S2140168C000F050F800F0B2F800F0FEF840F66E3333
S2140168D0C1F6FF731B7883F00103DBB2002B02D0F5
S2140168E000F026F907E040F66F33C1F6FF731B7818
S2140168F0184600F05DF980BD80B500AF00F002F8E3
S21401690080BD00BF80B582B000AF4FF00003FB71C1
S2140169104FF00003BB714FF00003FB711BE0FB79E6
S2140169201846FFF7F5FD4FF00000FFF7D1FD4FF0D9
S2140169300003BB7107E04FF00000FFF759FEBB797B
S21401694003F10103BB71BB795BB2002BF3DAFB7970
S21401695003F10103FB71FB79072BE0D907F1080767
S214016960BD4680BD80B586B000AF02460B46FA71C3
S214016970BB7140F21F53C1F6FF731B78002B50D139
S214016980FB79002B22D14FF001004FF00501FFF7F4
S2140169906FFDBB79002B0FD040F66833C1F6FF734D
S2140169A01B7807F10C0210464CF67C71C0F203010D
S2140169B01A4615F0E1F92BE007F10C0318464CF6E0
S2140169C08471C0F2030115F0D7F921E04FF00300FE
S2140169D04FF00501FFF74CFDBB79002B0FD040F6B9
S2140169E06933C1F6FF731B7807F10C0210464CF6AB
S2140169F08C71C0F203011A4615F0BEF908E007F1E2
S214016A000C0318464CF69471C0F2030115F0B4F964
S214016A1007F10C0318464AF66851C0F20301FFF766
S214016A203FFD07F11807BD4680BD00BF80B584B0A5
S214016A3000AF40F21F53C1F6FF731B78002B3FD106
S214016A404FF005004FF00501FFF712FD40F2275306
S214016A50C1F6FF731B78632B09D907F104031846A7
S214016A604CF69C71C0F2030115F086F91FE040F266
S214016A702753C1F6FF731B78002B09D107F10403D6
S214016A8018464CF6A471C0F2030115F075F90EE034
S214016A9040F22753C1F6FF731B7807F10402104634
S214016AA04CF6AC71C0F203011A4615F065F907F110
S214016AB0040318464AF66851C0F20301FFF7F0FCDA
S214016AC007F11007BD4680BD80B584B000AF40F227
S214016AD01F53C1F6FF731B78002B24D14FF007001C
S214016AE04FF00501FFF7C4FC40F66A33C1F6FF73A9
S214016AF01B781A4640F25853C1F6FF7353F82230FA
S214016B0007F1040210464CF6B471C0F203011A46AE
S214016B1015F032F907F1040318464AF66851C0F237
S214016B200301FFF7BDFC07F11007BD4680BD00BF9E
S214016B3080B584B000AF40F21F53C1F6FF731B78D7
S214016B40002B30D14FF002004FF03501FFF790FCDB
S214016B5040F64333C1F6FF731B7803F1410307F197
S214016B60040210464CF6B871C0F203011A4615F03D
S214016B7003F907F1040318464AF67851C0F20301F7
S214016B80FFF78EFC40F64333C1F6FF731B781A46B7
S214016B9040F6C823C1F6FF7333F81230184600F0EA
S214016BA087FA00F0AFFA07F11007BD4680BD00BFB7
S214016BB080B586B000AF0346FB7140F21F53C1F6A5
S214016BC0FF731B78002B5AD14FF002004FF03501AE
S214016BD0FFF74EFC07F10C0318464CF6C471C0F2E1
S214016BE0030115F0C9F807F10C0318464AF6785167
S214016BF0C0F20301FFF754FC4FF004004FF03501DB
S214016C00FFF736FCFB79012B0FD140F6B863C1F6CE
S214016C10FF731B7807F10C0210464CF6D071C0F2D8
S214016C2003011A4615F0A8F808E007F10C03184608
S214016C304CF6DC71C0F2030115F09EF807F10C0367
S214016C4018464AF67851C0F20301FFF729FC4FF0C7
S214016C5006004FF03501FFF70BFC07F10C03184651
S214016C604CF6C471C0F2030115F086F807F10C0367
S214016C7018464AF67851C0F20301FFF711FC07F1F6
S214016C801807BD4680BD00BFF0B599B004AF41F20C
S214016C90F803C1F6FF731B68002B00F0F480FCF7C5
S214016CA0F3F941F2F803C1F6FF731A6807F12A03F4
S214016CB010464FF48051C0F23F014FF00202FDF73B
S214016CC0ABFEFCF7FDF97B8D002B00F0DC80FCF7BA
S214016CD0DBF941F2F803C1F6FF731A6807F12803DE
S214016CE0104641F20201C0F23F014FF00202FDF7E9
S214016CF093FE41F2F803C1F6FF731A6807F1260303
S214016D00104641F20401C0F23F014FF00202FDF7C6
S214016D1083FE41F2F803C1F6FF731A6807F1040314
S214016D20104641F20A01C0F23F014FF02102FDF781
S214016D3073FEFCF7C5F93A8DFB8C1046194606F032
S214016D402FFBFFF7D9FD07F12C0318464CF6E87127
S214016D50C0F2030115F010F84FF001004FF00101E9
S214016D60FFF786FB07F12C0318464AF67851C0F266
S214016D700301FFF795FB4FF003004FF00101FFF70A
S214016D8077FB07F1040318464AF66051C0F2030187
S214016D90FFF786FB41F22413C1F6FF735B8803F10C
S214016DA0FF3240F2C443C1F6FF7353F8222041F28A
S214016DB02413C1F6FF731B881C4641F22413C1F647
S214016DC0FF739B88A3F5FA6641F22413C1F6FF739D
S214016DD0DB881D4641F22413C1F6FF731B89184652
S214016DE041F22413C1F6FF735B89194607F12C03A0
S214016DF0009601950290039118464CF6F471C0F284
S214016E000301234614F0B8FF4FF006004FF00101CE
S214016E10FFF72EFB07F12C0318464AF66051C0F225
S214016E200301FFF73DFB7B8D07F12C0210464DF267
S214016E301001C0F203011A4614F09EFF07F12C035D
S214016E40184620F0C3F902464AF66053C0F203031F
S214016E501B7803FB02F34FEA5303DBB2C3F13B0398
S214016E60DBB24FF007001946FFF702FB07F12C03D0
S214016E7018464AF66051C0F20301FFF711FB41F2D2
S214016E80941017F0D3FE07F15407BD46F0BD00BFBE
S214016E9080B58AB000AFFFF72FFD07F1040318464F
S214016EA04DF21C01C0F2030114F066FF4FF0010021
S214016EB04FF00101FFF7DCFA07F1040318464AF622
S214016EC06851C0F20301FFF7EBFA07F10403184615
S214016ED04DF22C01C0F2030114F04EFF07F104033A
S214016EE0184620F073F902464AF66853C0F20303C7
S214016EF01B7803FB02F34FEA5303DBB2C3F13B03F8
S214016F00DBB24FF005001946FFF7B2FA07F10403AA
S214016F1018464AF66851C0F20301FFF7C1FA40F27B
S214016F201F53C1F6FF734FF014021A7040F6142374
S214016F30C1F6FF734FF000021A7007F12807BD462D
S214016F4080BD00BF80B58CB000AF0346FB8040F229
S214016F501F53C1F6FF731B78002B0AD040F614238B
S214016F60C1F6FF731B7883F00103DBB2002B40F000
S214016F709A8041F2F803C1F6FF731B68002B00F0FC
S214016F809280FCF781F841F2F803C1F6FF731A68A4
S214016F9007F10A0310464FF48051C0F23F014FF04B
S214016FA00202FDF739FDFCF78BF840F21F53C1F6DC
S214016FB0FF734FF001021A7040F61423C1F6FF73F7
S214016FC04FF001021A70FFF797FC07F10C03184601
S214016FD04DF21C01C0F2030114F0CEFE4FF0010089
S214016FE04FF00101FFF744FA07F10C0318464AF681
S214016FF06851C0F20301FFF753FAFA887B8907F15B
S2140170000C0108464DF23801C0F2030114F0B4FE3B
S21401701007F10C03184620F0D9F802464AF66853E1
S214017020C0F203031B7803FB02F34FEA5303DBB200
S214017030C3F13B03DBB24FF005001946FFF718FA20
S21401704007F10C0318464AF66851C0F20301FFF730
S21401705027FA07F10C0318464DF24401C0F203016A
S21401706014F08AFE07F10C03184620F0AFF802462A
S2140170704AF66853C0F203031B7803FB02F34FEA98
S2140170805303DBB2C3F13B03DBB24FF006001946F4
S214017090FFF7EEF907F10C0318464AF66851C0F2FD
S2140170A00301FFF7FDF907F13007BD4680BD00BFBC
S2140170B080B586B000AF0346FB8040F21F53C1F691
S2140170C0FF731B78002B19D14FF004004FF03501E8
S2140170D0FFF7CEF9FB8807F10C0210464DF25C0172
S2140170E0C0F203011A4614F047FE07F10C031846D6
S2140170F04AF67851C0F20301FFF7D2F907F11807F3
S214017100BD4680BD80B584B000AF40F21F53C1F6C6
S214017110FF731B78002B3AD14FF006004FF0350174
S214017120FFF7A6F940F25053C1F6FF731B881BB256
S214017130002B09DB40F25053C1F6FF731B881AB2CD
S21401714040F28F139A4209DD07F1040318464DF207
S2140171506801C0F2030114F00FFE0FE040F2505335
S214017160C1F6FF731B881BB207F1040210464DF2ED
S2140171707401C0F203011A4614F0FEFD07F1040380
S21401718018464AF67851C0F20301FFF789F907F16C
S2140171901007BD4680BD00BF90B587B000AF03465F
S2140171A0FB71FFF7A9FB4FF002004FF01901FFF743
S2140171B05FF94DF28000C0F203004AF67851C0F242
S2140171C00301FFF76DF94FF006004FF02B01FFF7B3
S2140171D04FF9FA794CF6CD43CCF6CC43A3FB021318
S2140171E04FEAD303DBB21C46FA794CF6CD43CCF614
S2140171F0CC43A3FB02134FEAD3010B464FEA8303AA
S2140172005B184FEA4303D31ADBB207F10C021046B0
S2140172104DF28C01C0F20301224614F0ADFD07F1D8
S2140172200C0318464AF67851C0F20301FFF738F905
S21401723007F11C07BD4690BD80B500AFFFF75CFBAC
S2140172404FF004004DF29401C0F203014AF6785261
S214017250C0F2030200F074F980BD00BF80B500AF34
S2140172604FF002004FF02B01FFF702F94DF2A0009C
S214017270C0F203004AF67851C0F20301FFF710F995
S2140172804FF004004FF00201FFF7F2F84DF2A800AC
S214017290C0F203004AF67851C0F20301FFF700F985
S2140172A080BD00BF80B584B000AFFFF725FB40F27C
S2140172B02353C1F6FF731B781A4613464FEAC303DE
S2140172C09B184FEA430307F1040210464DF2B8013A
S2140172D0C0F203011A4614F04FFD4FF002004FF0C2
S2140172E00501FFF7C5F807F1040318464AF6705181
S2140172F0C0F20301FFF7D4F84FF005004FF0070185
S214017300FFF7B6F841F20010C1F6FF704DF2C40166
S214017310C0F203014DF2D002C0F2030214F02CFDBC
S21401732041F20010C1F6FF704AF67851C0F203012F
S214017330FFF7B6F807F11007BD4680BD80B586B0E9
S21401734000AF0346FB71FB79062B03D1FB79184688
S21401735000F036F8FFF7D0FAFB7907F10C02104679
S2140173604DF2E401C0F203011A4614F005FD07F1DF
S2140173700C034DF2F000C0F20300194614F0D4FDE0
S21401738007F10C034FF0020019464AF67852C0F294
S214017390030200F0D5F8FA7940F2F443C1F6FF7320
S2140173A053F822304FF0050019464AF67852C0F2DB
S2140173B0030200F0C5F807F11807BD4680BD00BFFF
S2140173C080B58AB002AF0346FB71FFF795FAFB79E9
S2140173D007F1080210464DF2E401C0F203011A4615
S2140173E014F0CAFC07F108034DF2F000C0F20300E6
S2140173F0194614F099FD07F108034FF001001946EC
S2140174004AF67852C0F2030200F09AF8FA7940F28E
S214017410F443C1F6FF7353F822304FF003001946C8
S2140174204AF67852C0F2030200F08AF84FF00500DF
S2140174304FF00A01FFF71CF84DF2F400C0F203000A
S2140174404AF66851C0F20301FFF72AF84FF006002A
S2140174504FF00A01FFF70CF84DF2D000C0F203001E
S2140174604AF66851C0F20301FFF71AF84FF005001B
S2140174704FF04601FEF7FCFF4DF2FC00C0F20300A0
S2140174804AF66851C0F20301FFF70AF84FF006000A
S2140174904FF04601FEF7ECFF41F2FC03C1F6FF7325
S2140174A01A8848F21F53C5F2EB13A3FB02134FEAE7
S2140174B053139BB2FB6141F2FC03C1F6FF731B88B9
S2140174C01A46FB694FF0640101FB03F3D21A4CF62E
S2140174D0CD43CCF6CC43A3FB02134FEAD303BB61E7
S2140174E041F2FC03C1F6FF731B881A46FB694FF095
S2140174F0640101FB03F3D11ABA6913464FEA830309
S2140175009B184FEA4303CB1A7B6107F108037A699C
S214017510009218464DF20411C0F20301FA69BB69E4
S21401752014F02AFC07F1080318464AF66851C0F21F
S2140175300301FEF7B5FF07F12007BD4680BD00BF7A
S21401754080B584B000AF0346B9607A60FB73B86853
S2140175501FF03CFE03467A68127802FB03F34FEAFB
S2140175605303DBB2C3F13B03DBB2FA7B1046194689
S214017570FEF77EFFB8687968FEF792FF07F11007FD
S214017580BD4680BD80B586B000AF4FF008004FF411
S214017590FA6116F001FE47F65530C0F201004FF0D1
S2140175A000014FF001024FF0640317F02BF84FF083
S2140175B0320017F03BFB47F27D60C0F201004FF04E
S2140175C000014FF001024FF47A7317F01BF80246E0
S2140175D041F24C13C1F6FF731A6048F29510C0F2DF
S2140175E001004FF000014FF001024FF0010317F0C8
S2140175F009F807F10403184619F018FE0346002B94
S21401760007D04DF2C810C0F2030014F08DFCF8F755
S2140176101FFF07F1040346F61070C1F6FF70194606
S21401762019F034FF0346002B07D04DF2F010C0F2DC
S214017630030014F079FCF8F70BFF07F11807BD46B5
S21401764080BD00BF80B582B000AF78604DF2942057
S214017650C0F2030014F068FC42F6E06017F0E6FAA8
S21401766040F25453C1F6FF731B78002B01D007F08C
S21401767039F94FF4FA6017F0D9FAF1E780B586B018
S21401768000AFF860B9607A603B6040F62E73C1F6D1
S214017690FF731B78002B40F0538240F21E53C1F655
S2140176A0FF731B78002B06D040F6CA63C1F6FF7342
S2140176B04FF000021A7040F63833C1F6FF731B789C
S2140176C0022B0DD140F6CA63C1F6FF731B7883F017
S2140176D00103DBB2002B03D04FF0010002F058FF8C
S2140176E040F6C423C1F6FF731B78002B19D040F671
S2140176F0C423C1F6FF731B7803F1FF33DAB240F6F9
S214017700C423C1F6FF731A7040F6C423C1F6FF7393
S2140177101B78002B05D14FF064004FF0020107F0F3
S21401772009FB40F66D33C1F6FF731B783C2B4BD03B
S21401773040F66D33C1F6FF731B7803F10103DAB22D
S21401774040F66D33C1F6FF731A7040F66D33C1F61D
S214017750FF731B783C2B29D140F22853C1F6FF73E7
S2140177604FF0E4021A7040F22753C1F6FF734FF050
S214017770E4021A7040F6D463C1F6FF734FF00002BC
S2140177801A7001F001FA40F69023C1F6FF734FF02C
S21401779000021A7040F25253C1F6FF734FF0010215
S2140177A01A704FF0000001F001FB0DE040F66D335A
S2140177B0C1F6FF731B780A2B06D140F22653C1F699
S2140177C0FF734FF000021A7040F6CE63C1F6FF73E6
S2140177D01B78002B23D040F66C33C1F6FF731B7861
S2140177E003F10103DAB240F66C33C1F6FF731A7087
S2140177F040F66C33C1F6FF731B78012B40F2A28171
S21401780040F6CE63C1F6FF734FF000021A7040F6E1
S2140178106C33C1F6FF734FF000021A7092E140F626
S2140178203833C1F6FF731B78022B00F0CD8040F68B
S2140178303D33C1F6FF731B783C2B1DD140F2275315
S214017840C1F6FF734FF0E4021A70FBF79FFA4FF090
S21401785064004FF0640107F06DFA40F6C423C1F6E8
S214017860FF734FF01E021A7040F63D33C1F6FF73E8
S2140178704FF000021A7068E140F63D33C1F6FF731F
S2140178801B7803F10103DAB240F63D33C1F6FF730C
S2140178901A7040F6FA63C1F6FF731B7803F1010311
S2140178A0DAB240F6FA63C1F6FF731A7040F6FA636D
S2140178B0C1F6FF731B78052B40F0868040F6FA630D
S2140178C0C1F6FF734FF000021A7040F22853C1F65A
S2140178D0FF731A7840F22753C1F6FF731A7040F20D
S2140178E02853C1F6FF734FF0E4021A704FF00003FD
S2140178F0FB7540F6CA63C1F6FF731B78002B35D0C3
S21401790040F6FB63C1F6FF731B784A2B11D940F290
S2140179102753C1F6FF731B784A2B0AD840F6CA6371
S214017920C1F6FF734FF000021A704FF00400FAF729
S21401793069FF40F6BA63C1F6FF731B88184606F066
S2140179409DFC0346002B0DD140F22753C1F6FF7371
S2140179501B784A2B06D840F6FB63C1F6FF731B78EB
S2140179604A2B06D94FF00103FB7502E04FF00103E5
S214017970FB75FB7D002B1DD040F6CC63C1F6FF7373
S2140179801B78002B02D04FF0800201E04FF000027E
S21401799040F22753C1F6FF731B78DBB21343DBB209
S2140179A0DBB24FF0850019464FF000024FF000039E
S2140179B0FEF7BEF840F22753C1F6FF731A7840F679
S2140179C0FB63C1F6FF731A7040F63B33C1F6FF73D3
S2140179D01B78002B40F0B88040F6C963C1F6FF73F0
S2140179E01B785BB2002B5EDD40F21F53C1F6FF73BE
S2140179F01B78002B49D140F66833C1F6FF731B781C
S214017A00022B0ED840F6C963C1F6FF731B785BB232
S214017A10052B06D14FF000004FF00001FEF7A2FF44
S214017A2033E040F66933C1F6FF731B78022B0ED89C
S214017A3040F6C963C1F6FF731B785BB2042B06D10F
S214017A404FF001004FF00001FEF78CFF1DE040F6FD
S214017A50CB63C1F6FF731B78002B16D040F66B3351
S214017A60C1F6FF731B781846FFF768FC40F66B33C8
S214017A70C1F6FF731B78012B0CBF00230123DBB279
S214017A804FF00000194607F019FA40F6C963C1F62F
S214017A90FF731B7803F1FF33DAB240F6C963C1F610
S214017AA0FF731A7051E007F091FA40F6CB63C1F606
S214017AB0FF731B78002B1CD040F6CD63C1F6FF7315
S214017AC01B78002B34D040F6CD63C1F6FF734FF020
S214017AD000021A704FF0000001F068F94FF0000044
S214017AE001F0E0F906F0CAFF01F0B2F806F0E4FF93
S214017AF01EE040F6CD63C1F6FF731B7883F00103E9
S214017B00DBB2002B14D040F6CD63C1F6FF734FF005
S214017B1001021A7040F6CC63C1F6FF731B7883F03E
S214017B200103DBB2002B03D04FF0010001F0BAF9DC
S214017B3040F6C963C1F6FF734FF005021A7004E000
S214017B4000BF02E000BF00E000BF07F11807BD4616
S214017B5080BD00BF80B586B000AFF860B9607A60BE
S214017B603B604FF00003FB7440F66F33C1F6FF73C2
S214017B701B78002B53D040F6F863C1F6FF731B78D1
S214017B8003F10103DAB240F6F863C1F6FF731A7027
S214017B9040F6F863C1F6FF731B78012B3FD940F618
S214017BA0F863C1F6FF734FF000021A7040F6902397
S214017BB0C1F6FF731B7883F00103DBB2002B2ED0D6
S214017BC040F69123C1F6FF731B7883F00103DBB205
S214017BD0002B24D040F67233C1F6FF731B7883F076
S214017BE00103DBB2002B1AD04FF00003BB820BE07F
S214017BF0BA8A40F67C03C1F6FF734FF00001995430
S214017C00BB8A03F10103BB82BB8AC82BF0D940F6BD
S214017C107C00C1F6FF704FF0C901FEF709FB40F684
S214017C20F963C1F6FF731B7803F10103DAB240F67C
S214017C30F963C1F6FF731A7040F6F963C1F6FF7374
S214017C401B78042B30D940F6F963C1F6FF734FF069
S214017C5000021A7040F63833C1F6FF731B78022B08
S214017C6022D140F64433C1F6FF731B78032B1BD198
S214017C7040F67633C1F6FF731B7883F00103DBB25F
S214017C80002B0FD040F66F33C1F6FF731B78002B25
S214017C9008D040F6B863C1F6FF731B78184605F0A6
S214017CA0D3F801E002F08AFB40F63933C1F6FF73E0
S214017CB01B78002B36D040F63933C1F6FF731B789C
S214017CC003F1FF33DAB240F63933C1F6FF731A70A7
S214017CD040F63933C1F6FF731B7803F00103DBB2BC
S214017CE0002B0CBF00230123DBB24FF01400194612
S214017CF04FF0000206F02CFF40F63933C1F6FF7351
S214017D001B78142B0ED103E04FF00A0016F08EFFFD
S214017D1040F6FC63C1F6FF735B78002BF4D107F0E5
S214017D20A1F833E240F64033C1F6FF731B78002B0F
S214017D3015D040F64033C1F6FF731B7803F1FF33CD
S214017D40DAB240F64033C1F6FF731A7040F640339C
S214017D50C1F6FF731B78002B01D106F0ADFE40F68D
S214017D60D163C1F6FF731B78002B01D006F0DCF857
S214017D704FF00003FB75D8E0FA7D40F24453C1F69C
S214017D80FF7333F812301BB2002BC0F2CA80FA7DA3
S214017D9040F24453C1F6FF7333F8123003F1FF3358
S214017DA099B240F24453C1F6FF7323F81210FA7DDC
S214017DB040F24453C1F6FF7333F81230002B40F003
S214017DC0AD80FA7D40F21453C1F6FF739A5CF97DDB
S214017DD040F63033C1F6FF735B5C9A424FD3FA7DAF
S214017DE040F6C063C1F6FF739B5C03F10103D9B291
S214017DF040F6C063C1F6FF739954FA7D40F6C0633E
S214017E00C1F6FF739B5C5AB2F97D40F21453C1F67A
S214017E10FF735B5C9A4209DDFA7D40F24453C1F67A
S214017E20FF734FF6FF7123F8121077E0FA7DF97DA4
S214017E3040F23853C1F6FF7333F8111040F2445341
S214017E40C1F6FF7323F81210FA7D40F6C063C1F63F
S214017E50FF739B5CDBB218464FF0000100F0B6FEE4
S214017E6040F6CE63C1F6FF734FF001021A7040F67A
S214017E706C33C1F6FF734FF000021A704EE0FA7DC4
S214017E8040F6C063C1F6FF739B5C03F1FF33D9B2C2
S214017E9040F6C063C1F6FF739954FA7D40F6C0639D
S214017EA0C1F6FF739B5C5AB2F97D40F21453C1F6DA
S214017EB0FF735B5C9A4209DAFA7D40F24453C1F6DD
S214017EC0FF734FF6FF7123F8121027E0FA7DF97D54
S214017ED040F23853C1F6FF7333F8111040F24453A1
S214017EE0C1F6FF7323F81210FA7D40F6C063C1F69F
S214017EF0FF739B5CDBB218464FF0000100F066FE94
S214017F0040F6CE63C1F6FF734FF001021A7040F6D9
S214017F106C33C1F6FF734FF000021A704FF0010385
S214017F20FB74FB7D03F10103FB7540F22353C1F69D
S214017F30FF731B78FA7D9A42FFF41EAF40F61423B6
S214017F40C1F6FF731B7883F00103DBB2002B1CD054
S214017F5040F21F53C1F6FF731B78002B15D040F279
S214017F601F53C1F6FF731B7803F1FF33DAB240F2F9
S214017F701F53C1F6FF731A7040F21F53C1F6FF7309
S214017F801B78002B01D1FEF78DFC40F6CE63C1F6BF
S214017F90FF731B78002B0AD040F6CD63C1F6FF7342
S214017FA01B7883F00103DBB2002B40F0EE8040F635
S214017FB03B33C1F6FF731B78002B55D000F03EF91A
S214017FC040F6C863C1F6FF731B78002B39D140F623
S214017FD03E33C1F6FF731B78002B32D140F63F3398
S214017FE0C1F6FF731B78002B2BD140F64133C1F647
S214017FF0FF731B78002B24D140F66E33C1F6FF7356
S2140180001B7883F00103DBB2002B1AD040F63D3318
S214018010C1F6FF734FF000021A7040F6C423C1F692
S214018020FF734FF01E021A7040F62E73C1F6FF73EF
S2140180301B7883F00103DBB2002B15D000F01EFC89
S21401804012E040F66E33C1F6FF731B78002B0BD09F
S21401805040F62E73C1F6FF731B7883F00103DBB283
S214018060002B01D004F0E0FA40F6D363C1F6FF73AB
S2140180701B7883F00103DBB2002B00F0878040F60B
S2140180803C33C1F6FF731B78002B7FD040F63D339F
S214018090C1F6FF734FF000021A7040F6C423C1F612
S2140180A0FF734FF01E021A7040F63C33C1F6FF73A1
S2140180B01B78962B0CD840F63C33C1F6FF731B7821
S2140180C003F10103DAB240F63C33C1F6FF731A70CE
S2140180D040F62E73C1F6FF731B78002B1ED040F6B8
S2140180E03C33C1F6FF731B78092B4FD940F63C335E
S2140180F0C1F6FF731A784CF6CD43CCF6CC43A3FBFE
S21401810002134FEA93010B464FEA83035B18D31A17
S214018110DBB2002B3AD005F087FF37E040F63C3360
S214018120C1F6FF731B78132B30D940F63B33C1F6EB
S214018130FF731B78002B29D140F6FC63C1F6FF7351
S214018140DB7883F00103DBB2002B1FD040F6FC6323
S214018150C1F6FF731B7983F00103DBB2002B15D048
S21401816040F21F53C1F6FF731B78002B0ED140F669
S2140181703C33C1F6FF734FF001021A704FF0010055
S2140181804FF0000106F09AFE00E000BF07F1180765
S214018190BD4680BD80B584B000AFF860B9607A6036
S2140181A03B6040F67003C1F6FF731B78002B0ED0C0
S2140181B040F66C03C1F6FF734FF001021A6040F6F9
S2140181C07003C1F6FF734FF000021A700BE040F621
S2140181D06C03C1F6FF731B6803F1010240F66C03E2
S2140181E0C1F6FF731A6040F6CA63C1F6FF731B78C7
S2140181F0002B10D040F69023C1F6FF731B78002B9E
S21401820009D040F69123C1F6FF731B7883F0010372
S214018210DBB2002B06D140F67233C1F6FF731B7832
S214018220002B05D04FF000004FF0000101F0A0FD3B
S21401823000BF07F11007BD4680BD00BF80B582B004
S21401824000AF4FF00003FB7140F6FC63C1F6FF730D
S2140182501B7883F00103DBB2002B07D040F6C8631E
S214018260C1F6FF734FF000021A7080E040F6383313
S214018270C1F6FF731B78022B76D040F6C863C1F6B1
S214018280FF731B78002B10D102F000F940F6403343
S214018290C1F6FF734FF01E021A7040F6C863C1F6AE
S2140182A0FF734FF001021A705EE040F6FC63C1F600
S2140182B0FF73DB78002B24D040F66A33C1F6FF73D8
S2140182C01B7803F10103DAB240F66A33C1F6FF7395
S2140182D01A7040F66A33C1F6FF731B78052B06D178
S2140182E040F66A33C1F6FF734FF000021A7040F28F
S2140182F06063C1F6FF734FF001021A70FEF7E4FBEC
S2140183002BE040F6FC63C1F6FF731B79002B24D0EB
S21401831040F66A33C1F6FF731B78002B07D140F68F
S2140183206A33C1F6FF734FF004021A700CE040F690
S2140183306A33C1F6FF731B7803F1FF33DAB240F6F6
S2140183406A33C1F6FF731A7040F26063C1F6FF73B9
S2140183504FF001021A70FEF7B7FB40F21E53C1F64A
S214018360FF734FF001021A704FF00103FB7140F6E4
S214018370CE63C1F6FF731B78002B40F0798240F67E
S214018380CD63C1F6FF731B7883F00103DBB2002BCC
S21401839040F06E8240F63C33C1F6FF731B78002B2B
S2140183A058D040F6FC63C1F6FF73DB78002B24D06F
S2140183B040F22253C1F6FF734FF014021A7040F2D6
S2140183C02253C1F6FF731B781846FEF7E5FE40F20E
S2140183D01F53C1F6FF734FF014021A7040F25E632A
S2140183E0C1F6FF734FF001021A7040F21E53C1F638
S2140183F0FF734FF001021A7061E140F6FC63C1F6AB
S214018400FF731B79002B00F05A8140F22253C1F60C
S214018410FF734FF001021A7040F22253C1F6FF7348
S2140184201B781846FEF7B8FE40F21F53C1F6FF73DD
S2140184304FF014021A7040F25E63C1F6FF734FF0FC
S21401844001021A7040F21E53C1F6FF734FF001028B
S2140184501A7034E140F6C863C1F6FF731B78002B2F
S21401846040F02D8140F6FC63C1F6FF73DB7883F0A4
S2140184700103DBB2002B0AD140F6FC63C1F6FF73A1
S2140184801B7983F00103DBB2002B00F0188140F664
S214018490FC63C1F6FF73DB78002B06D140F6FC6364
S2140184A0C1F6FF731B79002B5DD040F63B33C1F656
S2140184B0FF731B78002B30D140F66E33C1F6FF7385
S2140184C01B7883F00103DBB2002B26D040F62E7317
S2140184D0C1F6FF731B7883F00103DBB2002B01D0DA
S2140184E000F0CCF900F0B4FB40F63E33C1F6FF7362
S2140184F04FF000021A7040F63F33C1F6FF734FF09B
S21401850000021A7040F64133C1F6FF734FF00002C5
S2140185101A704FF00103FB71D0E040F63B33C1F611
S214018520FF731B78002B40F0C98040F66E33C1F60E
S214018530FF731B78002B00F0C18040F63833C1F67C
S214018540FF731B78022B00F0B98040F62E73C1F63C
S214018550FF731B7883F00103DBB2002B00F0AE80C3
S21401856004F062F8AAE040F6D263C1F6FF731B7806
S214018570002B7FD040F6CA63C1F6FF734FF00002AE
S2140185801A7040F64333C1F6FF731B781A4640F65D
S2140185908023C1F6FF734FF0000199544FF000009D
S2140185A001F07AF840F64333C1F6FF731B781A469A
S2140185B040F68823C1F6FF734FF00001995440F648
S2140185C04333C1F6FF731B781A4640F6A023C1F663
S2140185D0FF734FF0000123F8121040F64333C1F643
S2140185E0FF731B781A4640F6AC23C1F6FF734FF0B3
S2140185F0000123F812104FF00100FAF703F940F6D4
S2140186009023C1F6FF734FF000021A7040F25253E6
S214018610C1F6FF734FF001021A704FF030004FF0B1
S21401862000014FF000024FF00003FDF781FA40F21F
S2140186301E53C1F6FF734FF001021A7001F0BEFE21
S21401864000F052FB40F6D263C1F6FF734FF0000212
S2140186501A7040F63A33C1F6FF734FF000021A70F3
S21401866000F092FA40F25D63C1F6FF734FF001022B
S2140186701A7024E040F67833C1F6FF731B78002B9E
S2140186801DD040F6CA63C1F6FF734FF000021A70A0
S21401869040F21E53C1F6FF734FF001021A7040F606
S2140186A07833C1F6FF734FF000021A7040F261632F
S2140186B0C1F6FF734FF001021A7000E000BF40F6EA
S2140186C0FC63C1F6FF73DB7883F00103DBB2002B9A
S2140186D010D040F6FC63C1F6FF731B7983F00103EB
S2140186E0DBB2002B06D040F63B33C1F6FF734FF0EA
S2140186F000021A7040F6FC63C1F6FF735B7883F0E4
S2140187000103DBB2002B2BD040F6D363C1F6FF7317
S2140187101B78002B06D040F6D363C1F6FF734FF0EB
S21401872000021A7040F63C33C1F6FF731B78002B2B
S21401873042D040F63C33C1F6FF734FF000021A7088
S21401874040F6D363C1F6FF734FF000021A704FF084
S21401875014004FF000014FF0000206F0F9F92BE08B
S21401876040F63C33C1F6FF731B78002B24D14FF043
S21401877014004FF001014FF0000206F0E9F940F64F
S2140187803933C1F6FF734FF000021A7040F63C33DE
S214018790C1F6FF734FF001021A7040F62E73C1F650
S2140187A0FF731B7883F00103DBB2002B01D0FEF7C9
S2140187B03DF94FF00103FB7140F6FC63C1F6FF7310
S2140187C09B7883F00103DBB2002B07D040F6D06321
S2140187D0C1F6FF734FF000021A7031E040F6D06325
S2140187E0C1F6FF731B7883F00103DBB2002B27D0A1
S2140187F040F6D063C1F6FF734FF001021A7040F6DF
S2140188002E73C1F6FF731B7883F00103DBB2002BD6
S21401881001D005F017FC00F067FA40F64033C1F6C8
S214018820FF731B78002B08D001F030FE40F6403372
S214018830C1F6FF734FF01E021A704FF00103FB7171
S214018840FB79002B15D04FF064004FF0640106F061
S21401885071FA40F6C423C1F6FF734FF01E021A7078
S21401886040F63D33C1F6FF734FF000021A7000E088
S21401887000BF07F10807BD4680BD00BF80B582B0C6
S21401888000AF40F63B33C1F6FF731B78282B0CD89C
S21401889040F63B33C1F6FF731B7803F10103DAB2EE
S2140188A040F63B33C1F6FF731A7040F63B33C1F610
S2140188B0FF731B78282B40F2BB8040F6FC63C1F6A1
S2140188C0FF73DB78002B5CD040F6FC63C1F6FF73C8
S2140188D01B7983F00103DBB2002B52D040F6433301
S2140188E0C1F6FF731B781A4640F64333C1F6FF7391
S2140188F01B78194640F6C823C1F6FF7333F81110EA
S2140189004CF6CD43CCF6CC43A3FB01034FEA9303CD
S2140189109BB203F101039BB219464FEA8101CB18C2
S21401892099B240F6C823C1F6FF7323F8121040F639
S2140189304333C1F6FF731B781A4640F6C823C1F6C7
S214018940FF7333F81230C72B5BD940F64333C1F6B9
S214018950FF731B781A4640F64333C1F6FF731B7844
S214018960194640F6C823C1F6FF7333F81130A3F158
S214018970C80399B240F6C823C1F6FF7323F8121054
S2140189803FE040F64333C1F6FF731B781A4640F6C4
S214018990C823C1F6FF7333F812204CF6CD43CCF64C
S2140189A0CC43A3FB02134FEA93039BB21A464FEA4A
S2140189B08202D3189BB2A3F105039BB2FB80B7F9E1
S2140189C00630002B10DA40F64333C1F6FF731B78EE
S2140189D01A46FB8803F1C80399B240F6C823C1F6CC
S2140189E0FF7323F812100CE040F64333C1F6FF7311
S2140189F01B781A46F98840F6C823C1F6FF7323F898
S214018A00121040F64333C1F6FF731B781A4640F640
S214018A10C823C1F6FF7333F812301846FEF748FB39
S214018A2040F6D263C1F6FF734FF001021A70A6E05A
S214018A3040F63B33C1F6FF731B780A2B07D040F68E
S214018A403B33C1F6FF731B78142B40F2988040F637
S214018A50FC63C1F6FF73DB78002B48D040F6FC635D
S214018A60C1F6FF731B7983F00103DBB2002B3ED006
S214018A7040F64333C1F6FF731B781A4640F6C82307
S214018A80C1F6FF7333F8123003F1010399B240F6D1
S214018A90C823C1F6FF7323F8121040F64333C1F61C
S214018AA0FF731B781A4640F6C823C1F6FF7333F8E6
S214018AB01230C72B4DD940F64333C1F6FF731B78EE
S214018AC01A4640F64333C1F6FF731B78194640F643
S214018AD0C823C1F6FF7333F81130A3F1C80399B266
S214018AE040F6C823C1F6FF7323F8121031E040F6B2
S214018AF04333C1F6FF731B781A4640F6C823C1F606
S214018B00FF7333F81230002B15D040F64333C1F60D
S214018B10FF731B781A4640F6C823C1F6FF7333F875
S214018B20123003F1FF3399B240F6C823C1F6FF7342
S214018B3023F812100DE040F64333C1F6FF731B789D
S214018B401A4640F6C823C1F6FF734FF0C70123F853
S214018B50121040F64333C1F6FF731B781A4640F6EF
S214018B60C823C1F6FF7333F812301846FEF7A0FA91
S214018B7040F6D263C1F6FF734FF001021A7007F197
S214018B800807BD4680BD00BF80B483B000AF4FF07C
S214018B900003FB710CE0FA7940F24453C1F6FF730F
S214018BA04FF6FF7123F81210FB7903F10103FB71F5
S214018BB040F22353C1F6FF731B78FA799A42EAD33F
S214018BC007F10C07BD4680BC704700BF80B582B078
S214018BD000AF02460B46FA71BB714FF0010006F07A
S214018BE0C9F8FA7948F63963C3F6E303A3FB02131F
S214018BF04FEA93010B464FEAC3035B184FEA430360
S214018C00D31ADBB218464FF001014FF0010205F00E
S214018C109FFFFB7918464FF0010106F0C9F8FA7973
S214018C2040F22253C1F6FF731978BB79CB18D9B23B
S214018C3040F6D423C1F6FF73995440F6D163C1F6CA
S214018C40FF734FF001021A7007F10807BD4680BD99
S214018C5080B582B000AF4FF00003FB7131E0FA79C6
S214018C6040F6D423C1F6FF739B5C002B25D0FA791E
S214018C7048F63963C3F6E303A3FB02134FEA9301F5
S214018C800B464FEAC3035B184FEA4303D31ADBB222
S214018C9018464FF000014FF0010205F059FFFB792D
S214018CA018464FF0000106F083F8FA7940F6D4230F
S214018CB0C1F6FF734FF000019954FB7903F10103EC
S214018CC0FB7140F22453C1F6FF731B78FA799A427E
S214018CD0C5D340F6D163C1F6FF734FF000021A7098
S214018CE007F10807BD4680BD80B582B000AF40F6EB
S214018CF04333C1F6FF731B781A464FEAC202D318F4
S214018D004FEA4303FB713CE0FA7940F6D423C1F6FF
S214018D10FF739B5C002B18D0FA7948F63963C3F6CB
S214018D20E303A3FB02134FEA93010B464FEAC30387
S214018D305B184FEA4303D31ADBB218464FF0010122
S214018D404FF0010205F004FF17E0FA7948F639639F
S214018D50C3F6E303A3FB02134FEA93010B464FEA64
S214018D60C3035B184FEA4303D31ADBB218464FF02E
S214018D7000014FF0010205F0EBFEFB7903F1010360
S214018D80FB71F97940F64333C1F6FF731B7803F1A3
S214018D90010213464FEAC3039B184FEA4303994265
S214018DA0B2DB07F10807BD4680BD00BF80B582B0C3
S214018DB000AF0346FB7140F6CC63C1F6FF731B7828
S214018DC083F00103DBB2002B67D1FFF7DDFE05F070
S214018DD055FEFFF73DFF05F06FFE40F64433C1F642
S214018DE0FF731B78022B06D140F64433C1F6FF739E
S214018DF04FF003021A70FB79002B1ED04FF01300C0
S214018E004FF000014FF0000205F0A2FE4FF01200F5
S214018E104FF001014FF0000205F09AFE40F638339C
S214018E20C1F6FF734FF002021A7040F6CD63C1F629
S214018E30FF734FF001021A7030E04FF0000005F0AA
S214018E4099FF4FF012004FF000014FF0000205F0BD
S214018E507FFE40F63833C1F6FF734FF000021A70FA
S214018E6040F67633C1F6FF734FF000021A7040F6F3
S214018E701423C1F6FF731B78002B0FD040F6142382
S214018E80C1F6FF734FF000021A7040F21F53C1F68D
S214018E90FF734FF001021A7000E000BF07F10807E8
S214018EA0BD4680BD80B582B000AF0346FB71FFF7BB
S214018EB06BFE05F0E3FDFFF7CBFE05F0FDFD40F68A
S214018EC0CA63C1F6FF734FF000021A70FB79002BDC
S214018ED03DD04FF0000005F04DFF4FF012004FF06F
S214018EE000014FF0000205F033FE4FF013004FF083
S214018EF001014FF0000205F02BFE4FF00200F9F7DA
S214018F0081FC40F63833C1F6FF734FF001021A7048
S214018F1040F67633C1F6FF734FF000021A7003F085
S214018F208FF840F61423C1F6FF731B78002B1DD073
S214018F3040F61423C1F6FF734FF000021A7040F298
S214018F401F53C1F6FF734FF001021A700EE04FF087
S214018F5013004FF000014FF0000205F0F9FD40F656
S214018F603833C1F6FF734FF000021A7007F1080795
S214018F70BD4680BD80B582B000AF13460246FA7189
S214018F800A46BA71BB8040F6CA63C1F6FF734FF05A
S214018F9000021A7040F22653C1F6FF734FF0010229
S214018FA01A7040F66D33C1F6FF734FF000021A7067
S214018FB040F64433C1F6FF731B78002B11D140F6FF
S214018FC0CC63C1F6FF731B7883F00103DBB2002B81
S214018FD007D040F64433C1F6FF734FF001021A7012
S214018FE006E040F64433C1F6FF734FF000021A70F4
S214018FF040F6CD63C1F6FF731B7883F00103DBB245
S214019000002B02D0FB79012B75D040F63C33C1F61C
S214019010FF731B78002B70D140F25053C1F6FF73DB
S2140190201B881BB2002B69DB40F63D33C1F6FF738C
S2140190304FF000021A7040F63833C1F6FF731B7802
S214019040FA799A4202D1BB79002B2DD0FB79022BFB
S21401905023D140F6CC63C1F6FF731B78002B0BD0EF
S2140190604FF00100FFF7A2FE40F6CD63C1F6FF7395
S2140190704FF001021A7010E040F64433C1F6FF7358
S2140190801B78012B09D14FF091004FF000014FF0F2
S21401909000024FF00003FCF74BFDFB79012B03D1D7
S2140190A04FF00100FFF7FEFE40F63933C1F6FF73BD
S2140190B04FF001021A704FF014004FF001014FF00B
S2140190C0000205F045FDFB79022B17D040F6CA6376
S2140190D0C1F6FF731B7883F00103DBB2002B0DD0C2
S2140190E04FF090004FF000014FF000024FF00003E8
S2140190F0FCF71EFD02E000BF00E000BF07F1080715
S214019100BD4680BD80B584B000AFF871B971BA8034
S214019110FB704FF00003FB7340F66D33C1F6FF732F
S2140191204FF000021A7040F22653C1F6FF734FF05B
S21401913001021A70FB78002B32D040F6CA63C1F6E2
S214019140FF734FF000021A7040F69023C1F6FF73CA
S2140191504FF000021A7040F25253C1F6FF734FF0FF
S21401916001021A7004F0DAFF4FF0000000F094FAE2
S2140191704FF00300F9F746FBFB78012B02D0FB7892
S214019180032B06D140F67633C1F6FF734FF000028B
S2140191901A7040F64433C1F6FF734FF003021A709B
S2140191A03B7E002B0DD040F69023C1F6FF734FF0A7
S2140191B000021A7040F25253C1F6FF734FF00102DB
S2140191C01A7040F6CD63C1F6FF731B7883F0010376
S2140191D0DBB2002B03D0FB79012B00F0188240F69E
S2140191E03C33C1F6FF731B78002B40F0128240F22D
S2140191F05053C1F6FF731B881BB2002BC0F20C82C2
S21401920040F63D33C1F6FF734FF000021A7040F688
S2140192103833C1F6FF731B78FA799A4204D1BB79C9
S21401922003F00103002B1BD0FB79022B11D140F672
S214019230CC63C1F6FF731B78002B0AD04FF00100F8
S214019240FFF7B4FD40F6CD63C1F6FF734FF00102A0
S2140192501A70FB79012B03D14FF00100FFF722FEB4
S21401926040F63933C1F6FF734FF001021A704FF022
S21401927014004FF001014FF0000205F069FCFB7984
S214019280022B40F0B581BB7903F00803002B0CBF1D
S21401929000230123DAB240F6D563C1F6FF731A70D4
S2140192A040F6D563C1F6FF731B78002B07D040F656
S2140192B07A33C1F6FF734FF001021A7027E040F6C9
S2140192C0D763C1F6FF731B78002B19D040F698239D
S2140192D0C1F6FF731A684FF42243C0F24A439A421A
S2140192E00ED140F67A33C1F6FF734FF001021A70C1
S2140192F040F67233C1F6FF734FF000021A7006E0B3
S21401930040F67A33C1F6FF734FF000021A7040F64A
S214019310D563C1F6FF731A7840F6D763C1F6FF73BB
S2140193201A7040F6CA63C1F6FF731B78002B00F073
S2140193305081BB7903F00203002B00F04A8140F60E
S2140193409823C1F6FF731A684FF42243C0F24A43CA
S2140193509A420ED140F69023C1F6FF734FF00002F9
S2140193601A7040F25253C1F6FF734FF001021A70A1
S21401937051E140F69823C1F6FF731A6849F280035B
S214019380C0F281439A4207D140F69123C1F6FF739A
S2140193904FF001021A703EE140F69823C1F6FF73C2
S2140193A01A6844F2FF33C0F695039A424BD940F649
S2140193B09123C1F6FF734FF000021A7040F6902316
S2140193C0C1F6FF731B7883F00103DBB2002B2AD0B2
S2140193D040F25253C1F6FF731B78002B23D04FF097
S2140193E00003FB7309E0FB7B4FF00100194600F018
S2140193F077FFFB7B03F10103FB7340F22353C1F6B6
S214019400FF731B78FA7B9A42EDD340F69023C1F6A0
S214019410FF734FF001021A7040F25253C1F6FF7308
S2140194204FF000021A7040F69823C1F6FF731A68CF
S2140194304FF43C43CFF26A73D3184FF0010019463C
S21401944000F096FCE7E040F69123C1F6FF734FF07B
S21401945000021A7040F69023C1F6FF731B78002BAA
S21401946030D040F69823C1F6FF731B68002B1CD141
S21401947040F69423C1F6FF734FF000021A604FF0D6
S2140194800003FB7309E0FB7B4FF00100194600F077
S21401949027FFFB7B03F10103FB7340F22353C1F665
S2140194A0FF731B78FA7B9A42EDD33A7F40F69823F6
S2140194B0C1F6FF731B68D31818464FF0000100F081
S2140194C079FAA8E040F25253C1F6FF731B78002BDD
S2140194D000F0A18040F69423C1F6FF734FF000021E
S2140194E01A604FF00003FB7309E0FB7B4FF00100AD
S2140194F0194600F0F5FEFB7B03F10103FB7340F216
S2140195002353C1F6FF731B78FA7B9A42EDD340F6DC
S2140195108033C1F6FF734FF000021A8040F6A8634D
S214019520C1F6FF734FF000021A6040F67233C1F6BF
S214019530FF734FF000021A7040F67433C1F6FF73E2
S2140195404FF000021A704FF00003BB7314E0BA7BB1
S21401955040F67C03C1F6FF734FF000019954BA7BC5
S21401956040F68433C1F6FF734FF0000143F8221032
S214019570BB7B03F10103BB73BB7BC82BE7D940F66A
S2140195809023C1F6FF734FF001021A7040F6922342
S214019590C1F6FF734FF000021A7040F25253C1F643
S2140195A0FF734FF000021A7040F69823C1F6FF735E
S2140195B01B68002B2FD03A7F40F69823C1F6FF7325
S2140195C01B68D31818464FF0010100F0F3F900BFED
S2140195D021E040F69023C1F6FF734FF000021A70A7
S2140195E040F25253C1F6FF734FF001021A7013E0B6
S2140195F040F69023C1F6FF734FF000021A7040F256
S2140196005253C1F6FF734FF001021A7004E000BF17
S21401961002E000BF00E000BF07F11007BD4680BDB5
S21401962080B582B000AF0346FB8040F66D33C1F6CD
S214019630FF734FF000021A7040F22653C1F6FF7313
S2140196404FF001021A7040F62E73C1F6FF731B78B5
S214019650002B1AD140F63C33C1F6FF731B78002B62
S21401966015D140F6BC63C1F6FF731B88FA889A428F
S2140196700ED0FB88184600F00FF840F21E53C1F6D4
S214019680FF734FF001021A7002E000BF00E000BF56
S21401969007F10807BD4680BD80B487B000AF03461A
S2140196A0FB8040F6BC63C1F6FF73FA881A804FF060
S2140196B00003FB75A0E04FF00103FB814FF03F0371
S2140196C03B743B7C7B747B7CBB744FF00103BB75A6
S2140196D063E0FA88FB8913409BB2002B55D04FF00C
S2140196E001033B754FF03F03FB744FF000037B759E
S2140196F048E0F97D787D40F61822C1F6FF720B46E8
S2140197004FEAC3035B184FEA43031B18D3181B78B1
S214019710BA7D9A4207D13B7D6FEA0303DAB2FB7C3E
S2140197201340DBB2FB747B7D052B05D07B7D0B2BB9
S21401973002D07B7D112B1DD17B7D052B04D1BA7CFC
S214019740FB7C1340BB740EE07B7D0B2B04D17A7C33
S214019750FB7C13407B7406E07B7D112B03D13A7CA6
S214019760FB7C13403B744FF001033B754FF03F0306
S214019770FB7403E03B7D4FEA43033B757B7D03F1BE
S21401978001037B757B7D112BB3D9FB894FEA43031C
S214019790FB81BB7D03F10103BB75BB7D0C2B98D907
S2140197A0F97D41F23C12C1F6FF720B464FEA4303C4
S2140197B05B18D318BA7C1A70F97D41F23C12C1F6D7
S2140197C0FF720B464FEA43035B18D31803F10103FC
S2140197D07A7C1A70F97D41F23C12C1F6FF720B4693
S2140197E04FEA43035B18D31803F102033A7C1A705D
S2140197F0FB7D03F10103FB7540F22353C1F6FF73B2
S2140198001B78FA7D9A42FFF456AF07F11C07BD4656
S21401981080BC704780B485B000AF03463960FB71E9
S214019820FB79002B11D13B68002B39D140F6D86368
S214019830C1F6FF731B68012B32DC40F6D863C1F614
S214019840FF731B68B3F1FF3F2ADB4FF00003FB6099
S2140198500CE040F6DC63C1F6FF73FA684FF00001D6
S21401986043F82210FB6803F10103FB60FB68042B3D
S214019870EFDD40F6F063C1F6FF734FF000021A60A9
S21401988040F6D863C1F6FF734FF000021A6040F647
S214019890F463C1F6FF734FF000021A603B6882E082
S2140198A040F6F063C1F6FF731A6840F6F463C1F63A
S2140198B0FF73196840F6DC63C1F6FF7353F8213075
S2140198C0D21A40F6F063C1F6FF731A6040F6F463ED
S2140198D0C1F6FF731A6840F6DC63C1F6FF73396898
S2140198E043F8221040F6F063C1F6FF731A683B682E
S2140198F0D21840F6F063C1F6FF731A6040F6F463BF
S214019900C1F6FF731B6803F1010240F6F463C1F66A
S214019910FF731A6040F6F463C1F6FF731B68052BEC
S21401992006D140F6F463C1F6FF734FF000021A60E9
S21401993040F6F063C1F6FF731B68002B17DB40F699
S214019940F063C1F6FF731B6803F1040246F2676316
S214019950C6F2666383FB02134FEA63014FEAE273C2
S214019960CA1A40F6D863C1F6FF731A6016E040F6CD
S214019970F063C1F6FF731B68A3F1040246F2676346
S214019980C6F2666383FB02134FEA63014FEAE27392
S214019990CA1A40F6D863C1F6FF731A6040F6D86358
S2140199A0C1F6FF731B68184607F11407BD4680BC55
S2140199B0704700BF80B588B000AF78600B46FB707B
S2140199C04FF00003FB774FF00003FB7500F08CF9B6
S2140199D07B6803F117037B6040F69423C1F6FF739F
S2140199E01B687A68D31AA3F102033B61FB78002B4C
S2140199F00BD17A6840F2CF739A4206D93B69052BA0
S214019A0003DC3B6913F1050F02DA4FF0010301E0B5
S214019A104FF00003FB73FB7B03F00103FB73FB7B3F
S214019A2018463969FFF7F6FEB861BB69002B03DDFE
S214019A304FF00103FB7703E0BB69002B00F0968033
S214019A40FB7F002B7BD04FF00103BB775EE04FF02E
S214019A500003BB7700F09CF8B860BB68EB2B00F006
S214019A60878040F69423C1F6FF731A68BB69D21843
S214019A70BB689A4251D37A68BB689A424FD97A68D2
S214019A80BB68D21A40F2F3139A424AD8F87DFA7D9F
S214019A9040F6B823C1F6FF7333F81230194641F287
S214019AA05012C1F6FF720B464FEA43035B184FEAAA
S214019AB083034FF4965101FB00F15B18D3181A6823
S214019AC013464FEA83039B184FEA43031A4640F6B0
S214019AD09C23C1F6FF731B689A424BD840F6942329
S214019AE0C1F6FF73BA681A604FF00003BB61FB78DA
S214019AF0002B41D0FB7D4FF00000194600F0F0FB33
S214019B00034683F00103DBB2002B37D1BB7F002B6A
S214019B109DD1FB78002B9AD104E000BF02E000BF84
S214019B2000E000BF40F69423C1F6FF731A68BB69D4
S214019B30D21840F69423C1F6FF731A6021E040F66E
S214019B409423C1F6FF731B687A68D31AB3F5FA6FCC
S214019B5016D840F69423C1F6FF731A68BB69D2186B
S214019B6040F69423C1F6FF731A600AE000BF08E0CE
S214019B7000BF06E000BF04E000BF02E000BF00E057
S214019B8000BF00F0C7F807F12007BD4680BD00BF43
S214019B9080B584B000AF4FF00003FB604FF00003C8
S214019BA07B604FF00103BB724FF00003FB7260E075
S214019BB0FA7A40F6B823C1F6FF7333F81220F97A21
S214019BC040F67423C1F6FF7333F811309A424BD234
S214019BD0BB7A002B23D1F87AFA7A40F6B823C1F67D
S214019BE0FF7333F81230194641F25012C1F6FF7274
S214019BF00B464FEA43035B184FEA83034FF4965133
S214019C0001FB00F15B18D3181A6813464FEA830369
S214019C109B184FEA43031A46FB689A4225D2F87A04
S214019C20FA7A40F6B823C1F6FF7333F812301946B4
S214019C3041F25012C1F6FF720B464FEA43035B181E
S214019C404FEA83034FF4965101FB00F15B18D318DA
S214019C501A6813464FEA83039B184FEA4303FB60D7
S214019C604FF00003BB7200E000BFFB7A03F1010373
S214019C70FB7240F22353C1F6FF731B78FA7A9A42BD
S214019C8096D340F68033C1F6FF731A8840F68233C6
S214019C90C1F6FF731B889A421AD240F68033C1F68A
S214019CA0FF731B88184602F011F87860BB7A002B08
S214019CB005D07B68FB604FF00003BB7208E07A6852
S214019CC0FB689A4204D27B68FB604FF00003BB72CC
S214019CD0BB7A002B02D04FF0EB0300E0FB6818467E
S214019CE007F11007BD4680BD80B500AF03E04FF019
S214019CF0010014F09BFF40F69323C1F6FF731B7817
S214019D00002BF4D140F69323C1F6FF734FF0010206
S214019D101A7080BD80B400AF40F69323C1F6FF737E
S214019D204FF000021A70BD4680BC704780B500AF88
S214019D3003E04FF0010014F079FF40F67933C1F6E5
S214019D40FF731B78002BF4D140F67933C1F6FF730D
S214019D504FF001021A7080BD80B400AF40F679332F
S214019D60C1F6FF734FF000021A70BD4680BC704703
S214019D7080B582B000AF03463960FB71FFF7B4FFD0
S214019D80FB79002B05D040F69423C1F6FF733A68A1
S214019D901A60FB79184600F007F8FFF7BBFF07F1DA
S214019DA00807BD4680BD00BFF0B58BB006AF0346C1
S214019DB0FB7140F69423C1F6FF7319684CF6CD4348
S214019DC0CCF6CC43A3FB01234FEAD30213464FEA5A
S214019DD083039B184FEA4303CA1A002A0CD040F6A5
S214019DE09423C1F6FF731B6803F1010240F6942326
S214019DF0C1F6FF731A606FE240F69423C1F6FF7353
S214019E001A6840F69C23C1F6FF731B689A4206D86F
S214019E1040F69123C1F6FF731B78002B51D040F614
S214019E20AC63C1F6FF731B6803F1010240F6AC6335
S214019E30C1F6FF731A6040F6AC63C1F6FF731B6888
S214019E40012B12D140F69423C1F6FF731A6840F62F
S214019E50B463C1F6FF731A6001F05AFF40F67C0046
S214019E60C1F6FF7002F098F835E240F6B463C1F629
S214019E70FF731B6803F1010240F6B463C1F6FF737A
S214019E801A6040F6B463C1F6FF7319684CF6CD4309
S214019E90CCF6CC43A3FB01234FEAD30213464FEA89
S214019EA083039B184FEA4303CA1A002A40F0138221
S214019EB001F02EFF40F67C00C1F6FF7002F06CF850
S214019EC009E240F6B463C1F6FF734FF000021A6070
S214019ED040F6AC63C1F6FF734FF000021A6001F062
S214019EE017FFFB79184601F06FFF4FF00003FB7375
S214019EF0B2E1FB797B73FA7B40F67423C1F6FF73FC
S214019F0033F81230002B00F0A2814FF00103BB732F
S214019F1092E14FF00003BB7300E000BF7B7B002B98
S214019F2003D04FF000037B7335E0F87BFA7B40F6F5
S214019F30B823C1F6FF7333F81230194641F25012B6
S214019F40C1F6FF720B464FEA43035B184FEA8303E1
S214019F504FF4965101FB00F15B18D3181A681346AB
S214019F604FEA83039B184FEA43031A4640F69423AD
S214019F70C1F6FF731B689A420CD2FB7B4FF00000C0
S214019F80194600F0ADF9034683F00103DBB2002B5E
S214019F90C3D05BE100BF00F0E3F9034683F00103A1
S214019FA0DBB2002B29D040F67433C1F6FF731B7861
S214019FB083F00103DBB2002B40F0578140F6723389
S214019FC0C1F6FF731B78002B40F04F8140F69023BB
S214019FD0C1F6FF734FF000021A7040F6A863C1F68F
S214019FE0FF734FF000021A6040F64333C1F6FF7369
S214019FF01B781846FCF79CFD6EE1FA7B40F6B82309
S21401A000C1F6FF7333F81220F97B40F67423C1F6CC
S21401A010FF7333F811309A4280F01381F87BFA7B94
S21401A02040F6B823C1F6FF7333F81230194641F2F1
S21401A0305012C1F6FF720B464FEA43035B184FEA14
S21401A04083034FF4965101FB00F15B18D3181A688D
S21401A05013464FEA83039B184FEA43031A4640F61A
S21401A0609C23C1F6FF731B689A4200F2EC804FF006
S21401A07000033B73F87BFA7B40F6B823C1F6FF7307
S21401A08033F81230194641F25012C1F6FF720B46F0
S21401A0904FEA43035B184FEA83034FF4965101FBE3
S21401A0A000F15B18D3181A6813464FEA83039B180E
S21401A0B04FEA43031A4640F69423C1F6FF731B6822
S21401A0C09A4240F08180FA7B40F6C823C1F6FF73BE
S21401A0D033F8123098B2FC7BFA7B40F6B823C1F60F
S21401A0E0FF7333F81230194641F25012C1F6FF726F
S21401A0F00B464FEA43035B184FEA83034FF496512E
S21401A10001FB04F15B18D3181D79FC7BFA7B40F642
S21401A110B823C1F6FF7333F81230194641F25012D4
S21401A120C1F6FF720B464FEA43035B184FEA8303FF
S21401A1304FF4965101FB04F15B18D31803F10103A8
S21401A1401C79FE7BFA7B40F6B823C1F6FF7333F821
S21401A1501230194641F25012C1F6FF720B464FEA11
S21401A16043035B184FEA83034FF4965101FB06F154
S21401A1705B18D31803F102031B7902B24FF0FF31CB
S21401A18000914FF0000101914FF0000102914FF054
S21401A190000103914FF001010491F97B05911046EE
S21401A1A02946224603F006FBFB7B4FF000001946CA
S21401A1B000F096F8034683F00103DBB2002B44D18E
S21401A1C04FF00103BB7337E040F69423C1F6FF73EB
S21401A1D01B6803F5FA60FC7BFA7B40F6B823C1F6F0
S21401A1E0FF7333F81230194641F25012C1F6FF726E
S21401A1F00B464FEA43035B184FEA83034FF496512D
S21401A20001FB04F15B18D3181A6813464FEA83035F
S21401A2109B184FEA4303984207D240F69223C1F6B1
S21401A220FF734FF001021A7006E040F69223C1F662
S21401A230FF734FF000021A70BB7B002B7FF469AEF0
S21401A24006E000BF02E000BF00E000BF00E000BF84
S21401A250FB7B03F10103FB7340F22353C1F6FF734B
S21401A2601B78FA7B9A42FFF444AE40F6B823C1F657
S21401A270FF731B88194641F25012C1F6FF720B4656
S21401A2804FEA43035B184FEA8303D3181A684FF06B
S21401A2900303C0F200139A4210D940F67433C1F694
S21401A2A0FF731B7883F00103DBB2002B06D140F667
S21401A2B07233C1F6FF731B78002B0DD040F6942342
S21401A2C0C1F6FF731B6803F1010240F69423C1F641
S21401A2D0FF731A6000E000BF07F11407BD46F0BD2A
S21401A2E080B483B000AF02460B46FA71BB71FB79AE
S21401A2F0002B09D0BA7940F6B823C1F6FF734FF0A8
S21401A300000123F8121022E0BA7940F6B823C1F60C
S21401A310FF7333F8123003F1010399B240F6B82304
S21401A320C1F6FF7323F81210BA7940F6B823C1F6C6
S21401A330FF7333F81220B97940F67423C1F6FF7320
S21401A34033F811309A4202D34FF0000301E04FF088
S21401A3500103184607F10C07BD4680BC704700BFD5
S21401A36080B483B000AF4FF00003FB7116E0FA79BA
S21401A37040F6B823C1F6FF7333F81220F97940F698
S21401A3807423C1F6FF7333F811309A4202D24FF0AC
S21401A39001030DE0FB7903F10103FB7140F2235346
S21401A3A0C1F6FF731B78FA799A42E0D34FF00003A7
S21401A3B0184607F10C07BD4680BC704780B500AF54
S21401A3C040F64433C1F6FF731B78012B5DD940F686
S21401A3D04433C1F6FF734FF003021A7040F6383368
S21401A3E0C1F6FF731B78022B4BD101F0DBF8034655
S21401A3F0002B26D040F67133C1F6FF731B7883F02D
S21401A4000103DBB2002B1CD040F66F33C1F6FF739D
S21401A4101B78002B0ED040F67733C1F6FF731B78FE
S21401A420002B07D040F6CA63C1F6FF734FF0000257
S21401A4301A7006E040F6CA63C1F6FF734FF00102D8
S21401A4401A7040F6CA63C1F6FF731B78002B15D04D
S21401A45040F6CC63C1F6FF731B78002B02D04FF099
S21401A460E40301E04FF064034FF0860019464FF015
S21401A47000024FF00003FBF75BFB06E000F01EFB5B
S21401A48003E04FF0000000F083F880BD80B582B095
S21401A49000AF4FF00003BB7140F63833C1F6FF73CF
S21401A4A01B78022B70D040F6CB63C1F6FF731B7886
S21401A4B0002B69D140F64333C1F6FF731B781A4669
S21401A4C040F64833C1F6FF739B5C3B7040F643335E
S21401A4D0C1F6FF731B781A4640F64833C1F6FF7380
S21401A4E09B185B797B7040F64333C1F6FF731B788C
S21401A4F01A4640F64833C1F6FF739B189B7ABB7029
S21401A5004FF00003FB713CE0FB79062B04D1BB79CD
S21401A51003F10103BB7106E0FB790C2B03D1BB7978
S21401A52003F10103BB71BB7907F10801CB1813F8DE
S21401A530083C03F00403002B08D0FB7918464FF0C3
S21401A54001014FF0020204F003FB07E0FB79184615
S21401A5504FF000014FF0020204F0FAFABB79BA7923
S21401A56007F108018A1812F8082C4FEA5202D2B2F3
S21401A57007F10801CB1803F8082CFB7903F1010356
S21401A580FB71FB79112BBFD907F10807BD4680BDCA
S21401A59080B58AB000AF0346FB714FF0000387F821
S21401A5A0263007F108034FF000021A6003F1040396
S21401A5B04FF000021A6003F104034FF000021A6024
S21401A5C003F104034FF000021A6003F104034FF095
S21401A5D000021A6003F104034FF000021A6003F14F
S21401A5E004034FF000021A6003F104034FF0000267
S21401A5F01A7003F1010340F64433C1F6FF731B786A
S21401A600012B40F2D38040F22153C1F6FF731A7832
S21401A61040F22053C1F6FF731B789A4206D140F2EE
S21401A6201E53C1F6FF731B78002B1BD040F220533C
S21401A630C1F6FF731A7840F22153C1F6FF731A7000
S21401A64040F21E53C1F6FF734FF000021A7040F637
S21401A650CA63C1F6FF734FF000021A704FF005008F
S21401A660F8F7D0F84FF0000387F8273094E097F812
S21401A670272040F22C53C1F6FF7333F8122097F8C7
S21401A680271040F6C823C1F6FF7333F811309A42FB
S21401A69033D197F8272040F65833C1F6FF739A5CFA
S21401A6A097F8271040F64833C1F6FF735B5C9A4271
S21401A6B023D197F8272040F65833C1F6FF739B182D
S21401A6C05A7997F8271040F64833C1F6FF735B189E
S21401A6D05B799A4211D197F8272040F65833C1F694
S21401A6E0FF739B189A7A97F8271040F64833C1F6FD
S21401A6F0FF735B189B7A9A4248D097F8272097F801
S21401A700271040F6C823C1F6FF7333F8111040F244
S21401A7102C53C1F6FF7323F8121097F8272097F8E9
S21401A720271040F64833C1F6FF73595C40F658339C
S21401A730C1F6FF73995497F8271097F8272040F62B
S21401A7404833C1F6FF739B185A7940F65833C1F661
S21401A750FF735B185A7197F8271097F8272040F671
S21401A7604833C1F6FF739B189A7A40F65833C1F600
S21401A770FF735B189A7240F6CA63C1F6FF734FF017
S21401A78000021A704FF00600F8F73CF897F82730E9
S21401A79003F1010387F8273040F22353C1F6FF7314
S21401A7A01B7897F827209A42FFF461AF40F21E53B8
S21401A7B0C1F6FF731B78002B0AD140F6CA63C1F6B7
S21401A7C0FF731B7883F00103DBB2002B00F071816D
S21401A7D040F64633C1F6FF731B78022B03D1FB7993
S21401A7E0002B00F0668197F8263007F12800C31881
S21401A7F04FF0410203F8202C97F8263003F10103AD
S21401A80087F8263097F8261040F25053C1F6FF73AA
S21401A8101B881BB24FEA23139BB2DBB223F0030360
S21401A820DAB207F12800431803F8202C97F82630EF
S21401A83003F1010387F8263097F8261040F25053AB
S21401A840C1F6FF731B88DBB24FEA8303DAB207F166
S21401A8502800431803F8202C97F8263003F101034B
S21401A86087F8263097F8261040F6B863C1F6FF73CE
S21401A8701B7803F11403DAB207F12800431803F832
S21401A880202C97F8263003F1010387F8263097F835
S21401A890261040F22053C1F6FF731B7803F1140310
S21401A8A0DAB207F12800431803F8202C4FF0000312
S21401A8B087F827309CE097F8263003F1010387F8E4
S21401A8C0263097F8261097F8272040F6C823C1F6B9
S21401A8D0FF7333F81230DBB203F11403DAB207F177
S21401A8E02800431803F8202C40F22353C1F6FF73C7
S21401A8F01B7897F827209A4247D297F8263003F11B
S21401A900010387F8263097F8261097F8272040F697
S21401A9104833C1F6FF739B189B7A23F00303DAB220
S21401A92007F12800431803F8202C97F8263003F186
S21401A930010387F8263097F8261097F8272040F667
S21401A9404833C1F6FF739B185B7923F00303DAB231
S21401A95007F12800431803F8202C97F8263003F156
S21401A960010387F8263097F8261097F8272040F637
S21401A9704833C1F6FF739B5C23F00303DAB207F199
S21401A9802800431803F8202C2CE097F8263003F112
S21401A990010387F8263097F8263007F12802D318E6
S21401A9A04FF0000203F8202C97F8263003F101033C
S21401A9B087F8263097F8263007F12800C3184FF09D
S21401A9C0000203F8202C97F8263003F1010387F8DC
S21401A9D0263097F8263007F12802D3184FF00002E8
S21401A9E003F8202C97F8273003F1010387F8273066
S21401A9F097F82730042B7FF65EAF97F8263003F1E1
S21401AA00010387F8263097F8261040F6CC63C1F686
S21401AA10FF731B78002B02D04FF0800201E04FF04D
S21401AA20000240F22753C1F6FF731B78DBB21343D3
S21401AA30DBB2DBB203F11403DAB207F128004318E4
S21401AA4003F8202C40F22253C1F6FF731B78012B2A
S21401AA5015D197F8263003F1010387F8263097F8C9
S21401AA60261040F66A33C1F6FF731B7803F11C0308
S21401AA70DAB207F12800431803F8202C14E097F8FF
S21401AA80263003F1010387F8263097F8261040F6A2
S21401AA906A33C1F6FF731B7803F11403DAB207F1C8
S21401AAA02800431803F8202C07F108031846FBF783
S21401AAB067FA07F12807BD4680BD00BF80B584B0A0
S21401AAC000AF4FF00003FB734FF000037B734FF0B2
S21401AAD00003BB733B464FF000021A6003F1040308
S21401AAE04FF000021A6003F104034FF000021A60EF
S21401AAF003F10403FB7B07F11000C3184FF060025B
S21401AB0003F8102CFB7B03F10103FB73F97B40F286
S21401AB105053C1F6FF731B881BB24FEA23139BB237
S21401AB20DBB223F00303DAB207F11000431803F88F
S21401AB30102CFB7B03F10103FB73F97B40F25053AE
S21401AB40C1F6FF731B88DBB24FEA8303DAB207F163
S21401AB501000431803F8102C07F10D03184603F0F4
S21401AB6051FB0346BB73BB7B682B40F0948040F6D9
S21401AB707333C1F6FF731B78002B00F08C8040F610
S21401AB806F33C1F6FF731B78002B00F0848040F60C
S21401AB903833C1F6FF731B78022B7CD140F6713334
S21401ABA0C1F6FF731B7883F00103DBB2002B0ED0D6
S21401ABB0FB7B03F10103FB73FB7BBA7B42F00102D3
S21401ABC0D2B207F11001CB1803F8102C0DE0FB7B75
S21401ABD003F10103FB73FB7BBA7B62F07F02D2B207
S21401ABE007F11000C31803F8102CFB7B03F10103D7
S21401ABF0FB73F97B40F67C33C1F6FF731A8848F283
S21401AC001F53C5F2EB13A3FB02034FEA93139BB248
S21401AC10DBB203F11403DAB207F11000431803F8AC
S21401AC20102CFB7B03F10103FB73F97B40F67C33AD
S21401AC30C1F6FF731A8848F21F53C5F2EB13A3FB44
S21401AC4002034FEA93134FF0C80000FB03F3D31A35
S21401AC509BB2DBB203F11403DAB207F1100043181A
S21401AC6003F8102CFB7B03F10103FB73FB7B07F15D
S21401AC701001CB184FF00C0203F8102CFB7B03F1EC
S21401AC800103FB73FB7B07F11002D3184FF0200280
S21401AC9003F8102C9CE0FB7B03F10103FB73FB7BA9
S21401ACA007F11000C318BA7B03F8102C7B7B042B2A
S21401ACB05ED8FB7B03F10103FB73F97B7B7B1A46B2
S21401ACC040F6AC23C1F6FF7333F812304FEA131384
S21401ACD09BB2DBB223F00303DAB207F1100043188C
S21401ACE003F8102CFB7B03F10103FB73F97B7B7BE1
S21401ACF01A4640F6AC23C1F6FF7333F81230DBB2C6
S21401AD004FEA8303DAB207F11000431803F8102C58
S21401AD10FB7B03F10103FB73F97B7B7B1A4640F651
S21401AD20C823C1F6FF7333F812304FEA13139BB2F0
S21401AD30DBB223F00303DAB207F11000431803F87D
S21401AD40102CFB7B03F10103FB73F97B7B7B1A461B
S21401AD5040F6C823C1F6FF7333F81230DBB24FEA70
S21401AD608303DAB207F11000431803F8102C2FE022
S21401AD70FB7B03F10103FB73FB7B07F11001CB188F
S21401AD804FF0000203F8102CFB7B03F10103FB7369
S21401AD90FB7B07F11002D3184FF0000203F8102CCA
S21401ADA0FB7B03F10103FB73FB7B07F11000C31868
S21401ADB04FF0000203F8102CFB7B03F10103FB7339
S21401ADC0FB7B07F11001CB184FF0000203F8102CA3
S21401ADD0FB7B03F10103FB73F97B40F6B863C1F615
S21401ADE0FF731B7803F11403DAB207F1100043185E
S21401ADF003F8102CFB7B03F10103FB73F97B40F690
S21401AE004233C1F6FF731B7803F11403DAB207F17C
S21401AE101000431803F8102C3B461846FBF7C4F8FD
S21401AE2007F11007BD4680BD80B48BB000AF7860D7
S21401AE304FF00003BB77BB7F7A68D3181B784FEAC5
S21401AE4003139AB2BB7F03F101037968CB181B7811
S21401AE504FEA9303DBB213439BB27B83BB7F03F1C1
S21401AE6002037A68D3181B784FEA03139AB2BB7FA2
S21401AE7003F103037968CB181B784FEA9303DBB21F
S21401AE8013439BB23B83BB7F03F104037A68D31859
S21401AE901B784FEA03139AB2BB7F03F10503796867
S21401AEA0CB181B784FEA9303DBB213439BB2BB83E9
S21401AEB04FF00003FB7741E24FF00603BB77FA7FC2
S21401AEC040F6A023C1F6FF7333F812303B844FF0EF
S21401AED000037B61FA7F40F6C823C1F6FF7333F89F
S21401AEE012307A8B9A4240F02582FA7F40F6AC23E4
S21401AEF0C1F6FF7333F812303A8B9A4240F01A8249
S21401AF00BB7F7A68D3181B78A3F11403FB74BB7F4D
S21401AF1003F10103BB77FB7CEB2B00F07681FA7C17
S21401AF2048F63963C3F6E303A3FB02134FEA930320
S21401AF30DBB21A4647F64063C0F2050303FB02F391
S21401AF40FB60BB7F7A68D3181B784FF4FA6202FB6A
S21401AF5003F31A46FB68D318A3F51C43A3F1400379
S21401AF60FB60BB7F03F10103BB77BB7F7A68D31815
S21401AF701B781A4613464FEA83039B184FEA43038E
S21401AF801A46FB68D318A3F1C803FB60BB7F03F125
S21401AF900103BB77FA7C48F63963C3F6E303A3FBE8
S21401AFA002134FEA93010B464FEAC3035B184FEABD
S21401AFB04303D31ADBB2FA68D318FB60BB7F7A6807
S21401AFC0D3181B78A3F11403FB72BB7F03F10103B3
S21401AFD0BB77FB7A03F00703BB72FB7A4FEAD30316
S21401AFE0FB72FB7A112B18D8FA7A4DF21013C0F2C5
S21401AFF003039B5C87F82730FA7A4DF22413C0F2DC
S21401B00003039B5C87F82630FA7A4DF23813C0F2B8
S21401B01003039B5C87F8253023E0BB7F7A68D3184F
S21401B0201B784FEA930387F82730BB7F03F10103B0
S21401B030BB77BB7F7A68D3181B784FEA930387F8F0
S21401B0402630BB7F03F10103BB77BB7F7A68D31839
S21401B0501B784FEA930387F82530BB7F03F1010382
S21401B060BB77BB7A03F00103002B17D0BB7F7A684E
S21401B070D3181B78A3F1140387F82430BB7F03F1A0
S21401B0800103BB7797F82430C82B0ED940F2225320
S21401B090C1F6FF731B7887F8243006E040F222538E
S21401B0A0C1F6FF731B7887F82430BB7A03F00203DE
S21401B0B0002B14D0BB7F7A68D3181B78A3F1140336
S21401B0C087F82330BB7F03F10103BB7797F8233062
S21401B0D0C82B08D94FF0000387F8233003E04FF060
S21401B0E0000387F823303A8C40F28F139A4200F21D
S21401B0F08880F87F398C41F25012C1F6FF720B46F8
S21401B1004FEA43035B184FEA83034FF4965101FB62
S21401B11000F15B18D318FA681A60F87F398C41F28F
S21401B1205012C1F6FF720B464FEA43035B184FEA13
S21401B13083034FF4965101FB00F15B18D31897F87F
S21401B14027201A71F87F398C41F25012C1F6FF722E
S21401B1500B464FEA43035B184FEA83034FF49651BD
S21401B16001FB00F15B18D31803F1010397F82620C1
S21401B1701A71F87F398C41F25012C1F6FF720B46F4
S21401B1804FEA43035B184FEA83034FF4965101FBE2
S21401B19000F15B18D31803F1020397F825201A7102
S21401B1A0F87F398C41F25012C1F6FF720B464FEA16
S21401B1B043035B184FEA83034FF4965101FB00F1FA
S21401B1C05B18D31897F82420DA71F87F398C41F28E
S21401B1D05012C1F6FF720B464FEA43035B184FEA63
S21401B1E083034FF4965101FB00F15B18D31803F16A
S21401B1F0080397F823201A703B8C03F101033B8464
S21401B2007EE64FF00003BB8300E000BFBB8B002B44
S21401B21020D1FA7F40F68823C1F6FF734FF0010173
S21401B220995440F21E53C1F6FF734FF000021A7094
S21401B230FA7F40F6A023C1F6FF734FF0000123F812
S21401B2401210FA7F40F67423C1F6FF73398C23F887
S21401B250121007E0FA7F40F6A023C1F6FF73398C7F
S21401B26023F81210FA7F40F6AC23C1F6FF73B98BB0
S21401B27023F812105BE0F87F398C41F25012C1F6C8
S21401B280FF720B464FEA43035B184FEA83034FF402
S21401B290965101FB00F15B18D3184FF000021A60BB
S21401B2A0F87F398C41F25012C1F6FF720B464FEA15
S21401B2B043035B184FEA83034FF4965101FB00F1F9
S21401B2C05B18D3184FF000021A71F87F398C41F2DF
S21401B2D05012C1F6FF720B464FEA43035B184FEA62
S21401B2E083034FF4965101FB00F15B18D31803F169
S21401B2F001034FF000021A71F87F398C41F25012A7
S21401B300C1F6FF720B464FEA43035B184FEA83030D
S21401B3104FF4965101FB00F15B18D31803F10203B9
S21401B3204FF000021A713B8C03F101033B843B8C06
S21401B330112BA0D9FB7F03F10103FB7740F22353C6
S21401B340C1F6FF731B78FA7F9A42FFF4B5AD07F199
S21401B3502C07BD4680BC704780B584B000AF7860CE
S21401B3604FF000033B733B7B7A68D3181B784FEA98
S21401B37003139AB23B7B03F101037968CB181B7860
S21401B3804FEA9303DBB213439BB27B814FF000037A
S21401B3907B734EE04FF002033B737A7B40F6C82383
S21401B3A0C1F6FF7333F812307A899A423DD14FF0D5
S21401B3B00003BB7324E03B7B7A68D3181B78A3F1A8
S21401B3C01403FB733B7B03F101033B73FB7B0C2BE9
S21401B3D002D94FF00003FB73797BB87B40F6182245
S21401B3E0C1F6FF720B464FEAC3035B184FEA4303ED
S21401B3F01B18D318FA7B1A70BB7B03F10103BB73CE
S21401B400BB7B112BD7D97A7B40F68823C1F6FF7315
S21401B4109B5C002B09D07A7B40F68023C1F6FF7334
S21401B4204FF00101995402F0BBFE7B7B03F101034F
S21401B4307B7340F22353C1F6FF731B787A7B9A42E3
S21401B440A8D307F11007BD4680BD00BF80B584B004
S21401B45000AF0346FB804FF00003FB7389E0FA7BE5
S21401B46040F6C823C1F6FF7333F81230FA889A42C1
S21401B4707BD1FA7B40F67423C1F6FF734FF00001CF
S21401B48023F812104FF00003BB735BE0F87BB97B27
S21401B49041F25012C1F6FF720B464FEA43035B18A6
S21401B4A04FEA83034FF4965101FB00F15B18D31862
S21401B4B04FF000021A60F87BB97B41F25012C1F6D8
S21401B4C0FF720B464FEA43035B184FEA83034FF4C0
S21401B4D0965101FB00F15B18D3184FF000021A7168
S21401B4E0F87BB97B41F25012C1F6FF720B464FEA68
S21401B4F043035B184FEA83034FF4965101FB00F1B7
S21401B5005B18D31803F101034FF000021A71F87BA0
S21401B510B97B41F25012C1F6FF720B464FEA430364
S21401B5205B184FEA83034FF4965101FB00F15B1859
S21401B530D31803F102034FF000021A71BB7B03F12B
S21401B5400103BB73BB7B112BA0D9FA7B40F6882382
S21401B550C1F6FF734FF001019954FA7B40F6802340
S21401B560C1F6FF734FF001019954FB7B03F1010310
S21401B570FB7340F22353C1F6FF731B78FA7B9A42A2
S21401B580FFF46DAF02F00CFEFB88C82B06D140F627
S21401B590CA63C1F6FF734FF001021A7007F1100774
S21401B5A0BD4680BD80B483B000AF40F67333C1F6AC
S21401B5B0FF734FF001021A704FF00003FB712CE08D
S21401B5C0FA7940F68023C1F6FF739B5C002B19D0F5
S21401B5D0FA7940F68823C1F6FF739B5C002B11D0E5
S21401B5E040F67333C1F6FF731B7803F00103002B9B
S21401B5F00CBF00230123DAB240F67333C1F6FF73A2
S21401B6001A7006E040F67333C1F6FF734FF000027E
S21401B6101A70FB7903F10103FB7140F22353C1F663
S21401B620FF731B78FA799A42CAD340F67333C1F690
S21401B630FF731B78184607F10C07BD4680BC7047A0
S21401B64080B58CB000AF78604FF0000387F82F30DC
S21401B6504FF00003BB8597F82F307A68D3181B7814
S21401B6601A464FEA8202D3181A464FEA82011A4650
S21401B6700B46D3184FEAC3039AB297F82F3003F15B
S21401B68001037968CB181B78D3189BB2A3F6B47361
S21401B6903B8497F82F3003F102037A68D3181B789E
S21401B6A01A464FEA8202D3181A464FEA82011A4610
S21401B6B00B46D3184FEAC3039AB297F82F3003F11B
S21401B6C003037968CB181B78D3189BB2A3F6B4731F
S21401B6D07B8540F67E33C1F6FF731B88BB85BB8D29
S21401B6E0002B19D107F1100207F10E031046194677
S21401B6F001F0A2FE034683F00103DBB2002B0BD060
S21401B70040F22553C1F6FF731B7883F00103DBB2C9
S21401B710002B01D03B8ABB85BB8D03F5B8434FEAAE
S21401B720C3037B624FF0040387F82F3040F67C3367
S21401B730C1F6FF731B883A8C9A4240F0CC8197F889
S21401B7402F307A68D3181B78A3F11403FB7797F888
S21401B7502F3003F1010387F82F30FB7FEB2B00F02E
S21401B7600E81FA7F48F63963C3F6E303A3FB02139F
S21401B7704FEA9303DBB21A4647F64063C0F205036D
S21401B78003FB02F37B6197F82F307A68D3181B7896
S21401B7904FF4FA6202FB03F31A467B69D318A3F54A
S21401B7A01C43A3F140037B6197F82F3003F101039B
S21401B7B087F82F3097F82F307A68D3181B781A46F7
S21401B7C013464FEA83039B184FEA43031A467B69E5
S21401B7D0D318A3F1C8037B6197F82F3003F1010357
S21401B7E087F82F30FA7F48F63963C3F6E303A3FBE5
S21401B7F002134FEA93010B464FEAC3035B184FEA65
S21401B8004303D31ADBB21A467B69D3187B617A6984
S21401B81013464FEA83039B184FEA43037B6197F86D
S21401B8202F307A68D3181B784FEA03139AB297F829
S21401B8302F3003F101037968CB181B784FEA930385
S21401B840DBB213439BB2BB8397F82F3003F102039D
S21401B8507A68D3181B784FEA03139AB297F82F30F9
S21401B86003F103037968CB181B784FEA9303DBB225
S21401B87013439BB27B8397F82F3003F102037A6858
S21401B880D3181B7803F0F0034FEA03239AB297F814
S21401B8902F3003F104037968CB181B784FEA0313A2
S21401B8A09BB213439AB297F82F3003F105037968D8
S21401B8B0CB181B784FEA9303DBB213439BB29BB2C0
S21401B8C07B8297F82F3003F1060387F82F30BA8D65
S21401B8D040F6B7339A424ED8BB8D002B01D1F8F70C
S21401B8E043F9F7F7D1FB41F2F803C1F6FF731A6883
S21401B8F007F114031046796A4FF00402F8F7DCFFEB
S21401B900BB8B7B7641F2F803C1F6FF7319687B6A3D
S21401B91003F104027B7E084611461A46F8F7BCFD81
S21401B9207B8B7B7641F2F803C1F6FF7319687B6A5D
S21401B93003F105027B7E084611461A46F8F7ACFD70
S21401B94041F2F803C1F6FF7319687B6A03F1060238
S21401B95007F11203084611464FF00202F8F7ACFF52
S21401B9607B6A03F108037B62F7F7AAFBBB8D03F141
S21401B9700103BB85E3E64FF000037B8500E000BFD3
S21401B9807B8D002B40F08C804FF0000387F823302E
S21401B9900EE097F8232040F68023C1F6FF734FF0A0
S21401B9A00101995497F8233003F1010387F82330F6
S21401B9B040F22353C1F6FF731B7897F823209A426F
S21401B9C0E7D340F67133C1F6FF734FF001021A70E8
S21401B9D040F21E53C1F6FF734FF000021A7040F694
S21401B9E07E33C1F6FF734FF000021A8040F68233B1
S21401B9F0C1F6FF73BA8D1A80BB8D002B03D0BB8DA9
S21401BA001846FBF79FFA40F67533C1F6FF734FF001
S21401BA1000021A7040F68233C1F6FF731B88002BB2
S21401BA2020D040F67533C1F6FF731B7883F001030F
S21401BA30DBB2002B16D0F8F753F801F065F900F0E9
S21401BA402BFFFBF725FA40F67533C1F6FF734FF06F
S21401BA5001021A7040F6CA63C1F6FF734FF0010285
S21401BA601A702CE040F68233C1F6FF731B88002B58
S21401BA7024D140F6B063C1F6FF734FF000021A807E
S21401BA8040F6B063C1F6FF731B881846F7F750FF00
S21401BA9040F6CA63C1F6FF734FF001021A700DE05B
S21401BAA040F67E33C1F6FF73BA8D1A80BB8D002B2C
S21401BAB005D0BB8D1846FBF745FA00E000BF40F6FF
S21401BAC07C33C1F6FF737A8D1A80BA8D7B8D104652
S21401BAD01946F7F76DFF07F13007BD4680BD00BF79
S21401BAE080B588B000AFF860B9607A607B68FB61AA
S21401BAF040F68033C1F6FF731B88002B2ED140F62B
S21401BB007433C1F6FF734FF000021A7040F67233B9
S21401BB10C1F6FF734FF000021A7040F6A863C1F633
S21401BB20FF734FF000021A604FF000037B8312E0B0
S21401BB307B8BFA68D3184FF000021A707A8B40F6A6
S21401BB408433C1F6FF734FF0000143F822107B8B5C
S21401BB5003F101037B837B8BC82BE9D9FEF7E6F85B
S21401BB60F7F792FA41F2F803C1F6FF731A68FB6918
S21401BB7003F1040310461946F8F7D6FC03467B7614
S21401BB8041F2F803C1F6FF731A68FB6903F1050376
S21401BB9010461946F8F7C8FC03463B7641F2F8030F
S21401BBA0C1F6FF731968FB6903F1060207F1160374
S21401BBB0084611464FF00202F8F72EFFF7F780FA13
S21401BBC07B7EFA68D3183A7E1A70FB8A002B34D033
S21401BBD0797EFB8A1A4613464FEA83039B184FEA7F
S21401BBE043031A4640F68433C1F6FF7343F8212017
S21401BBF040F67233C1F6FF734FF001021A707A7E77
S21401BC0040F68433C1F6FF7353F82220BB68D2187E
S21401BC1040F6A863C1F6FF731B689A420DD97A7E77
S21401BC2040F68433C1F6FF7353F82220BB68D2185E
S21401BC3040F6A863C1F6FF731A6040F68033C1F67A
S21401BC40FF731B8803F101039AB240F68033C1F6F5
S21401BC50FF731A8040F68033C1F6FF731A8840F6E8
S21401BC608233C1F6FF731B889A420ED340F68033A7
S21401BC70C1F6FF734FF000021A8040F67433C1F626
S21401BC80FF734FF001021A7019E0FB6903F1080314
S21401BC90FB61F7F7F9F941F2F803C1F6FF731A6889
S21401BCA007F110031046F9694FF00402F8F7B4FEE5
S21401BCB0F7F706FA3A69BB689A423FF451AFFEF7C6
S21401BCC04BF807F12007BD4680BD00BF80B584B0A4
S21401BCD000AF0346FB80FB8803F5B8434FEAC30376
S21401BCE0FB60F7F7D1F941F2F803C1F6FF731A6862
S21401BCF007F108031046F9684FF00402F8F78CFEC6
S21401BD00F7F7DEF9BB68184607F11007BD4680BD98
S21401BD1080B582B000AF40F67233C1F6FF731B7870
S21401BD2083F00103DBB2002B48D1FDF7FFFF40F69D
S21401BD307233C1F6FF734FF000021A704FF0010321
S21401BD40FB8035E0FA8840F68433C1F6FF7353F87A
S21401BD502230002B28D0FA88F98840F68433C1F6C1
S21401BD60FF7353F82130A3F10A0140F68433C1F67C
S21401BD70FF7343F82210FA8840F68433C1F6FF7346
S21401BD8053F82230002B08D1FA8840F67C03C1F61E
S21401BD90FF734FF00001995406E040F67233C1F686
S21401BDA0FF734FF001021A70FB8803F10103FB8059
S21401BDB0FB88C82BC6D9FDF7CFFF00E000BF07F10F
S21401BDC00807BD4680BD00BF80B586B000AF0346FC
S21401BDD0FB71FB79FB754FF00003FB6040F6823385
S21401BDE0C1F6FF731B88002B7BD040F68033C1F66B
S21401BDF0FF731B8803F5B8434FEAC3033B61F7F7AC
S21401BE0043F941F2F803C1F6FF731A6807F10C0310
S21401BE10104639694FF00402F8F7FEFDF7F750F9BE
S21401BE2040F69423C1F6FF731A68FB689A4213D151
S21401BE3040F69423C1F6FF731B6840F67C00C1F6FA
S21401BE40FF7019463A69FFF74BFE40F67C00C1F6D3
S21401BE50FF7000F0A1F844E0FA6840F6A863C1F666
S21401BE60FF731B68D21840F69423C1F6FF731B6854
S21401BE709A4222D340F67C00C1F6FF7000F08CF89F
S21401BE8040F69423C1F6FF731A68FB689A4228D9D4
S21401BE9040F67433C1F6FF731B7883F00103DBB2FF
S21401BEA0002B1ED040F69423C1F6FF731A68FB6878
S21401BEB01046194600F01AF813E040F67433C1F63E
S21401BEC0FF731B7883F00103DBB2002B09D040F629
S21401BED09423C1F6FF731A68FB681046194600F0F2
S21401BEE005F807F11807BD4680BD00BF80B584B0D0
S21401BEF000AF7860396040F68033C1F6FF731B8867
S21401BF0003F101039AB240F68033C1F6FF731A803B
S21401BF1040F68033C1F6FF731B881846FFF7D6FE3E
S21401BF20F86040F68033C1F6FF731A8840F6823314
S21401BF30C1F6FF731B889A4211D340F68033C1F6CF
S21401BF40FF734FF000021A804FF00003FB6040F6CB
S21401BF507433C1F6FF734FF001021A7003E07A687A
S21401BF60FB689A42C7D840F6B063C1F6FF731B88D8
S21401BF70002B0DD040F67433C1F6FF731B7883F0A7
S21401BF800103DBB2002B03D07868396800F0AAF809
S21401BF9007F11007BD4680BD80B584B000AF78605C
S21401BFA040F6D663C1F6FF731B78002B42D140F2F0
S21401BFB02653C1F6FF731B7883F00103DBB2002B17
S21401BFC038D140F22653C1F6FF731B78002B32D0CE
S21401BFD040F67A33C1F6FF731B78002B16D040F675
S21401BFE07803C1F6FF731B68184640F618514FF0E8
S21401BFF000020FF0BBFF0346FB6040F64810C1F697
S21401C000FF704FF0C901FAF713F914E040F6780310
S21401C010C1F6FF731B68184640F618514FF0000230
S21401C0200FF0A4FF0346FB6078684FF0C901FAF7EA
S21401C030FFF800E000BF07F11007BD4680BD00BF56
S21401C04080B400AF40F67033C1F6FF734FF00002C4
S21401C0501A7040F67133C1F6FF734FF000021A7082
S21401C06040F67E33C1F6FF734FF000021A8040F6A9
S21401C0707C33C1F6FF734FF000021A8040F682331C
S21401C080C1F6FF734FF000021A8040F6B063C1F6A6
S21401C090FF734FF000021A8040F68033C1F6FF733B
S21401C0A04FF000021A8040F6A863C1F6FF734FF006
S21401C0B000021A6040F67233C1F6FF734FF00002B9
S21401C0C01A7040F67533C1F6FF734FF000021A700E
S21401C0D040F6CA63C1F6FF734FF000021A70BD4600
S21401C0E080BC704780B5ADF5247D00AF07F1040331
S21401C0F018603B4619604FF00003C7F88C3207F111
S21401C10004031B68C7F884324FF00003A7F8823295
S21401C1104FF00003C7F87C324FF00003C7F86832CF
S21401C1204FF0000387F8793207F1D4031A464FF42B
S21401C130C97310464FF000011A461BF02DF807F19F
S21401C14008031A464FF0C90310464FF000011A467D
S21401C1501BF022F807F10403186800F0FBFD034604
S21401C160A7F87632B7F97632002BC0F23081B7F9EC
S21401C170762247F2C013C1F6FF7353F8222007F167
S21401C18004031B689A4277D1B7F9763240F25B22F4
S21401C19002FB03F303F58053C7F87032F6F774FF1A
S21401C1A041F2F803C1F6FF731A6807F10803104657
S21401C1B0D7F870124FF0C902F8F72EFC0346A7F81D
S21401C1C06E3241F2F803C1F6FF731968D7F8703280
S21401C1D003F1C90207F1D403084611464FF4C972A8
S21401C1E0F8F71AFC0346A7F86E32F6F769FFFDF773
S21401C1F09DFD4FF00103A7F87A322FE0B7F87A22B7
S21401C20007F1D40333F81230002B15D0B7F87A12A1
S21401C210B7F87A2207F1D40333F812301A461346D8
S21401C2204FEA83039B184FEA43031A4640F68433CA
S21401C230C1F6FF7343F82120B7F87A22B7F87A32AD
S21401C24007F10801C95C40F67C03C1F6FF739954F7
S21401C250B7F87A3203F10103A7F87A32B7F87A32DF
S21401C260C82BCBD940F67233C1F6FF734FF00102EB
S21401C2701A70FDF771FDD3E1B7F9762247F2C013C4
S21401C280C1F6FF7353F822203B461B689A4240F2E0
S21401C29084804FF0010387F87932B7F9762247F2A6
S21401C2A0C013C1F6FF7353F82230C7F8883207F17E
S21401C2B004031B68C7F88432B7F9763240F25B2272
S21401C2C002FB03F303F58053C7F87032F6F7DCFE82
S21401C2D041F2F803C1F6FF731A6807F10803104626
S21401C2E0D7F870124FF0C902F8F796FB0346A7F885
S21401C2F06E3241F2F803C1F6FF731968D7F870324F
S21401C30003F1C90207F1D403084611464FF4C97276
S21401C310F8F782FB0346A7F86E32F6F7D1FEFDF773
S21401C32005FD4FF00103A7F87A322FE0B7F87A221D
S21401C33007F1D40333F81230002B15D0B7F87A1270
S21401C340B7F87A2207F1D40333F812301A461346A7
S21401C3504FEA83039B184FEA43031A4640F6843399
S21401C360C1F6FF7343F82120B7F87A22B7F87A327C
S21401C37007F10801C95C40F67C03C1F6FF739954C6
S21401C380B7F87A3203F10103A7F87A32B7F87A32AE
S21401C390C82BCBD9FDF7E0FC24E0B7F9762247F2AB
S21401C3A0C013C1F6FF7353F822203B461B689A421E
S21401C3B018D84FF0010387F879323B461B68C7F857
S21401C3C0883207F104031B68C7F884320AE04FF08D
S21401C3D00000FFF77BFCC7F8880207F104031B681F
S21401C3E0C7F88432B7F882321846FFF76FFC024668
S21401C3F0D7F888329A420FD2B7F8823203F1010396
S21401C400A7F88232B7F882321846FFF75FFC024679
S21401C410D7F888329A42EFD3FDF788FCD7F88832EE
S21401C420C7F88C32ECE097F87932002B46D04FF003
S21401C430000387F879324FF00103A7F87A3239E022
S21401C440B7F87A2240F68433C1F6FF7353F82230E8
S21401C450002B29D0B7F87A22B7F87A1240F684333F
S21401C460C1F6FF7353F82130A3F10A0140F6843375
S21401C470C1F6FF7343F82210B7F87A2240F68433E8
S21401C480C1F6FF7353F82230002B09D1B7F87A2290
S21401C49040F67C03C1F6FF734FF00001995403E0A8
S21401C4A04FF0010387F87932B7F87A3203F10103C6
S21401C4B0A7F87A32B7F87A32C82BC1D9B7F88232E0
S21401C4C01846FFF703FC0246D7F88C329A4240F032
S21401C4D09180F6F7D9FDB7F8823203F5B8434FEAF3
S21401C4E0C303C7F8703241F2F803C1F6FF731A6846
S21401C4F0D7F8703203F1040310461946F8F714F81A
S21401C500034687F86D3241F2F803C1F6FF731A68E5
S21401C510D7F8703203F1050310461946F8F704F808
S21401C520034687F86C3241F2F803C1F6FF731968C7
S21401C530D7F8703203F1060207F51A73084611465A
S21401C5404FF00202F8F768FAF6F7BAFD97F86D228F
S21401C55040F67C03C1F6FF7397F86C129954D7F82E
S21401C5606832002B27D0D7F8682213464FEA830398
S21401C5709B184FEA4303C7F8683297F86D22D7F83D
S21401C580681240F68433C1F6FF7343F822104FF069
S21401C590010387F87932D7F86822D7F88C32D21897
S21401C5A0D7F87C329A4206D9D7F86832D7F88C2267
S21401C5B0D318C7F87C32B7F8823203F10103A7F823
S21401C5C0823240F68233C1F6FF731B88B7F88222A7
S21401C5D09A4204D34FF00003A7F882320AE0B7F874
S21401C5E082321846FFF772FB0246D7F88C329A421F
S21401C5F03FF46FAFD7F88C3203F10A03C7F88C32D9
S21401C600D7F88C22D7F884329A427FF60CAF40F6E0
S21401C6107233C1F6FF7397F879221A70FDF79CFB07
S21401C62007F52477BD4680BD80B582B000AF40F6E1
S21401C6303B33C1F6FF731B78282B0CD840F63B33EF
S21401C640C1F6FF731B7803F10103DAB240F63B3300
S21401C650C1F6FF731A7040F63B33C1F6FF731B78C1
S21401C660282B40F2968040F6FC63C1F6FF73DB7818
S21401C670002B39D040F6FC63C1F6FF731B7983F0BB
S21401C6800103DBB2002B2FD040F6B863C1F6FF736F
S21401C6901A784CF6CD43CCF6CC43A3FB02134FEAF3
S21401C6A09303DBB203F10103DBB21A464FEA8202BF
S21401C6B0D318DAB240F6B863C1F6FF731A7040F6C3
S21401C6C0B863C1F6FF731B78622B3AD940F6B8639C
S21401C6D0C1F6FF731B78A3F16303DAB240F6B863C1
S21401C6E0C1F6FF731A702CE040F6B863C1F6FF730B
S21401C6F01A784CF6CD43CCF6CC43A3FB02134FEA93
S21401C7009303DBB21A464FEA8202D3189BB2A3F117
S21401C71005039BB2FB80B7F90630002B0ADAFB88CB
S21401C720DBB203F16303DAB240F6B863C1F6FF7316
S21401C7301A7006E0FB88DAB240F6B863C1F6FF73FA
S21401C7401A7040F6B863C1F6FF731B78002B07D04A
S21401C75040F66F33C1F6FF734FF001021A7008E01E
S21401C76040F66F33C1F6FF734FF000021A70FFF701
S21401C77067FC40F66F33C1F6FF731B781846FAF76D
S21401C78017FA40F67833C1F6FF734FF001021A70BC
S21401C7907DE040F63B33C1F6FF731B780A2B06D0CB
S21401C7A040F63B33C1F6FF731B78142B6FD940F666
S21401C7B0FC63C1F6FF73DB78002B25D040F6FC63E3
S21401C7C0C1F6FF731B7983F00103DBB2002B1BD08C
S21401C7D040F6B863C1F6FF731B7803F10103DAB2C2
S21401C7E040F6B863C1F6FF731A7040F6B863C1F637
S21401C7F0FF731B78632B23D940F6B863C1F6FF732A
S21401C8004FF000021A701BE040F6B863C1F6FF73E2
S21401C8101B78002B0DD040F6B863C1F6FF731B786A
S21401C82003F1FF33DAB240F6B863C1F6FF731A704C
S21401C83006E040F6B863C1F6FF734FF063021A7064
S21401C84040F6B863C1F6FF731B78002B07D040F69D
S21401C8506F33C1F6FF734FF001021A7008E040F61D
S21401C8606F33C1F6FF734FF000021A70FFF7E8FB53
S21401C87040F66F33C1F6FF731B781846FAF798F93E
S21401C88040F67833C1F6FF734FF001021A7007F1D4
S21401C8900807BD4680BD00BF80B586B000AF4FF02B
S21401C8A000037B8240F68233C1F6FF731B88012B9F
S21401C8B021D840F6B063C1F6FF734FF000021A802C
S21401C8C040F6B063C1F6FF731B884DF2D020C0F26C
S21401C8D0030019460FF028FB4DF2F420C0F20300C6
S21401C8E00FF022FB40F6B063C1F6FF731B881846B3
S21401C8F0F7F71EF8FEE040F68233C1F6FF731B8899
S21401C900B3F5967F03D84FF00103FB7512E040F6AE
S21401C9108233C1F6FF731B8807EE903AB8EE677A4A
S21401C920DFED767AC7EE277AB0EE670A00F04EFAA8
S21401C9300346FB754FF00003FB80FB7D9BB203F1C2
S21401C940FF33BB82BB8A002B02D14FF00103BB82AF
S21401C95040F68233C1F6FF731A88FB7D9BB2D31A69
S21401C9609BB23B82FB881846FFF7B0F9F860BB8A9A
S21401C9701846FFF7ABF9B86008E0BB8A03F101037C
S21401C980BB82BB8A1846FFF7A1F9B860BA68FB6894
S21401C9909A42F2D0BB68B3F1FF3F15D140F6B063BF
S21401C9A0C1F6FF734FF000021A804DF22C30C0F230
S21401C9B003000FF0B9FA40F6B063C1F6FF731B88A7
S21401C9C01846F6F7B5FF95E07B8AF868B9681A4607
S21401C9D000F096F8BB68FB607B8A1846F7F708F903
S21401C9E06BE0BB8A03F10103FB80FB7D9AB2BB8A35
S21401C9F0D318BB82BA8A40F68233C1F6FF731B880E
S21401CA0003F1FF339A4209DDFA8840F68233C1F614
S21401CA10FF731B8803F1FF339A4257DCBA8A40F64C
S21401CA208233C1F6FF731B8803F1FF339A4214DD8C
S21401CA30FA8840F68233C1F6FF731B8803F1FF3391
S21401CA409A420ADC40F68233C1F6FF731B8803F173
S21401CA50FF33BB824FF000033B82B7F91020FB7D0A
S21401CA609A4205DB3A8AFB7D9BB2D31A9BB23B8284
S21401CA707A8A40F22B139A420ED1B7F91030002B66
S21401CA800ADD40F68233C1F6FF731B8803F1FF33DC
S21401CA90BB824FF000033B82BB8A1846FFF716F9AC
S21401CAA0B8607B8AF868B9681A4600F029F8BB684E
S21401CAB0FB607B8A1846F7F79BF87B8A03F1010334
S21401CAC07B827A8A40F22B139A428AD940F6B06367
S21401CAD0C1F6FF737A8A1A8040F6B063C1F6FF7317
S21401CAE01B881846F6F724FF47F2C010C1F6FF7000
S21401CAF0F6F7B4FF07F11807BD4680BD0000964360
S21401CB0080B58EB000AFF860B9601346FB804FF079
S21401CB1000037B63FB683B62BB68FB614FF000036D
S21401CB207B864FF00003BB824FF00003FB624FF0A1
S21401CB30000387F825307B8E1846FFF7C7F8B862E2
S21401CB403A6ABB6A9A420CD97B8E03F101037B8653
S21401CB507B8E1846FFF7BAF8B8623A6ABB6A9A4201
S21401CB60F2D83B6A7B63BEE097F82530002B3FD0B6
S21401CB704FF0000387F825304FF00103FB8434E0C3
S21401CB80FA8C46F65073C1F6FF7333F81230002B59
S21401CB9027D0FA8C46F65073C1F6FF7333F812307D
S21401CBA003F1FF3399B246F65073C1F6FF7323F8CB
S21401CBB01210FA8C46F65073C1F6FF7333F8123032
S21401CBC0002B0AD1FA8C46F65073C1F6FF739B18F8
S21401CBD04FF0000283F8922103E04FF0010387F83B
S21401CBE02530FB8C03F10103FB84FB8CC82BC7D9D2
S21401CBF07A6BBB6A9A4272D1F6F746FA7B8E03F5D8
S21401CC00B8434FEAC303BB6141F2F803C1F6FF73B1
S21401CC101A68BB6903F1040310461946F7F784FC4A
S21401CC200346FB7541F2F803C1F6FF731A68BB6948
S21401CC3003F1050310461946F7F776FC0346BB7564
S21401CC4041F2F803C1F6FF731968BB6903F10602E6
S21401CC5007F11403084611464FF00202F7F7DCFE0F
S21401CC60F6F72EFAFA7D46F65073C1F6FF739B1857
S21401CC70BA7D83F89221BB8A002B17D0FA7DB98A38
S21401CC8046F65073C1F6FF7323F812104FF00103F6
S21401CC9087F82530BB8A1A467B6BD218FB6A9A4204
S21401CCA004D9BB8A1A467B6BD318FB627B8E03F1D1
S21401CCB001037B8640F68233C1F6FF731B887A8EAA
S21401CCC09A4203D34FF000037B8608E07B8E18461A
S21401CCD0FEF7FCFFB8627A6BBB6A9A428CD07B6B1C
S21401CCE003F10A037B637A6BFB699A427FF63CAFDA
S21401CCF0FA8847F2C013C1F6FF73F96943F82210A8
S21401CD0007F13807BD4680BD80B483B000AF4FF051
S21401CD100003FB8016E0FA8846F65073C1F6FF73EF
S21401CD209B184FF0000283F89221FA8846F650735A
S21401CD30C1F6FF734FF0000123F81210FB8803F1D0
S21401CD400103FB80FB88C82BE5D907F10C07BD461C
S21401CD5080BC704780B485B000AF78604FF00003A8
S21401CD60FB8147F2C013C1F6FF731A687B689A42CB
S21401CD7010D94FF6FF7321E0FB8903F10103FB8114
S21401CD80B7F90E2040F6B063C1F6FF731B889A42CE
S21401CD900DDA00E000BFB7F90E2047F2C013C1F666
S21401CDA0FF7353F822207B689A42E5D900E000BF62
S21401CDB0FB8903F1FF339BB2FB81FB891BB218464B
S21401CDC007F11407BD4680BC704700BF80B582B02E
S21401CDD000AF87ED010AD7ED017AF5EEC07AF1EEE4
S21401CDE010FA16D578681BF0B7FD02460B461046BA
S21401CDF019464FF000024FF00003C3F6E0731BF034
S21401CE004BFC02460B46104619461CF093F80346A7
S21401CE1015E078681BF0A0FD02460B461046194641
S21401CE204FF000024FF00003C3F6E0731BF036FC30
S21401CE3002460B46104619461CF07CF80346184677
S21401CE4007F10807BD4680BD80B582B000AF034636
S21401CE50FB71FB794FF0500019464FF000024FF07E
S21401CE600003F8F765FE07F10807BD4680BD00BF61
S21401CE7080B592B000AF786040F67633C1F6FF73A6
S21401CE804FF001021A704FF0000387F8463097F80A
S21401CE9046307A68D3181B781A464FEA4202D218EF
S21401CEA04FEAC202D31A1A464FEA82011A460B46C5
S21401CEB0D3184FEA43039AB297F8463003F10103B9
S21401CEC07968CB181B78D3189BB2A3F59053A3F1BE
S21401CED00C039BB2FB8597F8463003F102037A6890
S21401CEE0D3181B781A464FEA4202D2184FEAC202FA
S21401CEF0D31A1A464FEA82011A460B46D3184FEA4E
S21401CF0043039AB297F8463003F103037968CB18C6
S21401CF101B78D3189BB2A3F59053A3F10C039BB2D5
S21401CF207B8697F8463003F104037A68D3181B789A
S21401CF301A464FEA4202D2184FEAC202D31A1A46DA
S21401CF404FEA82011A460B46D3184FEA43039AB2B8
S21401CF5097F8463003F105037968CB181B78D31888
S21401CF609BB2A3F59053A3F10C039BB23B8697F8B3
S21401CF70463003F106037A68D3181B781A464FEA3F
S21401CF804202D2184FEAC202D31A1A464FEA820167
S21401CF901A460B46D3184FEA43039AB297F846301F
S21401CFA003F107037968CB181B78D3189BB2A3F556
S21401CFB09053A3F10C03A7F8443097F8463003F1D9
S21401CFC008037A68D3181B781A464FEA4202D21829
S21401CFD04FEAC202D31A1A464FEA82011A460B4694
S21401CFE0D3184FEA43039AB297F8463003F1090380
S21401CFF07968CB181B78D3189BB2A3F59053A3F18D
S21401D0000C03A7F84230B7F844304FEA0342B7F8AA
S21401D01042301343BB63BB6B002B0BD1FB8D002B44
S21401D02008D17B8E002B05D13B8E002B02D100F060
S21401D03071F96BE197F8463003F10A0387F8463039
S21401D0404FF0000387F8473000E000BF97F84630FE
S21401D0507A68D3181B78A3F1140387F8413097F840
S21401D060463003F1010387F8463097F84130002B2C
S21401D0700FD197F8473007F14802D31897F84120A7
S21401D08003F8402C97F8473003F1010387F847303F
S21401D09017E097F8473007F14802D31897F8412070
S21401D0A003F8402C97F8473003F1010387F847301F
S21401D0B097F84730202BC8D94FF0000387F828305F
S21401D0C000BF4FF48053C0F23F03FB63F5F7DCFF6C
S21401D0D041F2F803C1F6FF731968FB6B03F1060210
S21401D0E007F13403084611464FF00402F7F794FCA3
S21401D0F0F5F7E6FF7A6BBB6B9A427BD040F6773347
S21401D100C1F6FF734FF001021A7040F22553C1F6C3
S21401D110FF734FF001021A70FEF792FF4FF0000006
S21401D1204FF00001F6F744FCF5F7AEFF41F2F803C5
S21401D130C1F6FF731B6818464FF48051C0F23F01D9
S21401D140F7F726F80346002B4BD041F2F803C1F659
S21401D150FF731A6807F12E031046F96B4FF00202AF
S21401D160F7F7AAFB41F2F803C1F6FF731968FB6BE8
S21401D17003F1020207F13203084611464FF002029C
S21401D180F7F79AFB41F2F803C1F6FF731968FB6BD8
S21401D19003F1040207F13003084611464FF002027C
S21401D1A0F7F78AFB41F2F803C1F6FF731968FB6BC8
S21401D1B003F1060207F13803084611464FF0040250
S21401D1C0F7F77AFB41F2F803C1F6FF731868FB6BB9
S21401D1D003F10A0197F8472007F10803F7F76CFBFC
S21401D1E005E04DF28030C0F203000EF09DFEF5F72B
S21401D1F067FF8BE040F67733C1F6FF734FF000020E
S21401D2001A7007F12C0207F12A031046194600F09E
S21401D21013F9034683F00103DBB2002B14D040F26E
S21401D2202553C1F6FF734FF000021A7040F67733AC
S21401D230C1F6FF734FF001021A707A8D40F67C3307
S21401D240C1F6FF731A8061E0F5F71EFF41F2F8039D
S21401D250C1F6FF731B6818464FF48051C0F23F01B8
S21401D2604FF0020240F68233C1F6FF73F7F7D4FBA4
S21401D27041F2F803C1F6FF731B6818464FF47C11A0
S21401D2804FF0020240F6B063C1F6FF73F7F7C4FB36
S21401D29040F6B063C1F6FF731B88002B11D041F234
S21401D2A0F803C1F6FF731B6818464FF47041C0F2CD
S21401D2B03E014FF4966247F2C013C1F6FF73F7F7CB
S21401D2C0ABFBF5F7FDFE40F68233C1F6FF731B8814
S21401D2D0002B1BD040F68233C1F6FF731B8818461D
S21401D2E0F9F730FE4FF4FA6011F0A0FCF9F7D0FD23
S21401D2F040F21E53C1F6FF731B78002B06D040F296
S21401D3001E53C1F6FF734FF000021A7007F148076B
S21401D310BD4680BD80B582B000AF4FF00003FB80F4
S21401D3204FF000033B60F5F7AFFE41F2F803C1F69C
S21401D330FF731B6818464FF48051C0F23F01F6F7A1
S21401D34027FF0346002B1FD041F2F803C1F6FF73F7
S21401D3501A6807F1060310464FF48051C0F23F01E8
S21401D3604FF00202F7F7A8FA41F2F803C1F6FF738D
S21401D3701A683B46104641F20601C0F23F014FF0E3
S21401D3800402F7F799FA05E04DF28030C0F2030087
S21401D3900EF0CAFDF5F794FE07F10807BD4680BDFD
S21401D3A080B483B000AF02460B46FA80BB80FB8890
S21401D3B003F01F039AB241F22413C1F6FF731A80D9
S21401D3C0FB8803F4F0734FEA63139AB241F2241315
S21401D3D0C1F6FF735A80FB884FEA53239BB203F5CD
S21401D3E0FA639AB241F22413C1F6FF739A80BB889E
S21401D3F04FEAD3239AB241F22413C1F6FF73DA80BF
S21401D400BB8803F4FC634FEA63139AB241F2241318
S21401D410C1F6FF731A81BB8803F01F039BB24FEA64
S21401D42043039AB241F22413C1F6FF735A8107F1FE
S21401D4300C07BD4680BC704780B584B000AF7860ED
S21401D4403960F5F721FE41F2F803C1F6FF731A6859
S21401D45007F10E0310464FF48051C0F23F014FF022
S21401D4600202F7F7D9FA41F2F803C1F6FF731A6818
S21401D47007F10C0310464FF46041C0F23E014FF035
S21401D4800202F7F7C9FA41F2F803C1F6FF731A6808
S21401D49007F10A0310464EF20201C0F23E014FF0B8
S21401D4A00202F7F7B9FAF5F70BFEBA897B681A801C
S21401D4B07A893B681A80BA89FB899A4202D24FF070
S21401D4C0000301E04FF00103184607F11007BD46BF
S21401D4D080BD00BF80B483B000AF13460246FA8019
S21401D4E00A467A713B7140F66D33C1F6FF734FF011
S21401D4F000021A70B7F90630002B40F39A8040F606
S21401D500CD63C1F6FF731B7883F00103DBB2002BFA
S21401D51040F09E8040F64333C1F6FF731B781A46EF
S21401D52040F24453C1F6FF734FF0010123F8121085
S21401D53040F64333C1F6FF731B781A4640F2385360
S21401D540C1F6FF73F98823F8121040F64333C1F68B
S21401D550FF731B781A4640F63033C1F6FF737979AC
S21401D560995440F64333C1F6FF731B781A4640F2CE
S21401D5701453C1F6FF733979995440F64333C1F613
S21401D580FF731B781A4640F21453C1F6FF739A5C78
S21401D59040F64333C1F6FF731B78194640F6303325
S21401D5A0C1F6FF735B5C9A421AD340F64333C1F669
S21401D5B0FF731B781A4640F64333C1F6FF731B7898
S21401D5C0194640F63033C1F6FF735B5C03F1FF3357
S21401D5D0DBB2D9B240F6C063C1F6FF73995419E0C5
S21401D5E040F64333C1F6FF731B781A4640F64333C1
S21401D5F0C1F6FF731B78194640F63033C1F6FF7348
S21401D6005B5C03F10103DBB2D9B240F6C063C1F63D
S21401D610FF73995440F6CE63C1F6FF734FF00102D3
S21401D6201A7040F66C33C1F6FF734FF000021A70A1
S21401D6300FE040F64333C1F6FF731B781A4640F2FB
S21401D6404453C1F6FF734FF6FF7123F8121000E042
S21401D65000BF07F10C07BD4680BC704780B582B09D
S21401D66000AF02460B46FA71BB71FB7918464FF0C4
S21401D6700101FBF7ABFABB7983F00103DBB2002BA8
S21401D68006D040F66D33C1F6FF734FF000021A70F4
S21401D69040F6CE63C1F6FF734FF001021A7040F6F2
S21401D6A06C33C1F6FF734FF000021A7007F10807DA
S21401D6B0BD4680BD80B485B000AFF871B9717A718E
S21401D6C03B714FF00103BB734FF00003FB7368E03F
S21401D6D0BA79BB7B1340DBB2002B5AD0FB791A46D2
S21401D6E04FEA4202D3184FEA4303DAB2FB7BD31860
S21401D6F0DBB2A3F160037B737B79002B0AD07A7BC4
S21401D7003B7903F10103D9B240F6D423C1F6FF7386
S21401D71099543EE07A7B40F22253C1F6FF731B78A0
S21401D72003F10103D9B240F6D423C1F6FF7399542D
S21401D73040F22253C1F6FF731B78012B08D17A7B86
S21401D74040F6D423C1F6FF734FF00401995420E04C
S21401D7507A7B40F6D423C1F6FF739B5C002B10D076
S21401D7607A7B40F6D423C1F6FF739B5C022B10D85C
S21401D7707A7B40F6D423C1F6FF734FF00301995428
S21401D78007E07A7B40F6D423C1F6FF734FF015010C
S21401D7909954BB7B4FEA4303BB73FB7B03F1010345
S21401D7A0FB73FB7B052B93D907F11407BD4680BCA1
S21401D7B0704700BF80B584B000AFF88079713A71C8
S21401D7C0FB7040F6D563C1F6FF731B78002B40F063
S21401D7D01C8340F6D663C1F6FF731B78002B40F01E
S21401D7E0148397F8283083F00103DBB2002B06D0B0
S21401D7F040F66D33C1F6FF734FF000021A7040F623
S21401D8003833C1F6FF731B78022B21D040F6CC6368
S21401D810C1F6FF731B7883F00103DBB2002B40F0E7
S21401D820F6824FF013004FF000014FF0000201F0B6
S21401D8308FF94FF012004FF001014FF0000201F096
S21401D84087F940F63833C1F6FF734FF002021A70BB
S21401D85097F82C30FB73CEE24FF000033B734FF08A
S21401D8600003FB72B7F90620F97B40F6C823C1F620
S21401D870FF7333F811309A4240F06E81F97B41F222
S21401D8803C12C1F6FF720B464FEA43035B18D318EE
S21401D8901A787B7913407B71F97B41F23C12C1F611
S21401D8A0FF720B464FEA43035B18D31803F10103DB
S21401D8B01A783B7913403B71F97B41F23C12C1F671
S21401D8C0FF720B464FEA43035B18D31803F10203BA
S21401D8D01A78FB781340FB70FB7B1A464FEA42022C
S21401D8E0D318DBB203F11003BB7340F22253C1F627
S21401D8F0FF731B78142B04D097F82830002B00F008
S21401D9009680F87BFA7B40F6B823C1F6FF7333F8AE
S21401D9101230194641F25012C1F6FF720B464FEA19
S21401D92043035B184FEA83034FF4965101FB00F162
S21401D9305B18D318DB79B87B797997F82820FFF73D
S21401D940B9FEBA7BB97B40F60C73C1F6FF73595C1E
S21401D9507B790B43D9B240F60C73C1F6FF73995429
S21401D960BB7B03F10103BB73F87BFA7B40F6B8235C
S21401D970C1F6FF7333F81230194641F25012C1F660
S21401D980FF720B464FEA43035B184FEA83034FF4DB
S21401D990965101FB00F15B18D318DB79B87B397916
S21401D9A097F82820FFF786FEBA7BB97B40F60C7302
S21401D9B0C1F6FF73595C3B790B43D9B240F60C7341
S21401D9C0C1F6FF739954BB7B03F10103BB73F87B6C
S21401D9D0FA7B40F6B823C1F6FF7333F812301946C6
S21401D9E041F25012C1F6FF720B464FEA43035B1831
S21401D9F04FEA83034FF4965101FB00F15B18D318ED
S21401DA00DB79B87BF97897F82820FFF753FEBA7BC5
S21401DA10B97B40F60C73C1F6FF73595CFB780B4378
S21401DA20D9B240F60C73C1F6FF7399547CE0F87BCB
S21401DA30FA7B40F6B823C1F6FF7333F81230194665
S21401DA4041F25012C1F6FF720B464FEA43035B18D0
S21401DA504FEA83034FF4965101FB00F15B18D3188C
S21401DA60DB79B87B797997F82820FFF723FEBA7B14
S21401DA7040F60C73C1F6FF7379799954BB7B03F1B9
S21401DA800103BB73F87BFA7B40F6B823C1F6FF733C
S21401DA9033F81230194641F25012C1F6FF720B46A6
S21401DAA04FEA43035B184FEA83034FF4965101FB99
S21401DAB000F15B18D318DB79B87B397997F8282001
S21401DAC0FFF7F8FDBA7B40F60C73C1F6FF733979A0
S21401DAD09954BB7B03F10103BB73F87BFA7B40F6D9
S21401DAE0B823C1F6FF7333F81230194641F25012CB
S21401DAF0C1F6FF720B464FEA43035B184FEA8303F6
S21401DB004FF4965101FB00F15B18D318DB79B87B13
S21401DB10F97897F82820FFF7CDFDBA7B40F60C730D
S21401DB20C1F6FF73F978995440F64333C1F6FF7393
S21401DB30FA7B1A7097F8283083F00103DBB2002BCA
S21401DB4007D040F64333C1F6FF731B781846F8F743
S21401DB50EFFF4FF001033B73B7F91820F97B40F64E
S21401DB60C823C1F6FF7333F811309A4240F0E680BD
S21401DB70F97B41F23C12C1F6FF720B464FEA4303B2
S21401DB805B18D3181A783B7F13403B77F97B41F239
S21401DB903C12C1F6FF720B464FEA43035B18D318DB
S21401DBA003F101031A7897F82030134087F82030E4
S21401DBB0F97B41F23C12C1F6FF720B464FEA430372
S21401DBC05B18D31803F102031A7897F82430134030
S21401DBD087F82430FB7B1A464FEA4202D318DBB2A1
S21401DBE003F110037B7340F22253C1F6FF731B78D7
S21401DBF0012B57D07A7B3B7F104619464FF0000227
S21401DC004FF00003FFF756FD7A7B797B40F60C73E5
S21401DC10C1F6FF73595C3B7F0B43D9B240F60C73D8
S21401DC20C1F6FF7399547B7B03F101037B737A7B07
S21401DC3097F82030104619464FF000024FF00003C7
S21401DC40FFF738FD7A7B797B40F60C73C1F6FF73DC
S21401DC50595C97F820300B43D9B240F60C73C1F6E5
S21401DC60FF7399547B7B03F101037B737A7B97F8EF
S21401DC702430104619464FF000024FF00003FFF71C
S21401DC8019FD7A7B797B40F60C73C1F6FF73595CFC
S21401DC9097F824300B43D9B240F60C73C1F6FF73E4
S21401DCA099543EE07A7B3B7F104619464FF00002BE
S21401DCB04FF00003FFF7FEFC7A7B40F60C73C1F6CB
S21401DCC0FF73397F99547B7B03F101037B737A7B66
S21401DCD097F82030104619464FF000024FF0000327
S21401DCE0FFF7E8FC7A7B40F60C73C1F6FF7397F8F2
S21401DCF0201099547B7B03F101037B737A7B97F8A1
S21401DD002430104619464FF000024FF00003FFF78B
S21401DD10D1FC7A7B40F60C73C1F6FF7397F824109A
S21401DD20995440F64333C1F6FF73FA7B1A70FB7BB6
S21401DD301846F8F7FDFE4FF00103FB723B7B002B04
S21401DD4002D1FB7A002B03D04FF0010001F012F84C
S21401DD503B7B002B11D0BB7BA3F10203DBB2184641
S21401DD6001F066FBBB7B03F1FF33DBB2184601F023
S21401DD705FFBBB7B184601F05BFBFB7A002B15D0E3
S21401DD80BA7B7B7B9A4211D07B7BA3F10203DBB289
S21401DD90184601F04DFB7B7B03F1FF33DBB21846DF
S21401DDA001F046FB7B7B184601F042FB3B7B002BD8
S21401DDB002D1FB7A002B16D0FAF796FF40F6D16314
S21401DDC0C1F6FF734FF001021A7040F6CE63C1F63A
S21401DDD0FF734FF001021A7040F66C33C1F6FF7301
S21401DDE04FF000021A7097F82830002B11D1FB7BF8
S21401DDF003F10103FB7340F22353C1F6FF731B7853
S21401DE00FA7B9A42FFF428AD04E000BF02E000BFAF
S21401DE1000E000BF07F11007BD4680BD80B500AF2A
S21401DE2040F22253C1F6FF731B78142B13D04FF028
S21401DE30000000F09FFFFAF70BFF40F6D163C1F632
S21401DE40FF734FF000021A7040F6CE63C1F6FF73FF
S21401DE504FF000021A7080BD80B584B000AF034653
S21401DE60FB71FB7903F00703FB73FB7B042B0ED8D6
S21401DE7040F66A33C1F6FF73FA7B1A7040F26063AC
S21401DE80C1F6FF734FF001021A70F8F71DFEFB7919
S21401DE9003F00803002B07D040F22253C1F6FF73AC
S21401DEA04FF001021A7006E040F22253C1F6FF73EA
S21401DEB04FF014021A7040F25E63C1F6FF734FF022
S21401DEC001021A70FB7903F01003002B0CBF00232C
S21401DED00123DAB240F6D663C1F6FF731A7040F238
S21401DEE01E53C1F6FF734FF001021A7007F11007B7
S21401DEF0BD4680BD80B500AF40F6D363C1F6FF7363
S21401DF004FF001021A7040F63933C1F6FF734FF035
S21401DF101C021A70F9F7F6F840F21F53C1F6FF73A8
S21401DF204FF019021A7080BD80B582B000AF4FF075
S21401DF300003BB714FF00003FB7154E0FA7940F621
S21401DF40D423C1F6FF739B5C002B48D0FA7940F6C8
S21401DF50D423C1F6FF739B5C03F1FF33D9B240F6BD
S21401DF60D423C1F6FF739954FA7940F6D423C1F647
S21401DF70FF739B5C002B2FD1FB7918464FF00001F5
S21401DF8000F016FFFA7948F63963C3F6E303A3FBFC
S21401DF9002134FEA9303DAB240F64333C1F6FF7336
S21401DFA01B789A421BD1FA7948F63963C3F6E30324
S21401DFB0A3FB02134FEA93010B464FEAC3035B1818
S21401DFC04FEA4303D31ADBB218464FF000014FF075
S21401DFD0010200F0BDFD02E04FF00103BB71FB79C9
S21401DFE003F10103FB7140F22453C1F6FF731B7862
S21401DFF0FA799A42A2D340F6D163C1F6FF73BA7991
S21401E0001A7040F6D163C1F6FF731B7883F00103E3
S21401E010DBB2002B03D04FF0000000F0ABFE07F19F
S21401E0200807BD4680BD00BF80B500AF4FF0890030
S21401E0304FF000014FF000024FF00003F7F778FDB4
S21401E04080BD00BF80B500AF40F66E33C1F6FF73EA
S21401E0501B78002B1FD040F64333C1F6FF731B78A5
S21401E0601A4640F22353C1F6FF731B7803F1FF33C0
S21401E0709A4210DB40F64333C1F6FF734FF00002BD
S21401E0801A70F8F755FD40F66E33C1F6FF734FF080
S21401E09000021A7037E040F66E33C1F6FF731B7844
S21401E0A083F00103DBB2002B1ED040F64333C1F6EA
S21401E0B0FF731B781A4640F22353C1F6FF731B7891
S21401E0C003F1FF339A420FD140F66E33C1F6FF7368
S21401E0D04FF001021A7040F66F33C1F6FF731B78DA
S21401E0E01846F8F765FD0EE040F64333C1F6FF73B8
S21401E0F01B7803F10103DAB240F64333C1F6FF732E
S21401E1001A70F8F715FD4FF030004FF000014FF090
S21401E11000024FF00003F7F70BFD80BD80B483B01B
S21401E12000AF4FF00003FB7125E0FA7940F6882333
S21401E130C1F6FF734FF000019954FA7940F6802337
S21401E140C1F6FF734FF000019954FA7940F6A02307
S21401E150C1F6FF734FF0000123F81210FA7940F66A
S21401E160AC23C1F6FF734FF0000123F81210FB79C0
S21401E17003F10103FB7140F22353C1F6FF731B78D1
S21401E180FA799A42D1D340F6CA63C1F6FF734FF0CB
S21401E19000021A7007F10C07BD4680BC704700BF2D
S21401E1A080B582B000AF4FF00103BB714FF00003A2
S21401E1B0FB7110E0BA79F97940F68023C1F6FF7356
S21401E1C05B5C1340002B0CBF00230123BB71FB7962
S21401E1D003F10103FB7140F22353C1F6FF731B7871
S21401E1E0FA799A42E6D340F6CA63C1F6FF73BA7962
S21401E1F01A704FF00700F4F705FB07F10807BD4654
S21401E20080BD00BF80B485B000AF78604FF00003DA
S21401E210FB7323E0FA7B40F68023C1F6FF739B5C19
S21401E22083F00103DBB2002B14D07B68FA7B1A70F3
S21401E230FB7B4FEAC303BB73FA7B40F68823C1F628
S21401E240FF739B5C002B03D0BB7B43F04003BB7387
S21401E250BB7B0DE0FB7B03F10103FB7340F2235311
S21401E260C1F6FF731B78FA7B9A42D3D34FF068034B
S21401E270184607F11407BD4680BC704780B485B0C8
S21401E28000AF0346FB804FF00003FB7310E0FA7B00
S21401E29040F6C823C1F6FF7333F81230FA889A4263
S21401E2A002D14FF001030DE0FB7B03F10103FB7389
S21401E2B040F22353C1F6FF731B78FA7B9A42E6D3EA
S21401E2C04FF00003184607F11407BD4680BC70479F
S21401E2D080B483B000AF0346FB71FB79002B0ED1EF
S21401E2E040F67003C1F6FF734FF001021A7040F654
S21401E2F06D33C1F6FF734FF000021A700DE040F265
S21401E3002853C1F6FF731B78FA799A4205D240F278
S21401E3102853C1F6FF73FA791A7007F10C07BD4648
S21401E32080BC704780B582B000AF4FF00003FB7130
S21401E3304FF064004FF0640100F0FCFC00F046FE74
S21401E34001F03AF84FF28003C4F20F034FF4006273
S21401E3509A60F8F70FF8F8F781FF2AE0FB79002BAF
S21401E3600CBF00230123DBB2FA7902F10102FA7134
S21401E370002B0AD04DF2DC30C0F203000DF0D4FDC4
S21401E3804FF00700F8F7DAFF05E04DF22040C0F243
S21401E39003000DF0C9FD4FF022004FF000014FF0D1
S21401E3A000024FF00003F7F7C3FB4FF4FA7010F0CA
S21401E3B03DFC40F25053C1F6FF731B881BB213F1AC
S21401E3C0020FCBD04FF030004FF000014FF00002AB
S21401E3D04FF00003F7F7ACFB4FF47A7010F026FC11
S21401E3E003E04FF0640010F021FC40F26363C1F6D5
S21401E3F0FF731B7883F00103DBB2002BF1D1F8F732
S21401E40051FF4FF47A7010F011FC4FF005004DF2F9
S21401E4103841C0F203014AF67852C0F20302F9F716
S21401E4208FF84FF005004DF24841C0F203014AF65D
S21401E4307852C0F20302F9F783F84FF47A7010F0BD
S21401E440F5FB4FF005004DF23841C0F203014AF6E4
S21401E4507852C0F20302F9F773F84FF005004DF257
S21401E4605841C0F203014AF67852C0F20302F9F7A6
S21401E47067F84FF033004FF000014FF000024FF005
S21401E4800003F7F755FB4FF47A7010F0CFFB00F05E
S21401E490C1F80346002B0CBF00230123DBB283F037
S21401E4A00103DBB203F00103DAB240F6CB63C1F637
S21401E4B0FF731A7040F6CB63C1F6FF731B78002B0F
S21401E4C022D04FF47A7010F0B1FB40F66B33C1F6F0
S21401E4D0FF731B781846F8F731FF40F66B33C1F629
S21401E4E0FF731B78012B0CBF00230123DBB24FF017
S21401E4F00000194600F0E2FC40F21F53C1F6FF731C
S21401E5004FF000021A7013E0F8F7BEFB00F05EFD54
S21401E510F8F7C8F940F6CC63C1F6FF731B7883F0B1
S21401E5200103DBB2002B03D04FF00100FAF7BAFC6F
S21401E5304FF064004FF0640100F0FCFBF9F722F89D
S21401E54040F6C423C1F6FF734FF01E021A7007F19E
S21401E5500807BD4680BD00BF80B584B000AF7860B7
S21401E5604DF2A440C0F203000DF0DEFC4FF4FA5069
S21401E57010F05CFB40F2A453C1F6FF731B78002B2E
S21401E58043D000F051FB4FF00003BB734FF0000384
S21401E590FB7332E0FA7B40F6FC63C1F6FF739B5CCB
S21401E5A0002B13D0FA7B40F60473C1F6FF739B5C15
S21401E5B0002B1ED1FA7B40F6FC63C1F6FF734FF0C9
S21401E5C0000199544FF00103BB7312E0FA7B40F649
S21401E5D00473C1F6FF739B5C032B0AD1FA7B40F6EA
S21401E5E0FC63C1F6FF734FF0010199544FF001032C
S21401E5F0BB73FB7B03F10103FB73FB7B042BC9D9C4
S21401E600BB7B002B01D0F9F719FE4FF0050010F087
S21401E6100DFBAFE780B582B000AF4FF00003FB7192
S21401E6204FF000033B60FAF713FB4FF005004DF285
S21401E6303841C0F203014AF67852C0F20302F8F7F5
S21401E6407FFF4FF005004DF2C841C0F203014AF6C4
S21401E6507852C0F20302F8F773FF40F66933C1F649
S21401E660FF731B78002B09D140F66B33C1F6FF739D
S21401E6704FF001021A704FF00003F1E04FF0000076
S21401E68000F078FB4FF00A0010F0D0FA4FF240038A
S21401E690C4F20F034FF480025A604FF28003C4F2B3
S21401E6A00F034FF480529A604FF0960010F0BEFAB6
S21401E6B000F03CFE38603A6840F68B239A4210D848
S21401E6C04FF24003C4F20F034FF480029A6040F603
S21401E6D06B33C1F6FF734FF001021A704FF000035F
S21401E6E0BEE04FF28003C4F20F034FF480525A602B
S21401E6F000F01CFE38604FF0140010F097FA00F09E
S21401E70015FE38604FF24003C4F20F034FF4800247
S21401E7109A604FF00A0010F089FA3A6840F2BB237B
S21401E7209A428CBF00230123DAB2396840F2E243F1
S21401E730994294BF00230123DBB21343DBB2002BC3
S21401E74010D04FF28003C4F20F034FF480529A6048
S21401E75040F66B33C1F6FF734FF002021A704FF0AA
S21401E76000037DE04FF0010000F004FB4FF03200A3
S21401E77010F05CFA00F0DAFD38604FF0000000F0AF
S21401E780F9FA4FF28003C4F20F034FF480529A60F5
S21401E7904FF4617010F04AFA4FF005004DF238411F
S21401E7A0C0F203014AF67852C0F20302F8F7C8FE37
S21401E7B04FF005004DF2D841C0F203014AF67852F7
S21401E7C0C0F20302F8F7BCFE4FF00003FB7109E04C
S21401E7D000F0D6FB4FF00A0010F028FAFB7903F19F
S21401E7E00103FB71FB79632BF2D93A6840F61B43B0
S21401E7F09A422CD84FF005004DF23841C0F2030181
S21401E8004AF67852C0F20302F8F79AFE4FF0050076
S21401E8104DF2E841C0F203014AF67852C0F2030213
S21401E820F8F78EFE4FF0010000F020F840F2DC50C1
S21401E83010F0FCF900F040F94FF0020000F016F875
S21401E84040F2DC5010F0F2F900F036F906E040F63E
S21401E850CC63C1F6FF734FF001021A704FF001034B
S21401E860184607F10807BD4680BD00BF80B584B0D5
S21401E87000AF0346FB71FB79012B02D0022B04D0BB
S21401E88007E04FF01503FB7304E04FF02A03FB7318
S21401E89000E022E04FF00003BB731BE0BA7BB97BBC
S21401E8A040F60C73C1F6FF735B5CDBB203F040030A
S21401E8B0D9B2FB7B0B43DBB2D9B240F60C73C1F67F
S21401E8C0FF739954BB7B184600F0B2FDBB7B03F186
S21401E8D00103BB73BB7B052BE0D907F11007BD46CF
S21401E8E080BD00BF80B582B000AF4FF00003FB7162
S21401E8F040F63833C1F6FF731B78022B00F0B78061
S21401E90040F6CB63C1F6FF731B78002B40F0AF8057
S21401E91040F62F73C1F6FF731B78002B40F0A980D9
S21401E92040F62F73C1F6FF734FF001021A704FF0D5
S21401E930000000F01FFA4FF24003C4F20F034FF439
S21401E94080025A604FF0960010F070F94FF0000305
S21401E950FB706FE04FF000033B714FF00003BB719B
S21401E9604FF000037B7150E07B79062B15D1397986
S21401E970F87840F64832C1F6FF720B464FEA830339
S21401E9805B181B18D318BA791A703B7903F1010387
S21401E9903B714FF00003BB7117E07B790C2B14D150
S21401E9A03979F87840F64832C1F6FF720B464FEADD
S21401E9B083035B181B18D318BA791A703B7903F1D5
S21401E9C001033B714FF00003BB71FB79FA7902F149
S21401E9D00102FA71184600F0FFFB0346BB7040F6D1
S21401E9E03833C1F6FF731B78022B30D0BB794FEA60
S21401E9F05303BB71BB78002B03D0BB7963F07F0355
S21401EA00BB717B7903F101037B717B79112BABD948
S21401EA103979F87840F64832C1F6FF720B464FEA6C
S21401EA2083035B181B18D318BA791A70FB7803F1A5
S21401EA300103FB7040F22353C1F6FF731B78FA788B
S21401EA409A4287D34FF00000FBF7A2FD00E000BF1B
S21401EA504FF24003C4F20F034FF480029A6040F66F
S21401EA602F73C1F6FF734FF000021A7002E000BF69
S21401EA7000E000BF07F10807BD4680BD80B582B043
S21401EA8000AF4FF01003FB710FE0FA7940F60C73FC
S21401EA90C1F6FF734FF000019954FB79184600F058
S21401EAA0C7FCFB7903F10103FB71FB791F2BECD942
S21401EAB007F10807BD4680BD80B582B000AF4FF0B4
S21401EAC00003FB7116E0FA79F97940F60C73C1F68A
S21401EAD0FF735B5C23F03F03D9B240F60C73C1F6BB
S21401EAE0FF739954FB79184600F0A2FCFB7903F1F9
S21401EAF00103FB71FB79052BE5D907F10807BD4634
S21401EB0080BD00BF80B582B000AF4FF00003FB713F
S21401EB1016E0FA79F97940F60C73C1F6FF735B5C7F
S21401EB2023F07F03D9B240F60C73C1F6FF739954F4
S21401EB30FB79184600F07CFCFB7903F10103FB71BD
S21401EB40FB79052BE5D907F10807BD4680BD00BF57
S21401EB5080B584B000AF13460246FA710A46BA7110
S21401EB607B71FB79112B21D8FA794AF6AB23CAF6C9
S21401EB70AA23A3FB02034FEA93010B464FEA430382
S21401EB805B184FEA4303D31AFB737A79F9794AF68D
S21401EB90AB23CAF6AA23A3FB01034FEA9303DBB216
S21401EBA04FEA430302FA03F3BB7316E0FB79132B18
S21401EBB007D0142B09D0122B0BD14FF00203FB7395
S21401EBC008E04FF00103FB7304E04FF00003FB7312
S21401EBD000E025E04FF04003BB73F97BBB79002BC7
S21401EBE009D0FA7B40F60C73C1F6FF739A5CBB7BC7
S21401EBF01343DAB20BE0FA7B40F60C73C1F6FF73EF
S21401EC009A5CBB7B6FEA0303DBB21340DAB240F6D1
S21401EC100C73C1F6FF735A54FB7B184600F008FCD0
S21401EC2007F11007BD4680BD80B582B000AF00F089
S21401EC307BFC4FF28003C4F20F031B697B7100F06B
S21401EC4091FC4FF00203FB714FF00003BB716AE0C9
S21401EC507A79FB791340DBB2002B27D0BA7940F6DC
S21401EC600473C1F6FF739B5C042B08D1BA7940F696
S21401EC700473C1F6FF734FF0000199542CE0BA7982
S21401EC8040F60473C1F6FF739B5C002B24D0BA795F
S21401EC9040F60473C1F6FF739B5C03F1FF33D9B2F0
S21401ECA040F60473C1F6FF73995415E0BA7940F63D
S21401ECB00473C1F6FF739B5C022B0DD8BA7940F63C
S21401ECC00473C1F6FF739B5C03F10103D9B240F6EE
S21401ECD00473C1F6FF739954FB79102B13D0102BD4
S21401ECE004DC022B07D0082B09D018E0202B0ED00D
S21401ECF0402B10D013E04FF00803FB710FE04FF0EC
S21401ED001003FB710BE04FF02003FB7107E04FF09F
S21401ED104003FB7103E04FF00203FB7100BFBB79B8
S21401ED2003F10103BB71BB79042B91D907F10807E5
S21401ED30BD4680BD80B582B000AF02460B46FA7173
S21401ED40BB71FB799AB2BB794FF032004FF00001EC
S21401ED50F6F7EEFE40F21D53C1F6FF73FA791A700C
S21401ED6040F21C53C1F6FF73BA791A7007F108070F
S21401ED70BD4680BD80B483B000AF0346FB71FB790E
S21401ED80002B07D04FF28003C4F20F034FF400525A
S21401ED905A6006E04FF28003C4F20F034FF40052AC
S21401EDA09A6000BF07F10C07BD4680BC704700BFE4
S21401EDB080B584B000AF02460B46FA71BB71FA7992
S21401EDC04AF6AB23CAF6AA23A3FB02134FEA930320
S21401EDD0DBB203F11003FB73FA794AF6AB23CAF6EA
S21401EDE0AA23A3FB02134FEA93010B464FEA430300
S21401EDF05B184FEA4303D31ADBB24FF0010202FA63
S21401EE0003F3BB73BB79002B0FD0FA7BF97B40F67B
S21401EE100C73C1F6FF73595CBB7B0B43D9B240F64A
S21401EE200C73C1F6FF73995413E0FA7BF97B40F635
S21401EE300C73C1F6FF735B5CD9B2BB7B6FEA03034D
S21401EE40DBB20B40DBB2D9B240F60C73C1F6FF73EE
S21401EE509954FB7B184600F0EBFA07F11007BD4604
S21401EE6080BD00BF80B582B000AF4DF2F840C0F261
S21401EE7003000DF059F84FF000037B604FF46D432B
S21401EE80CEF200033B603B68DB687B607B684FEA41
S21401EE9003434FEA13437B607B6843F0BF6343F44D
S21401EEA000337B607B6843F004037B603B687A68D1
S21401EEB0DA6007F10807BD4680BD00BF80B582B0A5
S21401EEC000AF02460B46FA71BB7140F62E73C1F6CF
S21401EED0FF731B78002B4ED14DF20850C0F2030091
S21401EEE00DF022F8FFF70EFEFB79002B21D04FF034
S21401EEF014004FF001014FF00002FFF729FEF7F76B
S21401EF00FBFC4FF004004DF22451C0F203014AF617
S21401EF107852C0F20302F8F713FB4FF006004DF2E9
S21401EF203451C0F203014AF67852C0F20302F8F7F0
S21401EF3007FB40F62E73C1F6FF734FF001021A70FD
S21401EF404FF47043C4F20F034FF480525A604FF0EF
S21401EF5021004FF000014FF000024FF00003F6F7DA
S21401EF60E7FDBB79002B07D04DF23C50C0F2030001
S21401EF700CF0DAFFFEE700BF07F10807BD4680BDCB
S21401EF8080B582B000AFFFF74FFE4FF00003FB7174
S21401EF9015E0FA7940F60473C1F6FF739B5C002B0B
S21401EFA009D04FF00300F8F7C9F94FF000004FF011
S21401EFB00101FFF783FFFB7903F10103FB71FB7985
S21401EFC0042BE6D907F10807BD4680BD80B586B09B
S21401EFD000AF3B4618464FF0060100F0E5FE3868E4
S21401EFE0B968FA687B6900F0A7FF03461A4646F639
S21401EFF04C73C1F6FF731A807868B9683A697B6901
S21401F00000F09AFF03461A4646F64C73C1F6FF73A4
S21401F0105A8000F005F807F11807BD4680BD00BF0D
S21401F02080B500AF46F64C73C1F6FF735B881A468F
S21401F03040F66A33C1F6FF731B78194640F27853DF
S21401F040C1F6FF7353F821309A4207D840F6693368
S21401F050C1F6FF734FF000021A703BE046F64C73A0
S21401F060C1F6FF735B881A4640F66A33C1F6FF7332
S21401F0701B78194640F27853C1F6FF7353F82130D6
S21401F080D21A13464FEA83039B184FEA43031A46E4
S21401F09040F66A33C1F6FF731B78194640F28C536B
S21401F0A0C1F6FF7353F82130B2FBF3F3DAB240F640
S21401F0B06933C1F6FF731A7040F66933C1F6FF7300
S21401F0C01B78092B06D940F66933C1F6FF734FF05A
S21401F0D009021A7040F66A33C1F6FF731B78002BDB
S21401F0E043D146F64C73C1F6FF731B881A4640F2AD
S21401F0F07053C1F6FF731B689A4207D840F668330F
S21401F100C1F6FF734FF000021A7038E046F64C73F2
S21401F110C1F6FF731B881A4640F27053C1F6FF739F
S21401F1201B68D21A13464FEA83039B184FEA430320
S21401F1301A4640F27453C1F6FF731B68B2FBF3F331
S21401F140DAB240F66833C1F6FF731A7040F66833D8
S21401F150C1F6FF731B78092B11D940F66833C1F647
S21401F160FF734FF009021A7009E040F66933C1F6E1
S21401F170FF731A7840F66833C1F6FF731A7040F2CF
S21401F1801F53C1F6FF731B78002B0BD14FF0000005
S21401F1904FF00101F7F7E6FB4FF001004FF00101D8
S21401F1A0F7F7E0FB40F66833C1F6FF731B78DBB276
S21401F1B003F00F03DAB240F66933C1F6FF731B782A
S21401F1C04FEA0313DBB21343DBB2DAB240F2205349
S21401F1D0C1F6FF731A7080BD80B584B000AF0346D8
S21401F1E0FB71FB7918464FF00101FFF7E1FD4FF087
S21401F1F005000FF01BFD00F019F8F860FB791846C2
S21401F2004FF00001FFF7D4FD40F2A053C1F6FF73A3
S21401F2101B68FA689A4202D84FF0010301E04FF0EA
S21401F2200003184607F11007BD4680BD80B584B0BF
S21401F23000AF3C4802F088FD0346002B05D03B4654
S21401F2403848194602F046FD05E04DF25050C0F22E
S21401F25003000CF069FE344802F076FD0346002BED
S21401F26006D007F102033048194602F033FD05E0E7
S21401F2704DF27050C0F203000CF056FE7B8840F64B
S21401F280E44202FB03F3002B03DA03F57F4303F1A9
S21401F290FF034FEA23437B603B881A4640F2A8539C
S21401F2A0C1F6FF731B689A4206D84FF000033B80F5
S21401F2B04FF00003FB6017E03A8840F2A853C1F60E
S21401F2C0FF731B689BB2D31A9BB23B803B8840F608
S21401F2D0E44202FB03F3002B03DA03F57F4303F159
S21401F2E0FF034FEA2343FB607A68FB689A4205D81E
S21401F2F04FF44A43C3F69A33BB600CE0FA6844F213
S21401F3004023C0F20F0303FB02F27968FB68CB1AB5
S21401F310B2FBF3F3BB60BB68184607F11007BD46A6
S21401F32080BD00BFE876FF1FFC76FF1F80B582B068
S21401F33000AF204802F008FD0346002B06D007F177
S21401F34002031C48194602F0C5FC05E04DF2505078
S21401F350C0F203000CF0E8FD7B881A4640F2A85381
S21401F360C1F6FF731B689A4206D84FF000037B80F4
S21401F3704FF000037B6017E07A8840F2A853C1F68D
S21401F380FF731B689BB2D31A9BB27B807B8840F6C7
S21401F390E44202FB03F3002B03DA03F57F4303F198
S21401F3A0FF034FEA23437B607B68184607F1080793
S21401F3B0BD4680BDE876FF1F80B582B000AF4FF036
S21401F3C00003FB7107E0FB79184600F031F8FB7982
S21401F3D003F10103FB71FB79052BF4D94FF0100300
S21401F3E0FB7107E0FB79184600F022F8FB7903F180
S21401F3F00103FB71FB791E2BF4D907F10807BD4603
S21401F40080BD00BF80B582B000AF02460B46FA71E0
S21401F410BB71FA7940F60C73C1F6FF73B97999544A
S21401F420FB79184600F004F807F10807BD4680BDD1
S21401F43080B582B000AF0346FB7140F62D73C1F66E
S21401F440FF731B78002B69D100F06EF84FF2800332
S21401F450C4F20F034FF6FF72C0F204025A614FF076
S21401F460020000F08BF84FF28003C4F20F034FF254
S21401F4708002C4F20F02126922F0FF01FA790A43F0
S21401F4801A604FF28003C4F20F034FF480725A6081
S21401F4904FF28003C4F20F034FF480729A604FF26A
S21401F4A08003C4F20F034FF28002C4F20F02126906
S21401F4B022F0FF01F87940F60C72C1F6FF72125C79
S21401F4C00A431A60FB790F2B0ED94FF28003C4F260
S21401F4D00F034FF480629A604FF28003C4F20F0369
S21401F4E04FF480625A600DE04FF28003C4F20F03BE
S21401F4F04FF400729A604FF28003C4F20F034FF488
S21401F50000725A604FF28003C4F20F034FF47F4239
S21401F510C0F204025A6100F025F800E000BF07F1CE
S21401F5200807BD4680BD00BF80B500AF40F62D730D
S21401F530C1F6FF731B78002B04D011E04FF00100D9
S21401F5400FF074FB40F62C73C1F6FF731B78002B8B
S21401F550F4D140F62C73C1F6FF734FF001021A7016
S21401F56080BD00BF80B400AF40F62C73C1F6FF73B8
S21401F5704FF000021A70BD4680BC704780B485B05B
S21401F58000AF78604FF00003FB6003E0FB6803F117
S21401F5900103FB60FA687B689A42F7DB07F1140700
S21401F5A0BD4680BC704700BF80B400AF4FF2400339
S21401F5B0C4F20F031B6903F00403002B02D04FF0C3
S21401F5C0000201E04FF002024FF24003C4F20F03C3
S21401F5D01B6903F00203002B14BF00230123DBB2D7
S21401F5E0D318DBB203F10203DAB240F22353C1F6B9
S21401F5F0FF731A7040F22353C1F6FF731B781A4645
S21401F6004FEAC202D3184FEA4303DAB240F2245358
S21401F610C1F6FF731A70BD4680BC704780B500AF57
S21401F6204FF47043C4F20F0341F210025A614FF2D5
S21401F6304003C4F20F034FF40062C0F27C025A6129
S21401F6404FF28003C4F20F034FF47F42C0F204026C
S21401F6505A614FF2C003C4F20F034FF080025A61A1
S21401F6604FF47143C4F20F034FF000025A614FF496
S21401F6701043C4F204034FF41042C4F20402526B66
S21401F68022F4E06242F480725A634FF41043C4F2EB
S21401F69004034FF41042C4F20402526922F4E062F9
S21401F6A042F480725A614FF41043C4F204034FF4DB
S21401F6B01042C4F20402526C22F4E06242F48072F8
S21401F6C05A644FF41043C4F204034FF41042C4F2D8
S21401F6D00402126B22F4E06242F480721A634FF461
S21401F6E01043C4F204034FF41042C4F20402126938
S21401F6F022F4E06242F480721A614FF41043C4F2BD
S21401F70004034FF41042C4F20402126942F00302E9
S21401F7101A614FF41043C4F204034FF41042C4F2CA
S21401F7200402126C22F4E06242F480721A644FF40E
S21401F7302043C4F204034FF42042C4F20402526888
S21401F74022F4E06242F480725A604FF42043C4F21D
S21401F75004034FF42042C4F20402526842F003024A
S21401F7605A604FF42043C4F204034FF42042C4F21B
S21401F7700402926822F4E06242F480729A604FF4C6
S21401F7802043C4F204034FF42042C4F204029268F8
S21401F79042F003029A604FF42043C4F204034FF48C
S21401F7A02042C4F20402D26822F4E06242F480727B
S21401F7B0DA604FF42043C4F204034FF42042C4F24B
S21401F7C00402D26842F00302DA604FF42043C4F226
S21401F7D004034FF42042C4F20402526A22F4E062A7
S21401F7E042F480725A624FF42043C4F204034FF489
S21401F7F02042C4F20402526A42F003025A624FF4F3
S21401F8002043C4F204034FF42042C4F20402926A75
S21401F81022F4E06242F480729A624FF42043C4F20A
S21401F82004034FF42042C4F20402926A42F0030237
S21401F8309A624FF42043C4F204034FF42042C4F208
S21401F8400402D26A22F4E06242F48072DA624FF471
S21401F8502043C4F204034FF42042C4F20402126CA3
S21401F86022F4E06242F480721A644FF42043C4F238
S21401F87004034FF42042C4F20402526C22F4E06204
S21401F88042F480725A644FF42043C4F204034FF4E6
S21401F8902042C4F20402926C22F4E06242F48072C6
S21401F8A09A644FF42043C4F204034FF42042C4F296
S21401F8B00402D26C22F4E06242F48072DA644FF4FD
S21401F8C02043C4F204034FF42042C4F20402126D32
S21401F8D022F4E06242F480721A654FF42043C4F2C7
S21401F8E004034FF42042C4F20402526D22F4E06293
S21401F8F042F480725A654FF42043C4F204034FF475
S21401F9002042C4F20402926D22F4E06242F4807254
S21401F9109A654FF42043C4F204034FF42042C4F224
S21401F9200402D26D22F4E06242F48072DA654FF48A
S21401F9303043C4F204034FF43042C4F204021268A6
S21401F94022F4E06242F480721A604FF43043C4F24B
S21401F95004034FF43042C4F20402526822F4E06217
S21401F96042F480725A604FF43043C4F204034FF4F9
S21401F9703042C4F20402926822F4E06242F48072D9
S21401F9809A604FF43043C4F204034FF43042C4F299
S21401F9900402D26822F4E06242F48072DA604FF424
S21401F9A03043C4F204034FF43042C4F20402126935
S21401F9B022F4E06242F480721A614FF43043C4F2DA
S21401F9C004034FF43042C4F20402526922F4E062A6
S21401F9D042F480725A614FF43043C4F204034FF488
S21401F9E03042C4F20402926922F4E06242F4807268
S21401F9F09A614FF43043C4F204034FF43042C4F228
S21401FA000402D26922F4E06242F48072DA614FF4B1
S21401FA103043C4F204034FF43042C4F20402126AC3
S21401FA2022F4E06242F480721A624FF43043C4F268
S21401FA3004034FF43042C4F20402526A22F4E06234
S21401FA4042F480725A624FF43043C4F204034FF416
S21401FA503042C4F20402926A22F4E06242F48072F6
S21401FA609A624FF43043C4F204034FF43042C4F2B6
S21401FA700402D26A22F4E06242F48072DA624FF43F
S21401FA803043C4F204034FF43042C4F20402126B52
S21401FA9022F4E06242F480721A634FF43043C4F2F7
S21401FAA004034FF43042C4F20402526B22F4E062C3
S21401FAB042F480725A634FF43043C4F204034FF4A5
S21401FAC03042C4F20402926B22F4E06242F4807285
S21401FAD09A634FF43043C4F204034FF43042C4F245
S21401FAE00402D26B22F4E06242F48072DA634FF4CD
S21401FAF03043C4F204034FF43042C4F20402926C61
S21401FB0022F4E06242F480729A644FF44043C4F2F5
S21401FB1004034FF44042C4F20402D26922F4E062C4
S21401FB2042F48072DA614FF45043C4F204034FF496
S21401FB305042C4F20402126922F4E06242F4807276
S21401FB401A614FF45043C4F204034FF45042C4F216
S21401FB500402526922F4E06242F480725A614FF460
S21401FB605043C4F204034FF45042C4F204029269B3
S21401FB7022F4E06242F480729A614FF45043C4F278
S21401FB8004034FF45042C4F20402926E22F4E0627F
S21401FB9042F480729A664FF28003C4F20F034FF468
S21401FBA000529A604FF24003C4F20F034FF48002F2
S21401FBB09A604FF28003C4F20F034FF480529A60AA
S21401FBC04FF28003C4F20F034FF400625A604FF203
S21401FBD04003C4F20F034FF400229A604FF28003F1
S21401FBE0C4F20F034FF400725A604FF28003C4F25E
S21401FBF00F034FF480625A604FF28003C4F20F0382
S21401FC004FF480729A604FF47043C4F20F034FF4BE
S21401FC1080329A604FF47043C4F20F034FF480525F
S21401FC209A604FF47043C4F20F034FF010029A60CB
S21401FC304FF28003C4F20F034FF480229A604FF212
S21401FC408003C4F20F034FF400425A604FF2C00320
S21401FC50C4F20F034FF080029A604DF6C400C0F262
S21401FC60030001F073FD4DF6DC00C0F2030001F065
S21401FC706DFD47F27060C1F6FF7042F2072101F098
S21401FC809DFF034683F00103DBB2002B05D04DF246
S21401FC90CC50C0F203000CF047F93C4842F2062172
S21401FCA001F08CFF034683F00103DBB2002B05D085
S21401FCB04DF2F050C0F203000CF036F9344841F230
S21401FCC0064101F07BFF034683F00103DBB2002B04
S21401FCD005D04DF21460C0F203000CF025F92D4852
S21401FCE042F2052101F06AFF034683F00103DBB20D
S21401FCF0002B05D04DF23860C0F203000CF014F969
S21401FD00254842F2042101F059FF034683F001031E
S21401FD10DBB2002B05D04DF25C60C0F203000CF0A4
S21401FD2003F91E4841F2074101F048FF034683F0FC
S21401FD300103DBB2002B05D04DF28060C0F2030058
S21401FD400CF0F2F8164841F2010101F037FF0346C4
S21401FD5083F00103DBB2002B05D04DF2A460C0F2A4
S21401FD6003000CF0E1F80F4842F2010101F026FF12
S21401FD70034683F00103DBB2002B05D04DF2C860C9
S21401FD80C0F203000CF0D0F880BD00BF8476FF1FE0
S21401FD909876FF1FAC76FF1FC076FF1FD476FF1F35
S21401FDA0E876FF1FFC76FF1F90B585B000AF786040
S21401FDB00B46FB704FF00003FB7346E0FA7B1346DD
S21401FDC04FEA83039B184FEA830347F27062C1F63A
S21401FDD0FF729B18184601F0B7FF0346002B2AD086
S21401FDE0FA7B13464FEA83039B184FEA830347F2D5
S21401FDF07062C1F6FF729A18FB7B4FEA830379683B
S21401FE00CB181046194601F065FF0346002B18D0A3
S21401FE10FB7B4FEA83037A68D418FB7B4FEA8303A4
S21401FE207A68D3181B68FA7B1046194600F016F854
S21401FE300346236005E04DF2EC60C0F203000CF0CF
S21401FE4073F8FB7B03F10103FB73FA7BFB789A42A1
S21401FE50B4D307F11407BD4690BD00BF80B485B08A
S21401FE6000AF03463960FB71FB79062B48D801A128
S21401FE7051F823F091FE0100A7FE0100BDFE01002E
S21401FE80D3FE0100D3FE0100D3FE0100E5FE010012
S21401FE904FF49F43C0F21203FB604CF6A843C0F236
S21401FEA00303BB602CE04FF49F43C0F21203FB60D8
S21401FEB048F2A063C0F20103BB6021E048F22033A0
S21401FEC0C0F20C03FB6048F2A063C0F20103BB6002
S21401FED016E046F24003C0F20A03FB604CF2EC2344
S21401FEE0BB600DE03B6840F6E44202FB03F248F2D9
S21401FEF00103C8F20003A3FB02134FEAD33314E055
S21401FF003B6840F6E44202FB03F248F20103C8F202
S21401FF100003A3FB02134FEAD333F968BA688A18C1
S21401FF2002FB03F2BB68B2FBF3F3184607F11407B2
S21401FF30BD4680BC704700BF80B487B000AFF86094
S21401FF40B9607A603B604FF000037B61FA687B69B9
S21401FF509A4201D9FB687B61BA687B699A4201D9EA
S21401FF60BB687B617A687B699A4201D97B687B6151
S21401FF703A687B699A4201D93B687B617B699BB28F
S21401FF80184607F11C07BD4680BC70470BF0AEFC57
S21401FF900BF0A6FC0A480B4A0021121A17F0FCF8CF
S21401FFA016F0BAFC16F0DCFC16F054FC16F0E6FC73
S21401FFB00549002000F03AFC17F08CF8FEE700BF78
S21401FFC03006FF1F6C77FF1F300FFF1FFEE7000094
S21401FFD090B585B000AF786039604FF4597012F073
S21401FFE02BFEB860BB68002B02D14FF0FF3386E1D1
S21401FFF0B86845F2010113F06BF9BB687A68C3F87B
S21402000044223B68002B1BD03B681B78272B0CD165
S214020010BB6803F144023B6803F10103104619462C
S2140200204FF4807217F0EBF80AE038684DF2FC6184
S214020030C0F203010CF032F80246BB68C3F848224D
S214020040BB68D3F84832002B07D14FF000000EF001
S2140200506DF80246BB68C3F84822B8684FF0000144
S21402006000F05EFABB6803F14403002B0AD0BB68BB
S21402007003F144034DF20070C0F2030019460BF080
S21402008053FF05E04DF20C70C0F203000BF04CFF7C
S2140200904FF001000EF04AF8034618460CF082F9BB
S2140200A019E1BB6893F84C3283F00103DBB2002BF4
S2140200B000F0AE80BB6893F84430002B00F0A880B6
S2140200C0BB68D3F848424FF000000EF02FF8034604
S2140200D09C4209D0BB6803F144034DF21470C0F28F
S2140200E0030019460BF020FFBB6893F84430232B1D
S2140200F000F08E80BB6803F1440318464DF2187177
S214020100C0F2030117F04EF80346002B0CD1BB6871
S21402011003F14402BB6803F5A273104619464FF476
S214020120807217F06CF825E0BB6803F144031846AA
S2140201304DF21C71C0F2030117F034F80346002B8F
S2140201400CD1BB6803F14402BB6803F5A2731046E8
S21402015019464FF4807217F052F80BE0BB6803F5AD
S214020160A272BB6803F14403104619464FF480722C
S21402017017F045F8BB6803F14402BB6810461946FF
S21402018000F0C2F80246BB681A64BB681B6C002B00
S2140201903EDDBB681B6818460BF028FD4FF00003D7
S2140201A0FB601FE0BB681A68FB684FEAC303796806
S2140201B0CB181B681046194616F0F4FF0346002BB0
S2140201C00CD1FB684FEAC3037A68D3185B68BA6837
S2140201D0116CBA680846114698470BE0FB6803F1B3
S2140201E00103FB60FB684FEAC3037A68D3181B68F7
S2140201F0002BD7D1FB684FEAC3037A68D3181B6873
S214020200002B05D14DF22070C0F203000BF08CFEDD
S214020210BB6893F84C3283F00103DBB2002B5AD052
S2140202204DF20C70C0F203000BF07EFE4FF00100A0
S2140202300DF07CFF034618460CF0B4F8BB6803F1D9
S2140202404402BB68D3F8483210464FF480711A460F
S2140202500BF0A6FF0346002B2ED1BB68D3F848420C
S2140202604FF000000DF062FF03469C421ED0BB68B2
S214020270D3F8483218460CF0C7F84FF000000DF0DD
S21402028055FF0246BB68C3F84822BB684FF000021F
S21402029083F84421BB684FF0000283F844204DF2F5
S2140202A05870C0F203000BF03FFE05E0BB684FF04B
S2140202B0010283F84C220EE0BB6893F84430002B10
S2140202C009D1BB68D3F848424FF000000DF02EFF6C
S2140202D003469C42B2D1BB6893F84C3283F00103CA
S2140202E0DBB2002B7FF4DDAE4DF25C70C0F2030091
S2140202F00BF01AFEB86812F075FD4FF000031846B0
S21402030007F11407BD4690BD80B586B000AF786091
S21402031039607B687B614FF00003FB604FF000039F
S214020320FB724FF000033B6178E07B6903F1010347
S2140203307B6100E000BF7B691B78002B07D07B69DE
S2140203401B78184616F082FF0346002BEDD07B6919
S2140203501B78002B08D13B694FEA83033A68D3180F
S2140203604FF000021A6055E04FF00003BB72FB68C4
S21402037003F10103FB607B691B78272B03D07B69A3
S2140203801B78222B09D14FF00103FB727B691B7885
S214020390BB727B6903F101037B613B694FEA83030E
S2140203A03A68D3187A691A60FB7A83F00103DBB2E3
S2140203B0002B16D003E07B6903F101037B617B69A6
S2140203C01B78002B1AD07B691B78184616F03EFF66
S2140203D00346002BEFD111E07B6903F101037B6139
S2140203E000E000BF7B691B78002B04D07B691B787A
S2140203F0BA7A9A42F0D14FF00003FB727B691B78FF
S214020400002B07D07B694FF000021A707B6903F15C
S21402041001037B613B6903F101033B613B690F2BDF
S21402042088D9FB68184607F11807BD4680BD00BF8D
S21402043080B485B000AF786039604FF00003FB608F
S2140204404FF00003BB603B68002B17D14FF0000350
S2140204502BE0BA6813464FEA83039B184FEA43031E
S2140204601A467968FB68CB181B78D318A3F13003B9
S214020470BB60FB6803F10103FB6000E000BF7A6823
S214020480FB68D3181B78A3F13003092BE1D97A68ED
S214020490FB68D3181B78002B05D13B68BA681A6034
S2140204A04FF0010301E04FF00003184607F114076E
S2140204B0BD4680BC704700BF80B584B000AFF86010
S2140204C0B9607A60FB68032B23D1BB6803F104038F
S2140204D01B6818464DF2B071C0F2030116F062FEB8
S2140204E00346002B15D1BB6803F108031B681846A8
S2140204F04DF2B871C0F2030116F054FE0346002B0B
S21402050014BF00230123DAB27B681A704FF001038E
S21402051001E04FF00003184607F11007BD4680BD04
S21402052080B584B000AF786039607B68FB603B685A
S214020530002B13D1FB684FF00002C3F85822FB6869
S2140205404FF0000283F84D22FB6803F517724DF256
S214020550C073C0F203031B8813801FE038680BF0D9
S2140205607DFB0346002B16D0FB6803F24D2338684A
S21402057019464FF008020BF0A3FBFB683A68C3F873
S2140205805822FB6803F517724DF2C073C0F20303DC
S2140205901B88138002E04FF0010301E04FF00003D6
S2140205A0184607F11007BD4680BD00BF80B588B06B
S2140205B000AF786039604FF00003FB734FF0000322
S2140205C0BB613B683B6107F10F03786839681A46DE
S2140205D0FFF772FF0346FB77FB7F83F00103DBB274
S2140205E0002B00F084807B68012B35D13A694DF2EE
S2140205F0C473C0F2030353603A694DF2CC73C0F27F
S214020600030393603B694FF00002DA604DF2D47048
S214020610C0F203000BF088FC3B69D3F844327B61DE
S21402062015E07B691A683B691A604DF2EC70C0F2FD
S21402063003000BF079FC7B695B683A694FF00300B4
S21402064011469847B8617B6903F108037B617B69B1
S2140206501B68002BE5D14AE07B68022B44D13B683D
S2140206605A683B691A603A694DF2C473C0F20303D2
S21402067053603A694DF2F073C0F2030393603B692C
S2140206804FF00002DA603B69D3F844327B6117E030
S2140206903B681A687B691B681046194616F082FD8D
S2140206A00346002B08D17B695B683A694FF003006A
S2140206B011469847B86107E07B6903F108037B613E
S2140206C07B691B68002BE3D17B691B68002B0ED16C
S2140206D03B6803F104031B684DF2F870C0F2030096
S2140206E019460BF021FC02E04FF00103FB77FB7F7B
S2140206F0002B1BD0FB7B002B09D03B681B684DF6FA
S2140207002000C0F2030019460BF00EFC0EE03B6818
S2140207101B684DF63000C0F2030019460BF004FCCD
S2140207204DF64800C0F203000BF0FEFBBB6918460C
S21402073007F12007BD4680BD80B588B000AF78605F
S21402074039604FF00003FB724FF000033B613B68D9
S214020750FB6007F10B03786839681A46FFF7ACFEB0
S2140207600346FB77FB7F83F00103DBB2002B39D015
S2140207707B68012B33D14FF000037B61FB68D3F813
S2140207804432BB611BE0BB691B684DF67000C0F2C9
S214020790030019460BF0C8FB7B6903F00703072B1F
S2140207A005D14DF67800C0F203000BF0BDFB7B6965
S2140207B003F101037B61BB6903F10803BB61BB69FB
S2140207C01B68002BDFD17B6903F00703002B09D0DF
S2140207D04DF67800C0F203000BF0A6FB02E04FF0E5
S2140207E00103FB77FB7F002B15D0FB7A002B09D089
S2140207F03B681B684DF67C00C0F2030019460BF0FE
S21402080093FB08E03B681B684DF68000C0F20300CD
S21402081019460BF089FB3B69184607F12007BD46CF
S21402082080BD00BF80B400AFFEE700BF80B500AF5A
S2140208304DF69400C0F2030011F0AEF84FF000033C
S214020840184680BD80B489B000AF78600B46FB7056
S2140208507B68002B02D0FB78032B02D94FF00C03E7
S21402086035E2FA7813464FEAC3039B1A7A68D3181E
S2140208701B78BB61BB69092B02D94FF0160326E22F
S214020880BB694FEA43024DF6F403C0F20303D318E2
S2140208907B617B695B781946FA7813464FEAC30395
S2140208A09B1A7A68D3185B7803F004030B433B6108
S2140208B04FF0E023D3F8103D23F00603FB614FF020
S2140208C0E023FA69C3F8102D4FF46043C4F207031D
S2140208D04DF6F402C0F2030212785A7000BF4FF4CB
S2140208E05043C4F207039B78DBB203F00403002BE9
S2140208F0F5D000BF4FF46043C4F20703DB78DBB2E7
S214020900012BF7D1BB69042B12D14FF46043C4F21A
S21402091007034DF6F402C0F2030292795A7000BF42
S2140209204FF46043C4F20703DB78DBB2042BF7D143
S2140209303B6903F00103002B03D0FB6943F0040379
S214020940FB613B6903F00403002B03D0FB6943F011
S2140209500203FB614FF0E023FA69C3F8102DBB696E
S214020960062B55D14FF44043C4F20703F9780A46E2
S2140209704FEAC202521A79688A1892781A704FF4AD
S2140209804043C4F20703F9780A464FEAC202521AF3
S21402099079688A18D2785A704FF44043C4F2070333
S2140209A0F9780A464FEAC202521A79688A18127908
S2140209B09A704FF44043C4F20703F9780A464FEAA6
S2140209C0C202521A79688A185279DA704FF4404392
S2140209D0C4F20703F9780A464FEAC202521A796845
S2140209E08A1892791A714FF44043C4F207034FF003
S2140209F0FF025A714FF44043C4F207034FF0FF025E
S214020A009A714FF44043C4F207034FF0FF02DA71C3
S214020A10BB69072B05D0BB69082B02D0BB69092B23
S214020A2063D14FF44043C4F20703F9780A464FEA0B
S214020A30C202521A79688A1892781A704FF44043A2
S214020A40C4F20703F9780A464FEAC202521A7968D4
S214020A508A18D2785A704FF44043C4F20703F978E2
S214020A600A464FEAC202521A79688A1812799A70AE
S214020A704FF44043C4F20703F9780A464FEAC2022B
S214020A80521A79688A185279DA704FF44043C4F2DF
S214020A900703F9780A464FEAC202521A79688A1898
S214020AA092791A714FF44043C4F207034FF0FF02E3
S214020AB05A714FF44043C4F207034FF0FF029A7193
S214020AC04FF44043C4F207034FF0FF02DA714FF4CB
S214020AD04043C4F207034FF44042C4F20702927A3C
S214020AE0D2B242F00202D2B29A724FF48043C4F2F9
S214020AF006039B79DBB203F00C03FB604FF48043E2
S214020B00C4F206035B79DBB203F02003BB604FF44A
S214020B108043C4F206034FF48042C4F206025279BE
S214020B20D2B222F02002D2B25A714FF46043C4F21B
S214020B3007037A6912785A70BB69082B0BD0092B07
S214020B4011D0072B17D14FF46043C4F207034FF0BE
S214020B5003029A7010E04FF46043C4F207034FF0AA
S214020B6002029A7008E04FF46043C4F207034FF0A3
S214020B7001029A7000E000BFBB69032B08D100BFD8
S214020B804FF46043C4F20703DB78DBB2042BF7D1E1
S214020B903B6903F00203002B50D04FF4E043C4F24B
S214020BA004034FF4E042C4F2040202F5815202F159
S214020BB01C02126822F4805203F5815303F11C03CF
S214020BC01A604FF4E043C4F204034FF4E042C4F266
S214020BD0040202F5815202F11C02126822F400524B
S214020BE003F5815303F11C031A6030BF4FF4E04350
S214020BF0C4F204034FF4E042C4F2040202F5815246
S214020C0002F11C02126842F4805203F5815303F18A
S214020C101C031A604FF4E043C4F204034FF4E042AC
S214020C20C4F2040202F5815202F11C02126842F476
S214020C30005203F5815303F11C031A60BB69022BB1
S214020C400ED0BB69052B0BD0BB69062B08D0BB693F
S214020C50072B05D0BB69082B02D0BB69092B25D10F
S214020C60FB680C2B22D14FF48043C4F206039B7917
S214020C70DBB203F00C03082B18D14FF48043C4F206
S214020C8006034FF48042C4F206021278D2B202F091
S214020C903B02D2B21A7000BF4FF48043C4F206037E
S214020CA09B79DBB203F04003002BF5D04FF4804370
S214020CB0C4F206034FF48042C4F206025279D1B25D
S214020CC0BA68D2B20A43D2B25A714FF0000318463B
S214020CD007F12407BD4680BC704700BF80B400AF52
S214020CE04FF0E0234FF0E022D2F8102D22F002025D
S214020CF0C3F8102DBD4680BC704700BF80B483B0D9
S214020D0000AF4FF46043C4F207035B78DBB27B604C
S214020D104FF0E023D3F8103D03F004033B603B683A
S214020D20002B0CD17B6803F00703002B07D17B68EE
S214020D3003F0E003C02B02D04FF0010301E04FF0B6
S214020D400003184607F10C07BD4680BC704700BF7B
S214020D5080B485B000AF78604FF44043C4F2070316
S214020D605B79DBB2FB734FF44043C4F207039B7913
S214020D70DBB2BB734FF44043C4F20703DB79DBB24A
S214020D807B734FF44043C4F20703FA7BD2B25A7124
S214020D904FF44043C4F20703BA7BD2B29A714FF4BF
S214020DA04043C4F207031B7ADBB2DBB25BB2002B12
S214020DB00DDA4FF44043C4F207034FF44042C4F244
S214020DC00702127AD2B262F07F02D2B21A724FF4DD
S214020DD04043C4F207035B7ADBB2DBB25BB2002BA2
S214020DE00DDA4FF44043C4F207034FF44042C4F214
S214020DF00702527AD2B262F07F02D2B25A727B7B7A
S214020E00DBB24FEA03431A46BB7BDBB24FEA03234D
S214020E101A43FB7BDBB21A437B681A6007F114079E
S214020E20BD4680BC704700BF80B400AF4FF470432D
S214020E30C4F207031B78DBB203F00103002B02D0D7
S214020E404FF0010390E04FF47043C4F207031B789F
S214020E50DBB203F00203002B02D04FF0020383E062
S214020E604FF47043C4F207031B78DBB203F00403AB
S214020E70002B02D04FF0030376E04FF47043C4F227
S214020E8007031B78DBB203F02003002B02D04FF0DF
S214020E90040369E04FF47043C4F207031B78DBB225
S214020EA003F04003002B02D04FF005035CE04FF442
S214020EB07043C4F207031B78DBB2DBB25BB2002BD3
S214020EC002DA4FF006034FE04FF47043C4F2070312
S214020ED05B78DBB203F00103002B02D04FF007036E
S214020EE042E04FF47043C4F207035B78DBB203F0D0
S214020EF00203002B02D04FF0080335E04FF4704394
S214020F00C4F207035B78DBB203F00403002B02D0C3
S214020F104FF0090328E04FF47043C4F207035B78EE
S214020F20DBB203F00803002B02D04FF00A031BE0EB
S214020F304FF47043C4F207035B78DBB203F010038E
S214020F40002B02D04FF00B030EE04FF47043C4F2B6
S214020F5007035B78DBB2DBB25BB2002B02DA4FF040
S214020F600D0301E04FF000031846BD4680BC7047F3
S214020F7080B586B000AF02460B46FA71BB714FF0E1
S214020F8000037B614DF60810C0F203000EF0E4FF8A
S214020F9038613B69002B03D14FF012037B6124E0DA
S214020FA038690FF027F80346BB60FFF7A7FE034633
S214020FB0FB73B879B968FA7B4DF61813C0F20303CF
S214020FC04FEA400041184FEA41018A189B181B78E5
S214020FD0BB60BB68012B08D807F1080338691946BD
S214020FE04FF000020FF0AEFA78617B69184607F1FF
S214020FF01807BD4680BD00BF80B584B000AF7860DC
S2140210000B46FB707B68002B02D0FB78032B02D9C1
S2140210104FF00C0348E040F63473C1F6FF735A6A89
S21402102047F26D33C6F677439A4202D14FF0170362
S2140210303AE020484FF0010110F0F8FFF860FB6834
S214021040002B02D04FF02C032EE040F63473C1F68C
S214021050FF737A681A6040F63473C1F6FF73FA7843
S2140210601A7140F63473C1F6FF734FF000029A60AD
S21402107040F63473C1F6FF734FF00002DA6040F6B2
S2140210803473C1F6FF734FF0000283F82C2040F64B
S2140210903473C1F6FF7393F82C30FA78104619466B
S2140210A0FFF766FF4FF00003184607F11007BD462C
S2140210B080BD00BF440FFF1F80B588B000AFF86048
S2140210C0B9607A60FB68002B02D07B68002B02D1E5
S2140210D04FF00C038FE04A4811F054F9B861BB692F
S2140210E0002B02D04FF02C0385E04FF01C0012F0CC
S2140210F04BF978617B69002B05D1414811F08EF8D7
S2140211004FF0040377E0786940F21B4112F0E0F8F2
S21402111000BF40F63473C1F6FF73DB6803F10102C9
S21402112040F63473C1F6FF73DA6040F63473C1F6E4
S214021130FF73DB68002BECD07B694FF000021A606D
S2140211407B694FF000025A607B6903F10803184678
S214021150F9684FF00C0216F016F87B69BA685A6105
S21402116040F63473C1F6FF73DA687B699A6140F61B
S2140211703473C1F6FF739B68FB6126E07B691A69CC
S214021180FB691B699A4212D27B69FA695A60FB694B
S2140211901B68002B07D0FB691B687A695A60FB69DB
S2140211A01A687B691A60FB697A691A6010E0FB6943
S2140211B05B68002B06D1FB697A695A607B69FA691B
S2140211C01A6005E0FB695B68FB61FB69002BD5D101
S2140211D07B691B68002B05D140F63473C1F6FF739A
S2140211E07A699A607B699A697B681A60044811F08A
S2140211F015F84FF00003184607F12007BD4680BDDC
S214021200440FFF1F80B582B000AF0B4811F0BAF84A
S21402121078607B68002B02D04FF0FF0307E001F0F6
S2140212202FFC0346FB70044810F0F8FFFB781846C4
S21402123007F10807BD4680BD440FFF1F80B586B084
S21402124000AF0346FB71FB79032B02D94FF00C0368
S2140212508AE0484811F096F838613B69002B02D0C4
S2140212604FF02C0380E001F00BFC0346FB7340F6C4
S2140212703473C1F6FF739B687B6124E07B69DB688D
S214021280002B19D04FF000033B73FB7BBB73FB793B
S2140212907B737B69DB687A69526907F10C01084641
S2140212A0114698470346002B06D04FF02C033B61AD
S2140212B07B691B687B610BE07B695B68002B06D051
S2140212C07B695B687B617B69002BD7D100E000BF3E
S2140212D03B69002B22D140F63473C1F6FF731A68BD
S2140212E0FB7910461946FFF7ADFA38613B69002BC9
S2140212F014D140F63473C1F6FF73FA791A7140F6C8
S2140213003473C1F6FF731A7940F63473C1F6FF736D
S21402131093F82C3010461946FFF72AFE3B69002B3D
S2140213201ED01AE07B69DB68002B13D04FF0000357
S2140213303B73FB7BBB7340F63473C1F6FF731B79BA
S2140213407B737B69DB687A69526907F10C01084690
S214021350114698477B691B687B617B69002BE1D14C
S214021360044810F05BFF3B69184607F11807BD46B4
S21402137080BD00BF440FFF1F80B582B000AF0C488F
S21402138011F000F878607B68002B02D04FF0FF0364
S21402139009E040F63473C1F6FF731B79FB7004480C
S2140213A010F03CFFFB78184607F10807BD4680BDE3
S2140213B0440FFF1F80B584B000AFF8600B467A601A
S2140213C0FB7240F63473C1F6FF731B6803F1150314
S2140213D01B78062B15D1F86841F20D41C0F20201C6
S2140213E04FF0000212F00AFEFB7AF86819464FF038
S2140213F001020AF09DFA40F63473C1F6FF737A686A
S2140214001A6307F11007BD4680BD00BF80B584B0E1
S21402141000AF786007F10C031846FFF799FC40F618
S2140214203473C1F6FF731B6B002B07D040F6347380
S214021430C1F6FF731B6BFA681046984707F1100750
S214021440BD4680BD80B400AF4FF00F031846BD46C0
S21402145080BC704780B584B000AFF860B9607A602F
S2140214603B60FB68002B02D0BB68002B02D14FF01A
S2140214700C0334E0BB681B68002B02D14FF001035B
S2140214802DE0FB68BA681A60F9684FF000024FF068
S2140214900003C1E90423FB684FF000029A60FB6870
S2140214A04FF000025A60FB684FF00002DA60FB68F9
S2140214B04FF000029A61FB684FF00002DA61FB68A7
S2140214C04FF000021A62FB684FF000025A62FB6895
S2140214D01B681B68F86879683A6898470346184696
S2140214E007F11007BD4680BD80B584B000AF7860B6
S2140214F07B68002B03D07B681B68002B02D14FF061
S2140215000C0346E07B681B685B68002B02D14FF039
S21402151001033EE07B681B681B6978689847F860A1
S214021520FB68002B01D0FB6833E07B681B685B68B6
S21402153078689847F860FB68002B01D0FB6828E0C3
S2140215407B684FF000021A6079684FF000024FF095
S2140215500003C1E904237B684FF000025A607B68EF
S2140215604FF000029A607B684FF00002DA607B68F8
S2140215704FF000029A617B684FF00002DA617B68E6
S2140215804FF000021A627B684FF000025A624FF078
S2140215900003184607F11007BD4680BD80B586B029
S2140215A000AFF860B9607A60FB68002B06D0FB6873
S2140215B01B68002B02D07B68002B02D14FF00C0375
S2140215C027E0FB681B689B68002B02D14FF00103E3
S2140215D01FE0FB68BA685A6001F00EFA03461A4624
S2140215E0BB68DBB21046194601F00EFA38613A695A
S2140215F07B68B2FBF3F37B617B69002B02D14FF071
S21402160001037B61FB681B689B68F86879699847E9
S2140216100346184607F11807BD4680BD80B582B05E
S21402162000AF78607B68002B03D07B681B68002BBA
S21402163002D14FF00C030DE07B681B68DB68002BC1
S21402164002D14FF0010305E07B681B68DB6878680F
S21402165098470346184607F10807BD4680BD00BFF7
S21402166080B483B000AF78607B68002B02D14FF065
S214021670000301E07B68DB68184607F10C07BD46ED
S21402168080BC704780B582B000AF786039607B68F6
S214021690002B06D07B681B68002B02D03B68002B11
S2140216A002D14FF00C030EE07B681B685B69002BCF
S2140216B002D14FF0010306E07B681B685B6978681D
S2140216C0396898470346184607F10807BD4680BDA5
S2140216D080B487B000AFF860B9607A60FB68002B10
S2140216E002D14FF00C0311E0FB687B617B694FF07F
S2140216F000029A617B694FF000021A627B697A687F
S214021700DA617B69BA689A614FF00003184607F1FE
S2140217101C07BD4680BC704780B485B000AF7860B9
S2140217207B681B685B68FB60FB68002B07D0FB6866
S2140217301B6843F04002FB681A6000BF00E000BF6F
S21402174007F11407BD4680BC704700BF80B586B05F
S21402175000AF78604FF00F033B617B681B78194639
S21402176040F66872C1F6FF720B464FEA43035B18F7
S2140217704FEAC303D3181B68002B15D07B681B786F
S214021780194640F66872C1F6FF720B464FEA4303EB
S2140217905B184FEAC303D31803F104031B68002B3C
S2140217A002D04FF0000303E27B681B78184600F075
S2140217B01BFBF860FB68002B02D14FF00003F7E139
S2140217C07B681B78184600F025FF7B681B781A4654
S2140217D013464FEA43039B184FEAC30340F6687268
S2140217E0C1F6FF729B18BB60BB68FA685A60BB689A
S2140217F04FF00002DA607B685A69BB681A61BB6800
S2140218004FF480325A614FF00003FB75BB685B6988
S214021810B3F5806F0DD0B3F5806F03D8B3F5807F34
S21402182007D00BE0B3F5805F03D0B3F5803F08D056
S21402183004E0FB7D43F00103FB7503E04FF0000379
S214021840B6E100BF7B68DB78002B03D1FB7D43F05B
S2140218500203FB757B681B79002B03D1FB7D43F0EB
S2140218600403FB75FA7D4DF62013C0F2030353F80A
S214021870222047F21873C1F6FF731A607B685B7802
S214021880042B00F2718101A252F823F0C51902005E
S214021890911A0200A1180200151B02003F1B02004B
S2140218A07B689B785BB2B3F1FF3F52D147F2187365
S2140218B0C1F6FF731A6848F2FF63C0F293339A4286
S2140218C004D9FB684FF000029A6051E147F21873A0
S2140218D0C1F6FF731A684CF27F33C0F2C9139A42FC
S2140218E004D9FB684FF020029A6041E147F2187370
S2140218F0C1F6FF731A684EF2BF13C0F2E4039A42AF
S21402190004D9FB684FF040029A6031E147F218733F
S214021910C1F6FF731A6847F2DF03C0F272039A42F7
S21402192004D9FB684FF060029A6021E147F218730F
S214021930C1F6FF731A6843F66F03C0F239039A4280
